:100000000C94480E0C9400000C9400000C9400001A
:100010000C9400000C9400000C9400000C94BA5A4C
:100020000C9400000C9400000C94D5160C94000065
:100030000C9400000C9400000C9400000C94000040
:100040000C9493160C9400000C947E570C940000B2
:100050000C94B8570C9400000C9400000C94000011
:100060000C9400000C9400000C9400000C94000010
:100070000C9400000C9400000C9414590C94000093
:100080000C94585A0C9400000C94000000000100DD
:100090000200040008001000200040008000000161
:1000A0000002000400080010002000400080000151
:1000B00002040810204080005F4944000000000056
:1000C000000000000000590B8000100000005F528B
:1000D000733233324944000000000000590B8200A3
:1000E0001F0000005F526F74617465000000000023
:1000F0000000590B8100030000005F5461737465B8
:100100006E58000000000000590B010004000300BD
:100110005F54617374656E590000000000005A0B53
:100120000100060005005F44656661756C744B65EF
:10013000790000005C0B0100800000002A436F641E
:1001400065300000000000000000630B02000F2774
:1001500000002A436F6465310000000000000000C9
:100160005D0B02000F2700002A436F646532000018
:100170000000000000005F0B02000F27D0122A4D84
:1001800061784D6F64756C0000000000610B010028
:10019000100000002A5469736368450000000000E5
:1001A0000000620B0000010000005F4D7954657291
:1001B0006D4E720000000000650B01000800010098
:1001C0005F4D61737465725465726D730000660BE8
:1001D0000300080001005F454D6F646500000000EA
:1001E00000000000670B0300060000005F4543723B
:1001F000656457747200000000007D0B01007F00F1
:100200003F005F5273304D6F6465000000000000D6
:100210007C0B0100030000005F5634756E643500EE
:10022000000000000000680B0000010000005F50AB
:10023000756C736554696D65000000007B0B0100EF
:1002400064001E005F506175736554696D65000040
:100250000000B00B0100640000005F41736B43724B
:100260006564697400000000690B00000100000073
:100270005F53656E644465626974000000006A0B38
:100280000000010000005F4372656469744D6F6493
:10029000650000007A0B0100020000005F437265F8
:1002A0006469744D6173746572006B0B000001002A
:1002B00000002A5461626C6553746172740000001E
:1002C0006C0B02000F2700002A5461626C65456EBA
:1002D0006400000000006E0B02000F27E7032A4AAB
:1002E0006F6231000000000000000000700B03008E
:1002F000080001002A4A6F6232000000000000007E
:100300000000710B0300080000002A4A6F623300EE
:100310000000000000000000720B03000800000055
:100320002A4A6F6234000000000000000000730BD6
:100330000300080000002A4A6F6235000000000038
:1003400000000000740B0300080000002A4A6F62DE
:1003500036000000000000000000750B03000800DC
:1003600000002A4A6F623700000000000000000011
:10037000760B0300080000005F4572726F72310057
:100380000000000000007E0B04000A002E005F4504
:1003900072726F723200000000000000880B0400CF
:1003A0000A002E005F4572726F7233000000000079
:1003B0000000920B04000A002E005F4572726F72FB
:1003C00034000000000000009C0B04000A002E0016
:1003D0005F4572726F723500000000000000A60BCE
:1003E00004000A002E0000000000000000000000D1
:1003F000000000000000FF00000000005461737462
:1004000065722020000000024C69745A20202020D0
:10041000000004044C656974542020200000080783
:1004200050756C732020202000000C0550756C73F3
:100430002030202000008C0654617374203020206E
:100440000000800973657269656C6C200000100BF8
:1004500073657269656C20320000500C54617374CE
:1004600020322020000040035461737420706172B8
:100470000000140A466F6C676554202000001808BD
:100480003F3F3F3F3F3F2020000000022800600028
:100490009800D00008014001210C5800002D0B2DC0
:1004A00000002B0B2B00004D0A4D0000800E563132
:1004B00000810E563200820E563300830E563400F1
:1004C000210C580000840E563500310B312041427A
:1004D000430000320B32204445460000330B3320EA
:1004E00047484900004D0A4D000000000000340B51
:1004F00034204A4B4C0000350B35204D4E4F000048
:10050000360B362050515200002B0A2B0000000001
:100510000000370B37205354550000380B38205655
:1005200057580000390B3920595A2F00002D0A2D39
:10053000000000000000430C4300000000000030F9
:100540000B3020202E2C00002C0A2C000000000074
:10055000003D0A435200000000000000A0001B0004
:10056000006605D700A0001A0200660569000000B9
:10057000180400680569001E01190600680550721C
:100580006F64756B74200000537061727465202075
:100590000000706F7274696F6E696572656E00003D
:1005A0002E666F6C67650000506F7274696F6E65C0
:1005B0006E207369636865726E003000436865661B
:1005C0002D4D656E7500000031004B206C69737411
:1005D000656E0000000032004B206C6F657363682D
:1005E000656E000033004B20647275636B656E00AE
:1005F0000000340054206C697374656E00000000C4
:10060000350054206C6F65736368656E00003600BA
:100610005420647275636B656E0000004600537968
:100620007374656D0000000000004100506F72742B
:10063000696F6E000000000043004B7265646974CE
:1006400065000000000044004B7265642E436C722C
:10065000000000004A006D616E2E506F7274696F69
:100660006E0000000000000000000000000000001C
:10067000300053797374656D00000000000037008E
:1006800054657374000000000000000039005061E0
:1006900072616D65746572000000380050726F649D
:1006A000756B74650000000042004B656C6C6E65F4
:1006B000720000000000450056656E74696C6500AC
:1006C000000000006300436F6C6F72730000000055
:1006D000000000000000000000000000000000001A
:1006E0004572726F72200000000000000000C40B11
:1006F0000000050000004F70742E20200000000054
:1007000000000000C70B000003000000496D707579
:100710006C732000000000000000C50B0000050005
:10072000000054696D654F757420000000000000E2
:10073000C60B0000140000002E202C304142433133
:1007400044454632474849334A4B4C344D4E4F3569
:10075000505152365354553756575838595A2F39E5
:100760000500C11100000300D90B00000300C111F6
:100770000300170E0300D90B00000500E00800007D
:100780000A00C1110A00170E0A00D90B0A00C11194
:100790000A00170E2800D90B00000000F800000026
:1007A000FF000000FF0000007F80001E0F80007F20
:1007B000E7C0007FFFE0003FFFE00007FFC000014F
:1007C000FFC00001FF800001FF0003FFFE0007FFE4
:1007D000FC0007FFF00003FFF00003FFFE00001F16
:1007E000FFC001FFFFF001FFFFF801FFFFF8007FEE
:1007F000FFF80007FE00003FFF00007FFF80007F42
:10080000FF80007FC100001FE000001FF000001FFC
:10081000F000000FE0000007C0000007C000000764
:10082000C000000780000003000000030000000279
:10083000000000000000000000000000E0000000D8
:1008400000000003900000000000000E18000000EF
:100850000000003808000000000000C01800000080
:10086000000003807000000000000C01C0000001C7
:100870008006300700000003C00F401C0000000687
:10088000E01DC0700000000C3039C1C0000000182D
:100890001871C7180000001C0CE1DC7C0000000E81
:1008A00007C3F1C400000007038607060000000329
:1008B000800E1C0200000001C01C3003000000007C
:1008C000E03818010080000070700FC183C0000084
:1008D00038E003E08E6006001DC00020FC200F0001
:1008E0000F8000307030198007000010003030C0D9
:1008F0000000001800E06060000000080380603025
:100900000000000C0E003018000000043800180C25
:1009100000000006E0000C06000000038000060353
:1009200000000000000003018000000000000180C2
:10093000C000C0C060C030C030C030C030C030C0A7
:1009400030C030C030C030C030E030703018300CB3
:1009500030043FFC3FFC00000000000000000000ED
:100960000000000000000000000000000000000087
:10097000000000000000070018C0202020204D903B
:100980004D9040104010489047102020202018C063
:1009900007000000000007001FC03FE03FE072704A
:1009A00072707FF07FF0777078F03FE03FE01FC01B
:1009B00007000000000000000000000018C03DE03B
:1009C0003FE03FE03FE01FC00F8007000200000053
:1009D000000000000000000000000000020007000E
:1009E0000F801FC03FE01FC00F8007000200000003
:1009F0000000000000000000000007000F800F80D2
:100A00000F8037607FF07FF07FF0326007000F804B
:100A100000000000000000000000020002000700CB
:100A20000F801FC03FE03FE03FE01AC007000F808B
:100A300000000000000000000000000000000000B6
:100A4000000006000F000F0006000000000000007C
:100A5000000000000000FFF0FFF0FFF0FFF0FFF0EB
:100A6000FFF0F9F0F0F0F0F0F9F0FFF0FFF0FFF038
:100A7000FFF0FFF0FFF000000000000000000600A3
:100A8000090010801080108010800900060000000E
:100A9000000000000000FFF0FFF0FFF0FFF0F9F0B1
:100AA000F6F0EF70EF70EF70EF70F6F0F9F0FFF026
:100AB000FFF0FFF0FFF000000000000001E0006028
:100AC0001EA0332061806180618033001E00000021
:100AD0000000000000000000000007800CC018604B
:100AE000186018600CC00780030003000FC00300EB
:100AF00003000000000002000300038003C002C0E6
:100B000002C00280020002000E001E001E000C0047
:100B10000000000000000C000E000B0009800CC05B
:100B20000E400B4009C038C07840784031C003C047
:100B300003C00180000000000200020027201FC047
:100B400018C030607070306018C01FC027200200CD
:100B500002000000000000000000100018001C004F
:100B60001E001F001F801F001E001C001800100028
:100B700000000000000000000000008001800380F1
:100B800007800F801F800F80078003800180008016
:100B90000000000000000000020007000F801FC0DE
:100BA000020002000200020002001FC00F800700C6
:100BB00002000000000000001980198019801980CF
:100BC00019801980198019801980198000001980F6
:100BD00019800000000000001FE036C066C066C03B
:100BE00066C036C01EC006C006C006C006C006C02D
:100BF00006C00000000000001F8030C03000300040
:100C00001F8030C030C01F8000C000C030C01F80B7
:100C100000000000000000000000000000000000D4
:100C20000000000000000000000000001FE01FE0C6
:100C30001FE000000000020007000F801FC002003C
:100C4000020002000200020002001FC00F80070025
:100C500002001FC000000000020007000F801FC03C
:100C60000200020002000200020002000200020074
:100C7000020000000000000002000200020002006A
:100C8000020002000200020002001FC00F800700E5
:100C90000200000000000000000000000000010051
:100CA000018001C03FE001C00180010000000000A0
:100CB0000000000000000000000000000000040030
:100CC0000C001C003FE01C000C00040000000000B1
:100CD0000000000000000000000000000000000014
:100CE00000000000000040004000400040004000C4
:100CF0007FE000000000000000000000000008800D
:100D000018C038E07FF038E018C00880000000000C
:100D100000000000000000000000000000000000D3
:100D2000020007000F801FC03FE07FF000000000BE
:100D300000000000000000000000000000000000B3
:100D40007FF03FE01FC00F8007000200000000009E
:100D50000000000000000000000000000000000093
:100D60000000000000000000000000000000000083
:100D7000000000000000060006000F000F000F003A
:100D80000F000F000600060006000000000006002D
:100D90000600000000000000000019801980198082
:100DA00019800000000000000000000000000000AA
:100DB00000000000000000000660066006603FF0D2
:100DC0000CC00CC0198019807FC033003300330081
:100DD000000000000000060006001F803FC0360033
:100DE00036003F801FC006C006C03FC01F800600FF
:100DF00006000000000000000000001038303870CD
:100E000038E001C0038007000E001C0038E070E0ED
:100E100060E000000000000007000D8019801980CC
:100E20001B000E001E003E00336033C031803BC00B
:100E30001E60000000000E000E000E0006000600FE
:100E40000C00000000000000000000000000000096
:100E5000000000000000038006000E000C001C00D3
:100E60001C001C001C001C001C000C000E000600D6
:100E70000380000000001C00060007000300038040
:100E800003800380038003800380030007000600C3
:100E90001C000000000000000000000036C036C04A
:100EA0001F800F003FC00F001F8036C036C00000FB
:100EB000000000000000000000000000000006002C
:100EC000060006003FC03FC0060006000600000006
:100ED0000000000000000000000000000000000012
:100EE0000000000000000000000000000E000E00E6
:100EF0000E0006000C0000000000000000000000D2
:100F0000000000003FC03FC00000000000000000E3
:100F100000000000000000000000000000000000D1
:100F20000000000000000000000000000E000E00A5
:100F30000E0000000000000000100030007000E013
:100F400001C0038007000E001C0038007000600024
:100F50000000000000000F803FE03060607060F033
:100F600061B0633066306C307830703030603FE0B4
:100F70000F8000000000030007001F001F00030097
:100F800003000300030003000300030003001FE04D
:100F90001FE0000000001FC03FE070706030607014
:100FA00000E001C0038007000E001C0038007FF045
:100FB0007FF0000000001FC03FE070706030003024
:100FC00000700FE00FC000600030603070703FE0D4
:100FD0001FC00000000001C003C007C00EC01CC03D
:100FE00038C070C060C07FF07FF000C000C000C09B
:100FF00000C0000000007FF07FF060006000600033
:101000007FC03FE0007000300030603070703FE023
:101010001FC00000000003C007C00E001C00380005
:1010200030007FC07FE070706030603070703FE0F3
:101030001FC0000000007FF07FF00060006000C073
:1010400000C00180018003000300060006000C00C0
:101050000C00000000000F801FC038E030603060DE
:1010600038E01FC03FE070706030603070703FE06B
:101070001FC0000000001FC03FE070706030603093
:1010800070703FF01FF0006000E001C003801F009F
:101090001E000000000000000000000000000E0024
:1010A0000E000E000000000000000E000E000E00FA
:1010B00000000000000000000000000000000E0022
:1010C0000E000E000000000000000E000E000E00DA
:1010D000060006000C0000C001C0038007000E00DF
:1010E0001C00380038001C000E000700038001C0FF
:1010F00000C0000000000000000000000000000030
:101100003FE03FE0000000003FE03FE00000000063
:10111000000000000000300038001C000E00070036
:10112000038001C001C0038007000E001C003800CE
:101130003000000000001F803FC070E0606060E091
:1011400001C003800700060006000600000006003C
:101150000600000000001FC03FE0306067B06FB0C5
:101160006DB06DB06DB06DB06FE067C070003FC026
:101170000FC000000000060006000F000F000F0067
:1011800019801980198030C03FC03FC06060606026
:101190006060000000007F007F8061C060C060C0B0
:1011A00061C07F807FC060E06060606060E07FC0A1
:1011B0007F80000000000F801FC038E030606000BA
:1011C00060006000600060006000306038E01FC0B8
:1011D0000F80000000007F007F8061C060C0606001
:1011E0006060606060606060606060C061C07F80FF
:1011F0007F00000000007FE07FE060006000600092
:1012000060007F807F8060006000600060007FE0A1
:101210007FE0000000007FE07FE060006000600091
:1012200060007F807F806000600060006000600080
:101230006000000000000FC01FE038603000600058
:10124000600063E063E060606060306038601FE011
:101250000FE00000000060606060606060606060DF
:1012600060607FE07FE06060606060606060606040
:101270006060000000001F801F800600060006005E
:1012800006000600060006000600060006001F8095
:101290001F800000000000600060006000600060CF
:1012A00000600060006000606060606070C03FC00F
:1012B0001F8000000000606060E061C06380670024
:1012C0006E007C007C006E006700638061C060E09F
:1012D000606000000000600060006000600060006E
:1012E00060006000600060006000600060007FE0FF
:1012F0007FE000000000606070E070E079E079E07D
:101300006F606F60666066606060606060606060B3
:1013100060600000000060607060706078606C6009
:101320006C60666066606360636061E060E060E01E
:101330006060000000000F001F8039C030C0606096
:101340006060606060606060606030C039C01F8055
:101350000F00000000007F807FC060E06060606080
:10136000606060E07FC07F806000600060006000BF
:101370006000000000000F001F8039C030C06060B6
:101380006060606060606060636033C039C01FE0AF
:101390000F60000000007F807FC060E060606060E0
:1013A000606060E07FC07F806700638061C060E054
:1013B0006060000000001F803FC070E0606060005F
:1013C00070003F801FC000E00060606070E03FC0C0
:1013D0001F80000000003FC03FC00600060006005E
:1013E00006000600060006000600060006000600CD
:1013F0000600000000006060606060606060606027
:1014000060606060606060606060606030C03FC06D
:101410001F800000000060606060606030C030C00D
:1014200030C01980198019800F000F000F000600CE
:1014300006000000000060606060606060606060E6
:1014400060606060666066606F6079E070E070E0C8
:101450006060000000006060606030C030C01980D3
:101460000F00060006000F00198030C030C0606019
:101470006060000000006060606030C030C01980B3
:1014800019800F000F000600060006000600060087
:101490000600000000007FE07FE000C000C0018087
:1014A0000300060006000C001800300030007FE04A
:1014B0007FE000000000666066600F000F000F0014
:1014C00019801980198030C03FC03FC060606060E3
:1014D0006060000000006F605FA039C030C06060D5
:1014E0006060606060606060606030C039C01F80B4
:1014F0000F000000000060606060000060606060DD
:1015000060606060606060606060606030C03FC06C
:101510001F80000000001F801F80180018001800A6
:1015200018001800180018001800180018001F8074
:101530001F8000000000000000000000000000000C
:10154000000000000000000000000000000000009B
:1015500000007FF07FF00000070007000700060092
:101560000600030000000000000000000000000072
:10157000000000000000000000000000000000006B
:101580001FC03FE000601FE03FE0606060607FE000
:101590003FE000000000600060006000600060004C
:1015A0006F807FC070E060606060606060E07FC0FE
:1015B0007F8000000000000000000000000000002C
:1015C0001F803FC0706060006000600070603FC0BE
:1015D0001F8000000000006000600060006000608C
:1015E0001F603FE071E060606060606070603FE0DD
:1015F0001FE00000000000000000000000000000EC
:101600001F803FC070607FE07FC0600070003FC0FF
:101610001F800000000007800F801C0018001800C9
:1016200018007F007F00180018001800180018002C
:101630001800000000000000000000000000000092
:101640001FE03FE07060606070E03FE01F6000609E
:1016500000E03FC03F80600060006000600060000C
:101660006F007F8071C060C060C060C060C060C03B
:1016700060C000000000000000000600060000003E
:101680000E000E00060006000600060006001F8081
:101690001F800000000000000000018001800000A9
:1016A000038003800180018001800180018001802E
:1016B00019801F800F0030003000300030003000F3
:1016C0003180338037003E003E003700338031C028
:1016D00030C0000000000E000E00060006000600EC
:1016E00006000600060006000600060006001F8031
:1016F0001F8000000000000000000000000000004B
:1017000059807FC07FE06660666066606660666084
:101710006660000000000000000000000000000003
:101720003F803FC030E0306030603060306030601B
:101730003060000000000000000000000000000019
:101740001F803FC070E060606060606070E03FC01C
:101750001F800000000000000000000000000000EA
:101760007F807FC060E06060606070E07FC06F80FD
:101770006000600060000000000000000000000049
:101780001FE03FE070606060606070E03FE01F60FD
:101790000060006000600000000000000000000029
:1017A00037C03FE03860300030003000300030009B
:1017B00030000000000000000000000000000000F9
:1017C0003F007F8060007F003F80018001807F803C
:1017D0003F0000000000000018001800180018006A
:1017E0007F007F00180018001800180018001F80E4
:1017F0000F8000000000000000000000000000005A
:1018000060606060606060606060606070E03FE0E9
:101810001F60000000000000000000000000000049
:101820006060606030C030C0198019800F000F0008
:1018300006000000000000000000000000000000A2
:10184000666066606660666066606F603FC039C0F3
:1018500010800000000000000000000000000000F8
:1018600060C071C03B801F000E001F003B8071C034
:1018700060C0000000000000000000000000000048
:1018800030C030C0198019800F000F00060006001C
:101890000C000C0018000000000000000000000018
:1018A0007FC07F80030006000C00180030007FC05E
:1018B0007FC0000000000000000060600000000029
:1018C0001FC03FE000601FE03FE0606060607FE0BD
:1018D0003FE0000000000000000060600000000029
:1018E0001F803FC070E060606060606070E03FC07B
:1018F0001F80000000000000000060600000000089
:1019000060606060606060606060606070E03FE0E8
:101910001F600000000000003F007F8060C060C0CA
:1019200061C0678067C060E06060606060E067C061
:1019300067800000000000000000000000000600BA
:101940000F00198030C0606060607FE07FE00000C1
:1019500000000000000000001E0060077E0700F08D
:101960001EF060F77EF7FBDE1F00E007FF0700F8C0
:101970001FF8E0FFFFFF58002B003E3E006E656938
:101980006E006A61006B65696E204B7265646974F4
:10199000002000436F6C6F72546F7563682056733C
:1019A00020312E333100426C6F636B2000202047C2
:1019B000433D00546573740020204B653A0020209D
:1019C000496E3A0043616C6962726174696F6E00BE
:1019D0004F4B00546F74616C0054696E7920005451
:1019E000696E7920626164006B65696E204545709F
:1019F000726F6D004D4F44554C2053544F5000446E
:101A00006174612000696E697400533F0000666173
:101A10006C7363686572205469736368200054694D
:101A200073636820766F6E204B20004665686C6596
:101A300072200056656E74696C20616B7469760063
:101A400054696D656F757400435349204E722000D0
:101A5000436F646520006B65696E204B7265646935
:101A6000740058313939313030004D420050530044
:101A7000504C5520203A00436F6465203A00546969
:101A8000736368203A004B656C6C6E657220004D84
:101A900031004F31005350004350004459006275EB
:101AA0007379004D50002067657370657272740021
:101AB000256400004162726563686E756E67004B55
:101AC000656C6C6E65722000546F74616C004D6FB4
:101AD00064756C2000202000433F006E65696E0035
:101AE0006A6120200073656300496D7000504C5599
:101AF0003A20005370617274653A20005072313A96
:101B000020005072323A20005365697465203A20F3
:101B1000005479703A20003A20563A2020302B2089
:101B200030003A003A20544F3A200053703A004BAC
:101B30002066726569204A6F62204A6F62466C6156
:101B40006773004B20006672656920004A6F62204F
:101B50002000562020204572722050676C20496D6D
:101B60007020544F005620004B656C6C6E65723AC5
:101B7000004D49004D42004D43004D50004D4C007A
:101B800074657374202E2E004F4E0000253032589D
:101B90000025303458002533642E2530326400256A
:101BA0003564002564002532640025336400444414
:101BB00000004B23004253004221004246005423C0
:101BC00000544F004952004D5A0042510042520009
:101BD0004353004266004B23005423004245004318
:101BE00045004241004453005643004343004342F2
:101BF0000023502241534349492D492F4F222C2283
:101C0000312E3030222C323030382D30312D3031E1
:101C10003B0023482245636F222C22312E30302294
:101C20002C323030382D30312D30313B00235322CF
:101C300045636F222C22312E3030222C3230303846
:101C40002D30312D30313B00504F00504632333B68
:101C50005055002564002B302B303B0025640025B7
:101C600030325800253130640025642E253264005E
:101C70004F4E00006D696B726F746F756368000082
:101C800001002D4E414E00000100860E801C000018
:101C9000F894EE27ECBBF1E0F5BFE5BFE0936C00F4
:101CA000F8E1F1BDE1BD8DE0A2E0BB27ED938A959F
:101CB000E9F780E090E1A0E0B1E0ED930197E9F76A
:101CC000E8E8FCE185919591009761F0A591B591C7
:101CD00005901590BF01F00105900D920197E1F775
:101CE000FB01F0CFEFEFEDBFE0E1EEBFC0E0D3E0EE
:101CF0000C94E8170A9902C0E1E00895E0E0089525
:101D00001A93E0E0EA930E94261AE1E0E093310B97
:101D1000E0E0EA930E944B1A11E0153080F41A9328
:101D20000E94261AE4E6F0E0E0933B0BF0933C0BB4
:101D30001093350B1A930E944B1A1F5FEECF08C108
:101D40001A931FEFE2E00E94296A0E943C6A0E94F7
:101D50002960E03091F4E981EE0FE0520E94416A7F
:101D600041F4EDB7FEB7FA93EA931F930E94466AD7
:101D70001F910E943A600E944A6AE0E0E09371007D
:101D80000E944A6AE12FA8C30E944F6A10E01430F3
:101D9000E0F400E00430B8F4A12FECE30E94536AB1
:101DA0000E94576AE15BFF4FFA93EA930E94606AD0
:101DB0000E94606AE02FEE0FEE0FE10FEA930E949F
:101DC00006640F5FE7CF1F5FE2CF0E94656AE4EB16
:101DD000F0E00E946C6A0E94F2460E94846A0E94AF
:101DE000AB40E030E9F40E948B6A0E948B6AE6E91E
:101DF000F0E00E94906A0E94976A0E948B6A0E949B
:101E00008B6A0E9453440E949B6A0E94263F0E9454
:101E1000A26A0E94263FEEE1F0E00E94A96ADFCFAD
:101E20000E94AE400991199108950895E881E0302B
:101E300011F01C9A01C01C98219608950E948B6A8B
:101E40000E948B6A0E94AD6AEFE3F0E00E94B26AE2
:101E50000895A0910403A43011F00C947F0FE09139
:101E6000FC03E093FD030E948B6A0E94B56AE1E2E5
:101E7000EA930E948B6A0E948B6A0E944D410E94E5
:101E8000C26AEDE4EA930E948B6A0E948B6A0E9408
:101E90004D41E6E9F0E0FA93EA930E94B56AE4E581
:101EA000EA930E948B6A0E948B6A0E944D41E1EE88
:101EB000F0E0FA93EA930E94B56AEDE3EA930E9498
:101EC0008B6A0E948B6A0E94C76A0E948B6A0E947A
:101ED000CE6AEDE2EA930E948B6A0E948B6A0E94AE
:101EE000C76AE0EAF0E0FA93EA930E94CE6AEBE276
:101EF000EA930E948B6A0E948B6A0E944D4108956A
:101F00001A93A7DFA0910403A43001F1E0E0E0936D
:101F1000FD0310E01430D0F40E94D76A0E94DD6AFD
:101F2000FA93EA93EBE0F1E00E94E96A0E94E96A21
:101F3000FA93EA930E94D76AE491EA930E94D76ADF
:101F40000E94EE6A0E944D411F5FE4CF0E94F26A38
:101F5000199108950E94047CE0E0E093FD0330E0D5
:101F600010E000E03630F8F40E94F86A0E94DD6A62
:101F70000E94576AE153FF4F0E94E96A0E94E96A92
:101F8000FA93EA930E94F86AE491EA930E94F86A4D
:101F90000E94EE6A0E944D411F5F143011F410E060
:101FA0000F5F3F5FDFCF0E94F26A0E940B7C4BC342
:101FB0000E94FE6A0E94656AE9EBF0E00E946C6A8A
:101FC000EBE0E093FC03E0E0E093FD030E94026B92
:101FD0000E94076BEAEAF0E00E940C6BE091CF0BE5
:101FE000F091D00BE491EA93E091CF0BF091D00BFC
:101FF0000E94EE6A0E944D4101E00E94136B0E9414
:10200000166B11F00F5FF9CF0E94256B031718F4C0
:10201000E0E0E093B5050E94256B11E00E942C6B77
:102020000E94166B11F0153008F020C00E94026B60
:102030000E942F6BE0E4F0E00E947C793496FA93E2
:10204000EA93E2EEF0E00E940C6B0E942C6B0E947F
:10205000326BE491EA930E942C6B0E94326B0E94D7
:10206000EE6A0E944D413F5F1F5FD8CFF2DE62C033
:1020700023970E94047C30E010E0143088F500E0E3
:10208000043060F50E943E6B0E94446B0E943E6BE0
:10209000329604900C820E943E6B339604900D821F
:1020A000AD81A13210F4E0E0ED83E0E0EE830E9428
:1020B0004C6B0E94566B0E94E96AFA93EA930E9465
:1020C0003E6BE491EA930E948B6AFE013F96FA937D
:1020D000EA930E944D413F5F0F5FD2CF1F5FCDCF8C
:1020E0000E94F2460E940B7C279608950E94047C71
:1020F00030E010E01430F0F400E00430C8F40E9446
:102100003E6B0E94446B0E944C6B0E94566B0E9477
:10211000E96AFA93EA930E943E6BE491EA930E9483
:102120003E6B0E94EE6A0E944D413F5F0F5FE5CF1C
:102130001F5FE0CF0E94F2460E940B7C2496089518
:102140000E94027CA091B007A13051F40E945D6B07
:10215000ACE2B1E00E94A7795E2F47E12FEA09C007
:102160000E945D6BA0E4B1E00E94A7795E2F43E07E
:1021700028EE0E94616BA091B007A13071F4E6EBEC
:10218000F0E00E94786B0E947F6BEBE2EA93E8E755
:10219000F9E10E94896B0E944D41E3E0F0E00E946A
:1021A000786B0E948C6B0E948F6B0E949A6B3F5FD2
:1021B0000E94A06B11E0E0915A0B1E1740F500E061
:1021C000E091590B0E1708F50E94A76BD9F00E94F9
:1021D000AE6BE093FD03A02FBB270E948C6B0E9487
:1021E000B86B0E947C79DF01E42F0E94C06B0E94D3
:1021F000C46B0E949A6B3A930E949D21EF3F11F0AD
:102200000E94CA6B3F5F0F5FDBCF1F5FD4CFE091AF
:10221000FD03E093FC030E948B6A0E948B6AE4E654
:10222000F0E00E94906AEBE2EA930E948B6A0E94BF
:102230008B6A0E944D41E2E8F0E00E94896BE4E67F
:10224000F0E00E94906AE1E2EA930E948B6A0E94A9
:102250008B6A0E944D41FDDD0E94F2460E94097C7E
:102260005AC222970E94027CEDEEF6E0EE83FF83D5
:1022700040E04431A0F4AE81BF811196E0E0EC93E0
:10228000AE81BF811396EFEFEC93AE81BF81EC93EB
:10229000EE81FF813496EE83FF834F5FEACF0E9489
:1022A000A06B0E945D6BA0E4B1E00E94A7795E2F55
:1022B0000E94616B21FE1BC00E94D56B0E94D56BF2
:1022C000EFEAF0E00E948F6B0E949A6B0E94846A92
:1022D000E6EBF0E00E94DA6B0E947F6BEFE7EA9397
:1022E000EAE7F9E1FA93EA93E0E0F0E014C00E9433
:1022F000D56B0E94D56BE8EEF0E0FA93EA93E52FF8
:102300000E94DD6BFA93EA93E32FE058EA930E9470
:102310008B6AE2E2FBE0FA93EA930E944D413F5F51
:1023200011E0E0915A0B1E1710F00C94DA1100E046
:10233000E091590B0E17E0F50E94A76BB1F1A09147
:10234000320BE0E8EA23E03821F0A0917A0BA230CA
:1023500019F40E94AE6B0AC00E94E06BE03011F4E9
:10236000E0E001C0E8E0E093FC03E7E0E093FD0378
:10237000A02FBB270E948C6B0E94B86B0E947C79B7
:1023800033960E94C46B0E949A6B4E2FA091B607A1
:10239000E32F0E94E56BEA0FFB1F43833A930E94F1
:1023A0009D21EF3F11F00E94CA6B3F5F0F5FC0CFCE
:1023B0001F5FB7CF4EDD0E94F26A0E9442340E9436
:1023C000097C289608951A93A091590BE0915A0B15
:1023D000E150EA9FF001EF5F1E2FA981A13038F094
:1023E000E12FA0E40E948679A981EA1710F4E1E0C8
:1023F000E983E981E093B507A981A1501A9FF00113
:10240000E093B6070E947A44A091B007A83011F477
:1024100028DF01C095DE60C0E1E0E093FA03E2E06E
:10242000E093FB03E0E0E093FD03ECE0E093FC03CA
:102430000E94026B0E94EC6BFA93EA93E1E2EA934A
:10244000EDE7F9E10E94896B0E944D41EAE0E093DB
:10245000FC03E7E8F0E0FA93EA930E94EC6BFA934E
:10246000EA93EDE3EA93E2E8F9E10E94896B0E94C6
:102470004D410E94F24608951A93A981A43029F48F
:10248000A0E021FCA1E0A03009F426C0E9810E946F
:10249000F36B0490E9810E94F96BE491A02DAE1BCF
:1024A000A2501A2F0E94846AE4EBF0E0FA93EA93B8
:1024B000EB810E94F96B0E942F7A3296FA93EA938D
:1024C000EAE3F0E00E94016CEFE7EA93EAE7F9E162
:1024D0000E94896B0E944D411881229608950E94A6
:1024E0004F6AE0E0EA930E94261A0E94E06B0E2FEA
:1024F000ECE8F4E00E942F7A33971E2F0E948B6A3B
:102500000E948B6A0E94AD6A0E94086C0A930E9426
:1025100006640E94606A0E940D6C0E946E44E2E0B4
:10252000E093FB03E091300BEF70E093FD030E941A
:10253000126CEFE0E093FD03AA81A13051F40E94F8
:102540001A6C0E94076B0E945344E5E8F9E10E946F
:102550001F6C21FE0DC0E4E0EA938EDFE4E9F4E0B5
:102560000E94236CE6E9F4E00E94236C0E940C4771
:1025700090C0E8810E94F96B0E94286CEA810E9459
:10258000F36B0E94286C0E94AA44E881EA9374DFEE
:10259000B0C11A930A93EC81EA93EBDF1AEEEC8157
:1025A0000E94F36B0490EC810E94F96BE491A02DE2
:1025B000AE1BA2500A2FAC81A43029F4A0E021FC6C
:1025C000A1E0A03009F409C01EEAAA81BB811B96D4
:1025D000E0E0EC93EC81EA934FDF0E94AE6BE09376
:1025E000FD03EC81ABE0EA9FF001EC52FA4FFF9360
:1025F000EF930E94D56BEE810E94F96B0E942F7AB7
:1026000031960E94016C0E94136BFA93EA93EC8559
:10261000E058EA930E948B6AED85FE85FA93EA936F
:102620000E944D41AF91BF91EC93EC810E94F96BF8
:102630000E94286CEE810E94F36B0E94286C0E941D
:102640000C4719810881259608951A930A930E94D0
:102650005D6B0E942D6C0E948B6A0E94AD6A1A937A
:102660000A930E94976A0E941A6C0E941A6C0E9438
:102670005344EA81EA930E94261A0E94126CE4E60F
:10268000F0E00E94A96A0E948B6A1A930A930E9442
:102690000C4719810881239608951A930A930E9482
:1026A0005D6B0E942D6C0E948B6A0E94AD6A1A932A
:1026B0000A930E94976A0E941A6C0E941A6C0E94E8
:1026C0005344EC81FD810E941F6CAA81BB81A03024
:1026D000E0E1BE0734F4EA81FB81FA93EA930E94B9
:1026E0002F3FAA81BB81A130E0E1BE0744F0AEE7F5
:1026F000BBE0EA81FB81E150F0410E94336CE4E6EB
:10270000F0E00E94A96A0E948B6A1A930A930E94C1
:102710000C4719810881269608951A93E0915A056D
:10272000F0915B053197ACE0B0E00E945479EB5F2B
:10273000FC4FE081EF731E2F0E94406C99F40E94C1
:10274000476C0E948B6A0E944B6C0E94126C0E9424
:102750004F6C0E94536C0E945E6C0E941F3FE2E02F
:10276000E093FB03F7C30E941D62E0E0E093FC03EB
:10277000E093FC03A0910403A43039F40E94C26AE0
:10278000EDE4EA93E0E0F0E010C00E941A6C0E94D1
:102790001A6CE6EEF0E0FA93EA93E3E6F0E0FA93DF
:1027A000EA93EDE4EA93E1E9F9E1FA93EA930E940E
:1027B0008B6A0E944D4108950E947A440E941D62D6
:1027C0000E946C62E1E0E093FA030E94476C0E9471
:1027D000636C0E945344E3E9F9E10E941F6C0E947C
:1027E0008B6A0E94686C0E945344E6EAF9E10E94F9
:1027F0001F6C0E946D6CEA930E943E3FEDEAF9E186
:102800000E941F6CE0910403EA930E943E3F0895EA
:102810001A930A930E948B6A0E948B6A0E94534407
:10282000E3EBF9E10E941F6C0E948B6A0E94726CBC
:102830000E94AD6AE4E6F0E00E94B26A0E948B6AF0
:102840000E941A6C0E945344E0911E060E94776C0D
:10285000E8EBF9E10E941F6CE091C907EA930E943E
:102860003E3F0E948B6A0E940D6C0E945344E0918F
:102870001F060E94776CEEEBF9E10E941F6C00913D
:10288000190610E0153060F4E12F0E947C6C11F005
:10289000E1E301C0E0E3EA930E94E8431F5FF2CF67
:1028A0000E948B6A0E94D56B0E945344E0912006DF
:1028B0000E94776C0E948B6A0E94076B0E945344AF
:1028C000E09121060E94776C0E948B6A0E94836CC3
:1028D0000E945344E09122060E94776C0C946A197E
:1028E000E881E064E7B9369A349BFECF349AE4B1CC
:1028F000F5B121960895E881F981AA81BB81AE17CF
:10290000BF0724F4EA1BFB0B0C94B519A881B9810D
:10291000EA81FB81EA1BFB0B0C94B51928970E94F6
:10292000047C0E94886C11F4E4E001C0E1E0E093D3
:1029300062000E943C6AE5E0E09361000E943C6A0C
:102940000E94916CE0936405F0936505E091700539
:10295000F0917105E0936205F0936305E1E0EA937D
:10296000BFDFE0937005F09371050E94886C11F44D
:10297000E2E001C0E8E0E09362000E943C6AEAE025
:10298000E09361000E943C6A0E94966CE0936005AF
:10299000F0936105E0916E05F0916F05E0935E059F
:1029A000F0935F05E0E0EA939BDFE0936E05F09320
:1029B0006F050E94966CA0916005B0916105EA0FC9
:1029C000FB1FA0916E05B0916F050E949B6C8F015B
:1029D0000E94916CA0916405B0916505EA0FFB1F00
:1029E000A0917005B09171050E949B6C9F01E091D0
:1029F0006005F09161050E94A26CFF93EF930E9425
:102A0000966C0E94A26CAF91BF91EA0FFB1FFF93DF
:102A1000EF93E0916E05F0916F050E94A26CAF916B
:102A2000BF91EA0FFB1FE0936A05F0936B05E091FD
:102A30006405F09165050E94A86CFF93EF930E94D6
:102A4000916C0E94A86CAF91BF91EA0FFB1FFF939E
:102A5000EF93E0917005F09171050E94A86CAF9121
:102A6000BF91EA0FFB1FE0936C05F0936D05A091F9
:102A70006A05B0916B05E4E1F0E00E944E790E2EFC
:102A8000A0916C05B0916D05E4E1F0E00E944E79F3
:102A9000E02919F00E941243B1C00093660510931B
:102AA000670520936805309369050E94AE6CA634D3
:102AB000E0E0BE0724F4A8E5B5E00E94B36C0E94F4
:102AC000B96C989724F40E94BE6C98970CF010C0D3
:102AD0000E94AE6C1A9721F4E1E0F0E00E94C36C12
:102AE0000E94AE6C989721F4E2E0F0E00E94C36C83
:102AF0000E94B96C999724F00E94BE6C99970CF4CF
:102B00007DC0A2E5B5E00E94B36C0E94C86C0E9433
:102B1000B96C0E94CD6C0E94D46C0E94D96CE0EF1D
:102B2000F0E060E070E00E9481797F936F93FF9303
:102B3000EF93A2E0B0E00E944A7A0F010E94C86CB5
:102B40000E94DE6CAF91BF918F919F910E943E7960
:102B50000E94D1790E94D46C0E94E36C0E94BE6CEA
:102B60000E94CD6CEC83FD836E837F83AC81BD813D
:102B70008E819F81E0E4F1E060E070E00E94817965
:102B80007F936F93FF93EF93A6E0B0E00E944A7AA1
:102B90000F010E94E36C0E94DE6CAF91BF918F9198
:102BA0009F910E943E790E94D179EC83FD836E83D0
:102BB0007F83E091FF03E03049F4E885F985E093F5
:102BC0004605F0934705EC81FD810EC0EC81FD8147
:102BD000E0934605F09347050E94D96CEFEEF0E0D4
:102BE00060E070E00E941179E0934805F093490598
:102BF0000E949B6A0E94A26A0E9488420E940B7CEB
:102C00002C9608951A930E947A44E2E0E093FB0325
:102C1000E2E3F0E00E94E96A0E94E86CE4ECF9E18A
:102C20000E941F6CE4E1EA930E94C83EE0E9F1E0F3
:102C30000E94EC6CE4E1EA930E94C83E0E94F06CB2
:102C40000E94F87B14F4A895F9CF10E0143010F02E
:102C50000C948216E2E0E093FA030E94F56CDF0127
:102C60000E94236CFD0132960E94236C0E946E44E8
:102C70000E94F56C3496E491EA930E94E843E1E007
:102C8000E093FA030E94F06C5F9714F4A895FACFD2
:102C9000EAE0EA930E94C83E0E94F56CDF01359697
:102CA0000E942F7ABF01FD010E94FB6CDB010E9494
:102CB0005A7A0E94026D0E942F6BE8E2F0E00E94B7
:102CC0007C79E65AFF4F0E94E86C0E94F56C0E94E6
:102CD000FB6C0E94076D0E94F06C5E9714F0A89543
:102CE000FACF0E94F56CDF010E94236CFD01329641
:102CF0000E94236CE8E1F0E00E94906A0E94976ACB
:102D00001F5FA4CF0E94026DEAEFF0E00E94E86C22
:102D1000E0EDF9E10E941F6CE0EDF7E00E94EC6C41
:102D20000E947A4417C10E940B6DE4E6E2BF7894DA
:102D30000E944842F3DD1091C907E6B3AFEFEA27DE
:102D4000E093C907AAEFBAE00E94B36CE091F703E1
:102D5000EF5FE093F703A091F703AE3149F4A09140
:102D6000F603E3E8EA27E093F603E0E0E093F703F5
:102D70000E9403600E944822E2B3EF700E2EA091E1
:102D8000AB07B091AC07EFE0F0E0AE27BF27EA2336
:102D9000FB230E942A79E029E2BBE091AB07E071B6
:102DA00011F41D9A01C01D9812C00E940B6DE6E03F
:102DB000E4BDE0B1E295EF701E2FE0916300E07199
:102DC0001E0F0E94086C0E9421220E94EB5F199145
:102DD0000E941A6D18950E94145F0E94995F0E94CC
:102DE000DA4A0E942B2008951A93A8950E947940F0
:102DF000E13011F00C944317E091BB05E1501E2F18
:102E0000A091BA05A13021F40E94286DE03009F4A8
:102E100010C00E94286DE093D005ACE01A9FF0012D
:102E2000E25FFC4FBF01E081E260DB01EC930E94B6
:102E30002F6DA091BA05A23011F0A430A1F40E9428
:102E4000286DE093D105E5E1E093D0050E94346D53
:102E500031F0FD01E25FFC4FE081E27009F403C054
:102E60001A930E943D6DA091BA05A33019F41A93EC
:102E70000E94A527A091BA05A53029F4E091BB05D1
:102E8000EA930E94F927E091F603E078D1F0E0910F
:102E9000F603EF77E093F6030E943547E091F603DF
:102EA000E07131F0E091F603E270EA930E94514341
:102EB000A091CA07A13328F0E2E0EA930E94A00E95
:102EC0001E2F89DF47C01A930E947A44E1E0F0E0A8
:102ED0000E94896B0E94534410E00E94416DE1E022
:102EE000F0E00E94016C0E945344E091B907E03089
:102EF00041F4E3EDF9E10E941F6C0E94476D0E94CE
:102F00001F3FA091B907A130B8F0E091B907E15097
:102F1000EA930E94526DEAE0EA930E9415440E94EF
:102F2000636C0E94596DE091B907E1500E94606D99
:102F30000E94686D0E941F3F1E5FE091B907EF5F1E
:102F4000E093B9071C3020F4A091B907AB3008F02A
:102F500001C0C5CF199108951A930E947A440E9426
:102F6000416D10E0163090F5E12FA981AE0FA0342D
:102F700058F5A981EA0FEA930E94261A0E948B6AEB
:102F8000E12FEE0F0E946D6DE091BA07EA93E12FF9
:102F9000AA81EA0FEA930E94061B0E94126C0E940B
:102FA0008B6AE12FEE0FEF5F0E946D6D0E94726DD4
:102FB0000E94076DE8E7EA930E94E8430E94776D5C
:102FC0000E94337A0E941F3F1F5FCCCF0C945E1C7F
:102FD000E0E0E5BFE0936D00E0936C00EBBBEFEF4A
:102FE000EABBE0E0E8BBE7BBE5BBEFEFE4BBE0EF4B
:102FF000E2BBE1BBE0E3E3B9ECEBE2B9E0E0E09394
:103000006200E0936100EFE0E0936500E09364000C
:10301000E0E0E0BFE7E0E3BFE4E6E2BFE0E0E1BF1D
:10302000EFBDEEBDEDBDECBDE7BDE6BDEBBDEABD60
:10303000E9BDE8BDE0937900E0937800E3E0E5BD09
:10304000E6E0E4BDE0E0E3BDE0938B00EAE0E0937E
:103050008A00E0E0E0938900E0938800E09381003B
:10306000E0938000E2E1E0938700E4E3E0938600F0
:10307000E0E0E0938500E0938400E0938300E09338
:103080008200E0936A00E0E3EABFE0E4E9BFE8BF62
:10309000E1E4E7BFE0E0E0937D00EBB9E8EDEAB9F9
:1030A000E6E0E0939500E0E0E0939000E7E6E9B920
:1030B000E0E0E0939B00E8EDE0939A00E6E0E09327
:1030C0009D00E0E0E0939800E3E3E0939900E0E8FE
:1030D000E8B9E0E0E0BDE0E4E7B9E7E8E6B9E0B58B
:1030E000EF7EE0BDE0E2E0937000E0E0E09372008C
:1030F000E4E4E0937400EFE1E1BDEFE0E1BD0E94A4
:103100005D5778940E94D9660E943F43E1E0EA93BC
:103110000E94160F0E946D6CE53128F0A9E0B0E026
:10312000E0E00E94627A48DB21E030E0E0E0EA93F0
:103130000E94A00EE093CA070E94806D3F5FA0919D
:10314000CA07A43511F03A3008F001C0EFCF0E9451
:103150001A6C0E94026B0E945344A091CA07A435C6
:1031600081F4E1E0EA930E94A00EE093CA07E9ED42
:10317000F9E10E941F6CE091CA07EA930E94E843BC
:1031800008C0E0E0E093CA0720E0EFEDF9E10E941B
:103190001F6C84D0E03049F40E941A6C0E94836D49
:1031A000E8EEF9E10E941F6C20E00E94C86C0F015C
:1031B000A2E0B0E00E944A7A0E161F0654F40E9464
:1031C000E36C0F01A6E0B0E00E944A7A0E161F06DB
:1031D0000CF018DD203081F40E941A6C0E94896D79
:1031E0000E945344E4EFF9E10E941F6CA895E2E3CA
:1031F000F0E00E94EC6CFACF0E941B350E941A6C22
:103200000E94836DEFEFF9E10E941F6C0E94A71CE2
:10321000E03019F0E5E0FAE102C0E0EDF9E1FA93FF
:10322000EA930E94FE430E941560E1E0EA930E9447
:10323000C83E00E010E00436E0E01E0724F40E94DF
:10324000995FE03009F005C00E94806D0F5F1F4F4D
:10325000F2CF0436E0E01E072CF00E94F06C5F977E
:103260000CF0D0DCC1DD0E94CC30FCCFFFCF0E943F
:103270008E6D17FD10E01A3008F41F5F0E949B6DE1
:103280001DC30E948E6D17FD02C0103011F4E0E0E6
:1032900015C311500E949B6DE1E010C31A930A936D
:1032A00010E00E94A66DA8950E942960E03021F4EC
:1032B000E0EA0E94A96D09F002C001E001C000E04F
:1032C0000E943A601F5F003011F4153008F001C011
:1032D000E8CFE02F0991199108950E94AE6D2EC498
:1032E0000E94AE6D0E94BB6D0895A881B9810E94B5
:1032F000F87B24F4A83EE3E0BE070CF005C00E9472
:10330000C16D0E949A60DBC2E0E0D9C2A881B98198
:103310000E94F87B24F4A83EE3E0BE070CF005C051
:10332000EA81E03011F4EFEFEA830E94C16DED8194
:10333000EA930E94C7605EC10E94047C20E030E0F6
:10334000283EE3E03E077CF4A8953A932A93CDDF2C
:103350001E2F1F3F29F0EFEFEA933A932A93D6DF0F
:103360002F5F3F4FEDCF0E940B7C249608951A9358
:103370000A93E0E0F0E0E093D10BF093D20BAA8146
:10338000A03468F40E94CA6DE55FFB4F8F010E9474
:10339000D16D1A930A93E1EDFBE00E94D46DE091A8
:1033A000D10BF091D20B24C11A931FEF1F5F1A9318
:1033B000DEDFA981BA81EA17FB0711F0113408F0AA
:1033C00001C0F4CFE12F188115C1EA81EF5FEA83D4
:1033D000EA93CDDFA881B981EA17FB0719F0AA812A
:1033E000A13408F001C0F1CFEA8104C10E94027C3F
:1033F00010E0103430F50E942F6BE8E2F0E00E94FC
:103400007C79E050FC4FAF01E0EAEA93FA01709654
:10341000FA93EA930E949A60EC713E2FE0EAEA93F5
:10342000FA017396FA93EA930E949A600E2F303154
:1034300019F4EE81E01709F002C0E12F03C01F5F0D
:10344000D8CFEFEF0E94097C279608951A930A932C
:10345000E091210BAA81EA17E9F0A03468F40E94F8
:10346000CA6DE050FC4F8F010E94D86D0E94D46D50
:10347000EA81E093210B0EC0EFEFE093210B0E9455
:10348000E36DEDE2EA930E94896D0E940D67E0E032
:10349000E0932C0BADC01A930A930E94CA6DE050C2
:1034A000FC4F8F01AA81A03420F40E94D86D0E94A5
:1034B000BB6D9EC01A930A93E0914A0BAA81EA174A
:1034C000D9F00E94E86D40F40E94F46D0E94D46D22
:1034D000EA81E0934A0B10C0EFEFE0934A0BEBE474
:1034E000FBE0FA93EA93EDE2EA930E94896D0E9471
:1034F0000D67E0E0E093550B7BC01A930A930E949E
:10350000E86D20F40E94F46D0E94BB6D71C01A93A7
:103510000A93E091C80BAA81EA1761F10E94FF6D3E
:1035200018F50E94D16D1A930A93E9ECFBE00E9412
:10353000D46DEA81E093C80BE0E0E0931D06A09112
:10354000CA0BA13020F0A091CA0BA83008F00BC024
:10355000A0E7BBE0E091CA0B0E94096EAE0FBF1F4F
:10356000EC91E0931D0606C0EFEFE093C80BE0E09E
:10357000E093C90B3DC01A930A930E94FF6D40F47B
:103580000E94D16D1A930A93E9ECFBE00E94BB6D97
:103590002FC01A930A93E091C30BAA81EA17C1F0D6
:1035A0000E940C6E70F4E0EAEA930E94076B1A9393
:1035B0000A93E4ECFBE00E94D46DEA81E093C30B34
:1035C00007C0EFEFE093C30B0E94166E0E940D67D9
:1035D0000FC01A930A930E940C6E50F4E0EAEA932B
:1035E0000E94076B1A930A93E4ECFBE00E94BB6D08
:1035F00019810881239608950E94166E0E940D6716
:10360000E881EF5FE093C50B2196089524970E940F
:10361000027C0E941D6E0E940D67AB85A13010F0E8
:10362000A63008F007C0EB850E94096E0E94246E48
:103630000E94376EEB85E03049F5E0E0EE83EF83E2
:10364000E887E98740E050E020E030E02530E0E026
:103650003E07A4F4F9010E94246E0E94376E0E9476
:10366000726D4E0F5F1F0E94776D0E943C6E0E942C
:103670000C790E94416E2F5F3F4FE8CF4093B30B10
:103680005093B40B0E94466E0E944B6E0E94097CC0
:103690002C9608951A930A93AB81A13010F0A630AE
:1036A00008F01CC0EB810E94096E0E942E790E94D6
:1036B0002A79DF01EA810E94546EE8E0F0E00E947E
:1036C0007C79E050FA4E8F01E0EAEA930E94026BA7
:1036D0001A930A93E1EBFBE00E94BB6D198108810C
:1036E0000C9429201A930A93EA810E94586EE831BB
:1036F00021F4198108810C9429200E9477200E2F33
:1037000010E01017E0F5EB81EA93EB81EA937EDF9E
:10371000A3EBBBE00E94B36CA091B50BB091B60BCC
:103720008091B70B9091B80B0E945D6E0E943E791C
:103730000E940C790E944B6EEB81EA93EB81EA9335
:10374000A9DFEB81E093B90B0E94626E309759F4C8
:103750000E946D6C0E94676EEF5EF84DDF01EA819A
:103760000E94C06B02C00E94626EE093BA0BF0939D
:10377000BB0B0E946D6E0E94726E1F5FC2CF1981DB
:1037800008810C9429200E94047C00E00B3048F44E
:10379000E02F0E94606D0E94786E0E942A7A0F5F6F
:1037A000F5CF0E94786E0E947D6E00E00034E8F450
:1037B0000A934CDEE091BA07EA930A9327DFE0917F
:1037C0002F0B0E94866E0F01E0912F0B0E94606DFF
:1037D0000E94247ADF01CB010E94776D0E940C7950
:1037E000D0010E942A7A0F5FE1CFA091B007A330E9
:1037F000E1F530E03031C8F50E942C6B0E948E6EEE
:1038000091F500E00A3078F5E32FE05DEA93EAE015
:10381000FAE10E94936EE02FE05D0E949A6E09F536
:1038200013E0E02F0E94866EFF93EF93E02F0E943B
:10383000606D0E94247A7F936F93FF93EF93EDB7AF
:10384000FEB7FA93EA931F930E94E45C1F91AF9135
:10385000BF918F919F910E940C79AF91BF910E946F
:103860002A7A0F5FCFCF3F5FC5CF00E00A3098F4D0
:10387000E02F0E94606D0E94247AA091C107B09150
:10388000C2078091C3079091C4070E940C790E94DF
:103890007D6E0F5FEBCFDBC31A93A895A981A6308D
:1038A00068F40E941D6E0E940D6710E0103430F421
:1038B000E981EA931A93EEDE1F5FF8CF1881229612
:1038C00008951A9311E0163020F41A93E5DF1F5F74
:1038D000FACF4CC3E1E0E093C90BE093CA0B0C9420
:1038E000E820A895EBE4FBE0FA93EA93E8E8F5E03A
:1038F000FA93EA930E94026B0E949F6EE093530B2F
:103900000E94A86EE093540BE0E0E093550B0C94FA
:10391000E820A895E1E2FBE00E94AF6EE9E2F0E06A
:103920000E94B46E0E94E36DEEE7F5E0FA93EA932D
:103930000E94026B0E949F6EE0932A0B0E94A86E69
:10394000E0932B0BE0EBE093300B0C94E8200E940B
:10395000027C0E94B86EE03228F0AAE0B0E0E0E01D
:103960000E94627A00E0B9DCA091560BB091570B2F
:10397000A633E2E1BE07C1F1E3E50E94BD6E1A3055
:1039800030F41A93AEDF1A93B8DD1F5FF8CFE0E58D
:103990000E94BD6E103430F41A93BBDF1A937BDDA6
:1039A0001F5FF8CF0E94800EEBE40E94BD6E1038BE
:1039B00030F41A938FDF1A93DEDD1F5FF8CFE1E456
:1039C000EA930E94E8437DDFE4E5EA930E94E8433E
:1039D000A9E0B0E0E0E00E94627AE6E3F2E1E09381
:1039E000560BF093570B01E010E0153210F00C94D9
:1039F0005C1D0E94C26E9F010E94C26EAF010E94B8
:103A0000CB6E70960E942F7A309721F0E130A0E0C3
:103A1000FA0781F4D9016C910E94CB6E72960E94D4
:103A20002F7AA62F0E94D16E24F40E94CB6E0E94A2
:103A3000D56E40C0E230A0E0FA07C9F4DA016D911A
:103A40007C910E94CB6E72960E942F7AE617F70740
:103A50002CF0DA010E94207AFF2342F40E94CB6E00
:103A600074960E942F7ADA01ED93FC9323C0E33021
:103A7000A0E0FA0749F4D901AC91AF3F21F40E94CC
:103A8000CB6E0E94D56E16C0E430A0E0FA0791F428
:103A9000D901AC91AF3F71F400E00E94CB6E0E945F
:103AA000DA6E44F40E94CB6E0E94D56E2F5F3F4FBA
:103AB0000F5FF3CF1F5F99CF13DC10E0153060F478
:103AC0001A9367DDA091C40BA63020F01A9394DD01
:103AD0001A937FDD1F5FF2CFE02F0E94097CA1C007
:103AE000E881EF5FE883A881A43610F0E0E0E88386
:103AF000E8810C94E8200E94E26E30960C94E82055
:103B0000A091CC0BBB27E091CB0BA8C0F9DF32977B
:103B100074F00E94E96EE091CB0B0E94EC6E0E9463
:103B2000BB6DE091CB0BEA93DBDFE093CB0B089509
:103B30000E94E96EE091CC0B0E94EC6EFA93EA933E
:103B40000E94E8600895E9EBFBE00E94F46E0E9499
:103B50000D670E94E96EE091CC0B0E94EC6E0E9412
:103B6000BB6DE091CC0BEA93BBDFE093CC0B0895E7
:103B70000E94047CE0E0E093CB0BE093CC0B10E0E0
:103B800030E0343680F5A8950E94E96E3A93B3DFB1
:103B9000FA93EA93E9EBFBE00E94D46D00E0A09178
:103BA000B90BA13010F0A03808F001C001E0E12FFE
:103BB000E03041F4013029F43093CC0B3093CB0B3F
:103BC00011E00FC0E13031F4003019F43093CB0B29
:103BD00012E007C0E23029F4013019F43093CC0B25
:103BE00013E03F5FCECF33C21A93A091670BA8704A
:103BF000B9F010E0E981FA810E942F6BAE17BF0780
:103C00007CF4ED81E093B90BEB81FC81E851FC4F32
:103C10000E94F96EE0E0F0E00E94726E1F5FEACF52
:103C2000188126960895E881EF5FE883A881A4367D
:103C300010F0E0E0E883E8810C94E820E881E150AE
:103C4000E883A881A43610F0E3E6E883E8810C94C9
:103C5000E820A091CE0BBB27E091CD0BF0E0319690
:103C60000E94FE6EEC59FF4FDF01E4E6F0E00E9497
:103C7000D97908950E94E26EE050FE4F0C94E8203E
:103C8000EEEBFBE00E94F46E0E940D67E881EA9380
:103C90007CD10C94E8201A934FDBE1E0E0931E0BFB
:103CA00065C1A89510E0143680F41A9367D1A091ED
:103CB000BE0BAF3F31F40E94036FAF3FEFEFBE0783
:103CC00011F01A93DDDF1F5FEECF0E94086F68943A
:103CD00020F84CC10E94047C1091CE0BAD81AA2328
:103CE000C2F5E091CD0BE11719F0AD81AA230AF0DE
:103CF0002FC01A9343D10E94036FEE81FF81EA1710
:103D0000FB0729F4E885A091BE0BEA1709F01DC056
:103D10000E940E6FEC81FD810E941679EA17FB0765
:103D200054F40E94136F0E941C6FE0E0EC83ED835B
:103D30001A932BD10AC00E94136FEC83FD83E0E03D
:103D4000F0E00E941C6F0E94216F0E94276FC9CF74
:103D50003FC0E091CD0BE11729F0AC81BD810E94FD
:103D6000F87B0CF01BC01A9309D10E94036FEE81FF
:103D7000FF81EA17FB0729F4E885A091BE0BEA173B
:103D800009F009C00E94136F0E941C6F1A93FDD0A6
:103D9000E0E0EC83ED830E94276FDBCFAC81BD8137
:103DA0000E94F87BACF4E885E093BE0BEE81FF81C6
:103DB0000E942C6FEC81FD810E941C6FE091CD0B65
:103DC000EA93E3D0E091CD0BEA932DDFE093CD0BA6
:103DD00040DF7E9714F00C94371F1091CD0B0091AB
:103DE000CD0B1A932BDF1E2F1A93C8D0A091BE0BB8
:103DF000A13010F0A03808F022C00A931FDF0E2F68
:103E00001017E9F00A93C1D030E03330C0F4ABE0D2
:103E10003A9FF001DF01ED52FA4FE081E03031F0DE
:103E2000FD01EE52FA4FE0811E1709F006C0ABE02B
:103E30003A9FF001EE52FA4F00833F5FE6CFE091E8
:103E4000CE0BE11771F6101791F0EEEBFBE00E943C
:103E5000F46E0E940D67102F0A93F0DE0E2F0A9366
:103E600094D0E091CE0BE017B9F71093CE0B689485
:103E700020F8EC81FD810E940B7C299608951A930D
:103E8000A8951091CE0BE091CD0BE117C1F00E94E7
:103E9000316F0E94F87B64F4EB81A091BE0BEA17AE
:103EA00039F40E94036FE981FA81EA17FB0709F0F0
:103EB00003C0E12F1881CDC00E94276FE4CFEFEF40
:103EC0001881C7C00E940E6F0E94F87B84F4E091B5
:103ED0001D06E87031F4E091C707A091BE0BEA1708
:103EE00031F40E94356F0E943A6FE03408F001C04F
:103EF00015C112C1A895E091CD0BA881EA1749F030
:103F0000E8810E943E6F11F0E88162C10E94456F16
:103F1000F2CFEFEF5DC11A93A8951091CE0BE0910F
:103F2000CD0BE117E1F00E94316F0E94F87B8CF419
:103F3000E0911D06E87031F4E091C707A091BE0B37
:103F4000EA1739F40E94036FE981FA81EA17FB0747
:103F500009F002C0E12F72C20E94276FE0CFEFEF9D
:103F60006DC21A931091CE0B1A93C4DF1991089564
:103F70000E94456FE881EA93BDDF2AC10E94E96E85
:103F80000E944B6F0E94D46D23C10E94E96E0E9473
:103F90004B6F0E94BB6D1CC1E091CE0BA881EA174C
:103FA00041F40E940E6F109721F4A091BE0BA03037
:103FB00009F01CC0E881EA9363DE0E94456FE88146
:103FC000E093CE0BE091CD0BA091CE0BEA1719F048
:103FD000E881EA93D3DF0E940E6F109721F4A0913D
:103FE000BE0BA03009F001C0E5CF03C0E881EA9321
:103FF000CCDFEEC00E94047C0E94086F10E030E02D
:10400000343628F5A8953A93B9DF00E0A091BE0BAD
:10401000A03808F401E0E12FE03041F4013029F448
:104020003093CE0B3093CD0B11E00FC0E13031F463
:10403000003019F43093CD0B12E007C0E23029F4C0
:10404000013019F43093CE0B13E03F5FD9CF0E94BB
:104050000B7C249608951A930A93A091B007A4307C
:1040600009F44FC11091C7070091000CE091C907F6
:10407000E03059F0E093C707689424F80E94546F29
:10408000E0E0E093C807E0E520C0E091C807E03039
:1040900021F0E093C707E2E518C0E0E0E093C7072E
:1040A000E093000CE0915C0BE03031F0E0915C0BB0
:1040B000E150EA930E94871AA091C90BA17039F0D0
:1040C000E0915C0BE093C707E4E4E093000CA0915F
:1040D000C7071A1721F4A091000C0A1711F0689471
:1040E00023F80FC1A091320BECE1EA230895A091CF
:1040F000320BA07411F0E2E00895A091320BA07889
:1041000059F40CC0A091210BAF3F31F0EBDFE4304C
:1041100019F0E8DFE03111F4E0E00895E1E00895FE
:104120000895A881AF3F09F452C0DCDFE43011F4F8
:10413000E1E04EC04CC0A881A23019F4D3DFE830D2
:1041400011F0E1E045C043C0E8810E945A6FE35B93
:10415000F94FE081E13010F0E43108F002C0E1E015
:1041600037C035C0A881A13118F0E881E051E8835B
:10417000E8810E94606F0E946A6FA091680BA13075
:1041800018F0A881A43009F006C0E6E9F0E00E942A
:104190002F7A0E946A6F1CC0A881A13010F0A6304F
:1041A00008F007C0E8810E94096EE351F44FE081F6
:1041B0000FC00DC0A881A13010F0A63008F007C0D4
:1041C000E8810E94096EEE50F44FE08101C0E0E00A
:1041D000219608950E94047CEC81EA93EBDFEF7353
:1041E0001E2F1030C1F0EC81EA93E4DFE0743E2F23
:1041F000E12FE1500E947C6C0E2F303011F4003022
:1042000009F002C0E1E008C0303011F0003009F4DC
:1042100002C0E1E001C0E0E00E940B7C2596089519
:104220001A930A93E9EDFBE00E94AF6E0E94836C43
:104230000E940D6710E0153090F51A930E94C91A7C
:104240000E942F6BA351B44FE091C50BEC930E94D9
:10425000756FEE50F44F0F01A091C40BEFE3EA230A
:10426000AE2FE091C70BE295E07FEE0FEE0FEA0F65
:10427000D001EC93E091C50BE1500E2F0F3F69F098
:10428000E02F0E94786FEA0FFB1FBF01E091C60B81
:104290000E94676EDB01ED93FC931F5FCCCF31C0B2
:1042A0001A930A93EAE2F6E00E94F46E0E940D6708
:1042B00010E0103430F51A930E94261A1A9331DF59
:1042C000E130E9F4E091350BEA9366DFE1500E2F1F
:1042D0000F3FA9F00E94136BE65DF94F1083A02FEA
:1042E000B0E0A15DB94FE091350BEC93E02F0E9457
:1042F0007E6FE0913B0BF0913C0BED93FC931F5FC5
:10430000D8CF099119910895A091B007A23031F04A
:10431000A83021F0A73011F0A53009F40DC0EDE46C
:10432000F6E00E94AF6EE0EFF0E00E94B46E78DF3E
:10433000B7DFE0E0E093230608951A93E981E0589F
:10434000E98310E01530C8F4E12F0E945A6F0F0185
:10435000E15BF94FE081AE2FE981EA1749F4F00102
:10436000E25BF94FE081AE2FE091C707EA1709F051
:1043700002C0E12F03C01F5FE5CFEFEF1881229647
:1043800008950E94047CED81EA93D7DF1E2F1F3F22
:10439000C9F0E12F0E945A6FE35BF94F9F01D901E9
:1043A0001296EC91EF77EC93EC81D9010E94866F25
:1043B0000E948D6FEF77DB010E94866FE25FFC4FFA
:1043C000A1E0A083E12F0E940B7C1FC41A931FEF72
:1043D000E0916C0BF0916D0BA981BA81AE17BF070C
:1043E0003CF0E0916E0BF0916F0BEA17FB070CF4B9
:1043F00011C0E981FA81FA93EA930E9475191E2F80
:10440000103031F01F3F21F0E091C707E11711F4A0
:10441000E1E014C01F3F39F4EEE0FAE1FA93EA93C9
:10442000EB81FC8106C0EEE1FAE1FA93EA930E9487
:10443000756FFA93EA930E944D13E0E0188123967A
:1044400008950E94047CE0911B06F0911C06AC814B
:10445000BD81EA27FB279F0110E0153080F4F901A8
:10446000E17039F00E942F6BA25EB94FEC91EF5FC3
:10447000EC93D9010E94926F9F011F5FEECFEC81F8
:10448000FD81E0931B06F0931C060E940B7CBDC3CC
:1044900026970E94027C30911B0610E01530A8F58B
:1044A0000E94756FE950F44F0081E12FA1E00E9456
:1044B00022792E2FE22FE32391F0003810F0003CF8
:1044C00008F001C00F5F003C31F4E22FA091190603
:1044D000EA2BE0931906003808F400E80FC0003416
:1044E00008F40F5F003439F4EFEFE227A0911906CA
:1044F000EA23E0931906003808F000E00E94756F87
:10450000E950F44F00831F5FC9CFE0E0F0E0E09393
:10451000AD07F093AE07E091B407EF5FE093B40707
:10452000E0917B0BA091B407EA1751F4E0917B0B6B
:10453000F0E0A0E0B1E00E94437AEA1BE093B40708
:10454000A091B007A13019F0A93009F0B0C0A09136
:10455000FA0AB091FB0AE4E1F0E00E94D9793097C1
:1045600019F4E1E0E093B707E0912306E030D9F0D9
:10457000E0912406EA93F6DDE0912506EA93F2DD68
:104580000E94976FE25EF94FE081A0912806B091FA
:1045900029060E94C06B0E949A6F0E949F6FA6E23C
:1045A000B6E00E94B36C0E94A46F109721F0E091D6
:1045B0005C05E07809F459C0E0915C05F0915D0577
:1045C000EF73F0705E2F5A930E94261AA091310B60
:1045D000A03049F497DDE13031F4E091B107EA937E
:1045E000AADDE03009F441C00E94A96F0E94546E18
:1045F000EC91EC71EC3021F4E091B407E07871F4C7
:104600000E94AE6FEC91EA93ADDDA8E3BBE0E091D0
:10461000B1070E94546EEC91EA93A4DDE52FADE45E
:10462000B6E00E94B36FAE0FBF1F0E94B36C0E9432
:10463000AE6FEC91EA93B0DD1E2F1130B0F00E9406
:10464000B76FEA0FFB1F0F010E94B76F0E94BB6F8D
:10465000E12F0E94096E0E94C16FD001ED93FC937F
:10466000E12F0E94096E0E949F6F10E01530F8F450
:104670000E94756FE65DF94F50815F3FB1F00E9477
:10468000756F0E94C56F0E94B76FEA0FFB1F0F0185
:104690000E94B76F0E94BB6F0E94756F0E94C16F2E
:1046A000D0010E94CB6F0E949F6F1F5FDFCFA09150
:1046B000B007A23039F0A83029F0A53019F0A730A2
:1046C00009F0B0C1E0E0E093B80700E0053010F079
:1046D0000C9412250E94136B0E94CE6FE35BF94F7E
:1046E000E887F987A885B985AC91A03019F0A28137
:1046F000A07809F095C1E091B807EF5FE093B807A3
:10470000A885B98513960E94207A309781F0A885F4
:10471000B9850E94D36F0E94DA6F19F00E94DF6F93
:1047200009F004C0A885B9850E94E76F79C10E948D
:10473000A46F109739F00E94DA6F19F00E94DF6FB2
:1047400009F46EC120E030E0333010F00C94B8244E
:104750000E94136B0E94CE6FEE5AF94FDF010E9448
:104760002C6B0E94ED6FE60FF71FEE83FF83AE8187
:10477000BF81EC91E27021F40E94F36F109709F46D
:10478000D9C0EE81FF81A581B681109751F00380D9
:104790001480AE81BF8115960E94207A0E161F06E6
:1047A0000CF00EC0AE81BF8115960E94F86FE091AB
:1047B000B00B0E94676EA885B9851396ED93FC93A4
:1047C000AE81BF81EC91E17021F40E94D36F3196EC
:1047D00053C00E94FD6FE0DCE1501E2F0E94756FF8
:1047E000E25EF94FE081E03019F50E940270AE0FF1
:1047F000BF1F0E94B36CE12F0E94786F0E94067069
:10480000309759F00E9402700E940B700E94786FDE
:104810000E940670E015F1050CF009C00E94136BB0
:104820000E94117011F00E9416700E941E701BC031
:10483000EE81FF813396BF01DF010E94207ADF0104
:104840000E94756FE25EF94F0E9426700E94FE6E14
:10485000DB010E94CB6F0E949F6F0E940270AE0F1F
:10486000BF1F0E94F86FEE81FF81A481AA2322F46A
:10487000AE81BF810E94E76FAE81BF81EC91EC7188
:10488000EC3021F4E091B407E078B1F40E94F36FCA
:104890005E972CF4AE81BF81EC91E07209F404C004
:1048A000EE81FF81A18106C00E94FD6F5BDCEE817D
:1048B000FF81A281AA9356DC0E94297089F0AE8103
:1048C000BF8117960E9430700E94297049F40E949F
:1048D000136B0E94117011F00E9416700E941E70DE
:1048E0000E94FD6F77DCE03029F10E94136B0E947B
:1048F000117071F00E941670A885B985EC91E15095
:10490000ACE0EA9FF0010E948D6FE058DB01EC9370
:10491000A885B9851296EC91E058A885B9851296BC
:10492000EC93E3E0E0931A060E94FD6F43DCEF7323
:10493000E093FD0BAE81BF8113960E94207A3097E1
:10494000A9F42F5F303041F4E885F985E685ED7FE5
:10495000A885B9851E96EC93313041F4E885F98538
:10496000E789ED7FA885B9855796EC933F5FECCE3C
:10497000233011F00C9410250E94DA6F11F00E9480
:1049800016700E944732E030A1F00E943670E8E0D5
:10499000EC93A885B9851296EC91AA85BB851496EF
:1049A000EC93A885B985EC91AA85BB85EC930E9410
:1049B0004370A885B985E0E0EC93E885F985A58189
:1049C000ECE1EA23E83061F50E946D6CAE2FE885DA
:1049D000F985E08DEA1741F4E885F985E18DE1502C
:1049E000EA930E9437191CC00E944732E030C1F0A0
:1049F0000E943670E3E0EC93AA85BB85EFEFEC9361
:104A00001696E885F985E08D0E944B70AA85BB85D6
:104A10001296E885F985E18D0E944B700E944370E3
:104A20000F5F54CEA091B007A23029F0A83019F042
:104A3000A53009F05CC010E0153010F00C9477251B
:104A40000E94756FE65DF94F50815F3F11F40C9441
:104A500075250E94756F0E94C56F0E944F70EA0F06
:104A6000FB1F0F010E944F700E94BB6F0E94756F69
:104A70000E94C16FD0010E94CB6F0E949F6F0E9465
:104A80004F700E94BB6F0E94F87BBCF4E12F0E9424
:104A90007E6F0E94207ADF010E94F87B74F40E94EE
:104AA0004F700E940B700E947E6F0E94207AD0018E
:104AB000AE1BBF0B0E94F87B0CF017C00E944F701A
:104AC000EA0FFB1FBF010E944F700E940B700E94F3
:104AD0007E6F0E94207A0E94DE6CDB01ED93FC93D6
:104AE0005A93E5E0EA930E9497401F5FA5CFE091BB
:104AF000B307E03041F4E091AD07F091AE07E093E9
:104B0000AB07F093AC070E94097C2C9608950E9495
:104B1000027CE8DAE03111F40C94022620E030E067
:104B200040E050E010E0133040F50E9453700E94C6
:104B30005670309701F10E9459700E94606F2E2BC1
:104B40003F2B0E9459700E94607029F0E3E0E093CF
:104B50001A06E0E058C00E9465700E94606F2E2B1C
:104B60003F2B0E9465700E94607029F0E3E0E093A3
:104B70001A06E0E048C01F5FD6CF00E00530C0F560
:104B80000E94136B0E94CE6FE35BF94FE081E0302F
:104B900069F110E0133050F50E94136B0E94CE6F44
:104BA000EE5AF94FDF010E94756F0E94ED6FDB0135
:104BB000AE0FBF1F1196EC910E94606F4E2B5F2BC2
:104BC0000E94136B0E94CE6FEE5AF94FDF010E94D4
:104BD000756F0E94ED6FDB01AE0FBF1F1296EC9157
:104BE0000E94606F4E2B5F2B1F5FD4CF0F5FC6CF2D
:104BF000F901E423F523309729F0E1E0E0931A0668
:104C0000E0E001C0E1E00E94097C269608951A9335
:104C1000E091FE0BE03011F40C944E26E0917C0BF9
:104C2000E13059F4A091FE0BA13311F4EFE001C083
:104C3000E0E0EA930E94E65731C0E23059F4A091D7
:104C4000FE0BA13311F4E6E001C0E5E1EA930E9416
:104C5000E65724C0E330B1F410E0173040F40E946E
:104C6000756FE852F74F0E946C701F5FF6CFA091EE
:104C7000FE0BA13311F4E1E301C0E0E3EA930E94EB
:104C8000E6570CC00E947070E9E4EA930E94F25B60
:104C9000E091FE0B0E9477700E947C70199108953C
:104CA00022970E94027C30E0A091B007A23029F048
:104CB000A83019F0A53009F01FC1A985A03410F063
:104CC0000C947A27E091C707E03009F43AC1E985EE
:104CD0000E94586EE03131F4E1E3E093FE0B97DF80
:104CE000E1E02FC10FDAE03009F42BC110E01530FC
:104CF00070F4E12F0E945A6FE35BF94FE081AE2F11
:104D0000E885EA1711F4E0E01CC11F5FF0CFFFDE79
:104D1000E03011F40C947A2710E0E12F0E945A6FD2
:104D2000E35BF94FEE83FF83AE81BF81EC91E0300E
:104D300011F00C9473270E94E76F00E0033010F02D
:104D40000C944527E12F0E945A6FEE5AF94FDF016C
:104D50000E94136B0E94ED6FE60FF71FAF01DA019F
:104D600015960E94F86F0E948170DA011196EC93FB
:104D70000E948870DA011296EC93A091320BECEF4E
:104D8000EA230E2E0E948F70E029DA01EC93AAD953
:104D9000E43121F4DA01EC91ED7F03C0DA01EC910A
:104DA000E260DA01EC930A93C6D9E03011F40C9476
:104DB0003227FA01A181AA93EFD92E2F213078F062
:104DC000E22F0E94096E0E949F6FE22FE150A3EE36
:104DD000BBE00E94B36FAE0FBF1F0E94F86F0E942E
:104DE00097700E945670DA011396ED93FC93013090
:104DF00031F4E0913D0BF0913E0B309709F004C087
:104E00000E949A70E062EC93023031F4E0913F0B23
:104E1000F091400B309709F006C0AE81BF811E961D
:104E2000EC91E062EC93AE81BF815796EC91E06229
:104E3000EC930E948170EA93BDD9E07831F40E942E
:104E40008870EA93B7D9E07861F00E949770EE0F0E
:104E5000FF1F0E94BB6F0E94926FDA011596ED93BF
:104E6000FC9303C0DA010E94E76F3CD9EC3019F4DF
:104E7000E0E0E093B4070E949F700E94676EDA0141
:104E80001796ED93FC930F5F59CFA091B007A23016
:104E900011F0A53019F4A885A03808F007C0E091FA
:104EA000C707EA93EA85EA930E94721BE885AE8100
:104EB000BF81EC93E091C707AE81BF811196EC935F
:104EC000E985AE81BF811296EC93A885A03830F4B5
:104ED000E885E1500E94A670A1E0A0830E949A702C
:104EE000ED7FEC9331E01F5F303011F4153008F0A6
:104EF00001C013CFE32F25C0A091B007A13009F561
:104F0000A985AF3F41F0E985EA930E94261AE0E0C7
:104F1000EA930E94C83EE885E0932306E091350BB2
:104F2000E0932406E091380BE0932506E0E0F0E002
:104F3000E0932606F09327060E949A6F0E949F6FC7
:104F4000E1E00E94097C2A9608951A930A93A091A1
:104F5000B007A23011F0A53049F4EA810E94A67092
:104F6000A0E0A083EA81EA930E943D6DA091B00782
:104F7000A830D9F5EA810E94A670A0E0A083EA815A
:104F8000EA93E1E0EA930E94DD44EA810E94AC707A
:104F9000E081EF771E2FEA81ABE0EA9FF001E45257
:104FA000FA4FA0E0A083A0917A0BA03039F40E94C0
:104FB000B270DF010E94207A309709F010C00E9481
:104FC000B87000810E94B870AFEFA0830E94B270E9
:104FD0000E94BE701A930E94B912689420F8E09162
:104FE0007A0BE03011F0689420F81981088123963B
:104FF000089564970E94047CA091B007A23039F410
:10500000E091C707EA93E98DEA930E94721BA09191
:10501000B007A83011F00C946C280FEF30E0353059
:1050200048F40E942C6BE65DF94FE081AE2FE88DCD
:10503000EA1709F402C03F5FF2CF0E942C6BE25CDA
:10504000F94F00810F3F11F40C946C280E94C3703B
:1050500010810E94316F0E94F87B04F5A1ECBBE047
:105060000E9430700E94C9700E940E6FA083B183AD
:105070001A930E94C51FABE00A9FF001EC52FA4F51
:1050800020810A930E94CF700E9489332A930E9444
:10509000CF700E940E412A930E943D6D0E94D470F1
:1050A000D9F40E94C3700E94DA70E65DF94F0E9445
:1050B000DA70E25CF94FAFEFA0830E94C9700E94E2
:1050C000BE70E0E0F0E00E941C6F0E94216F0A9326
:1050D0000E94B912689420F80E940B7C699608958A
:1050E0001A9310E01031A0F40E94756FEE50F44F47
:1050F000E081EF73AE2FE981EA1729F4E12FEF5F2A
:105100000E94607009F402C0E1E003C01F5FEACFB3
:10511000E0E01881229608951A930E94DD70E4EF72
:10512000F1E00E94E470F9F00E94EA7010E015309E
:10513000D0F4A091030CAF5FE5E00E94D679E09334
:10514000030CEF5FEA93CCDFE03059F0E3E0E0934B
:105150001A06E091030CF0E0EF5FFF4EE093FD0BC9
:10516000A3C31F5FE4CFA0C31A93E0911906E09395
:10517000FC0BE8E7F0E0FA93EA93ECEDF0E0FA9349
:10518000EA930E94AA4410E01530C0F4E12FEF5FCB
:10519000EA93A6DFE03081F00E948B6AE12FEA5F9C
:1051A0000E946D6DEBE2FAE10E941F6CAEE7BBE07E
:1051B0000E94756F0E94336C1F5FE6CF75C3ACDF32
:1051C000A0911A06A13021F4E3E3FAE10E94F17004
:1051D000A0911A06A23021F4E0E4FAE10E94F170F5
:1051E000A0911A06A33041F4EBE2FAE10E94F970B3
:1051F000E050F04F0E94FF70A0911A06A43031F4E5
:10520000E8E4FAE10E94F9700E94FF70A0911A068A
:10521000A53029F4E091FD0BEA930E942513A0919B
:105220001A06A63031F4E0E5FAE10E94F9700E9416
:10523000FF70A0911A06A73021F4E6E5FAE10E947A
:10524000F170E0E0E0931A060895A881B981119603
:10525000E1E0EC930E94356FA881B9811296ED933D
:10526000FC930E947720A881B9811596EC930E9447
:105270006D6CA881B98116960E944B70E091BB05B8
:10528000A881B981EC93E091BE0BA881B9811496F5
:10529000EC93E091210BA881B9811896EC93A9C4F5
:1052A00064971A930A93A0917A0BA230E1F4E98DE6
:1052B000EA930E94261A0E947720A1ECBBE00E948C
:1052C0004B70AFEBBBE0E98D0E944B70E091C707DC
:1052D000E093BE0B0E94626E309721F00E94626ED6
:1052E0000E942C6F14C0A88DAF3F09F4C5C0E88D93
:1052F000EA930E94BE1FA98DAF3F29F40E94356F2B
:105300000E943A6FE98FE98DEA930E94261A0E9463
:1053100077200E2FAF89AF3F21F00E948220E0302E
:1053200009F001C0A9C00E940E6F0E94136BAE1756
:10533000BF071CF0ECDBE13009F09EC0A091690BC7
:10534000A03021F4A0917A0BA23011F50E946D6C6F
:10535000E13041F00E944732E03021F00E945D329E
:10536000E03009F002C00E9403710E946D6CE130D0
:1053700021F40E944D32E03009F409C00E940F71FF
:10538000E35BF84FFA93EA9360DF0E94157172C0F5
:10539000E98DEA930E941D711E2F113011F00C94BB
:1053A0003A2AA0916B0BA13059F4E091C707EA9318
:1053B0000E94356FFA93EA93EFEFFFEF0E9422719C
:1053C0000E940E6F0E94136B0E94FE6E0E941C6F63
:1053D000689420F8A0917A0BA03019F4AE89AF3F01
:1053E00009F42EC00E942671E852FA4F0E940E6FF7
:1053F000A083B183EE89EA93FE013396FA93EA9390
:105400000E9489330E942671EC52FA4FE081EA93A0
:10541000FE013396FA93EA930E940E410E94267190
:10542000E452FA4FA1E0A0830E942671E652FA4F9F
:10543000FF93EF930E94FA61AF91BF91ED93FC93BC
:105440000E94D47041F4E0E0E093BE0BE88DEA9353
:105450000E94CC1F04C0E88DEA930E94C51FE09112
:10546000C707EA930E94626E0E942B71FA93EA9337
:105470000E94F41DE1E001C0E0E0198108816A9614
:10548000089545DBE13041F40E944732E03021F0DD
:105490000E945D32E03009F007C00E94626E0E94F7
:1054A0002C6F0E940371C7C2CFC21A930A930E9445
:1054B0002E711F3F11F40C94A42AE091FE0BE030F2
:1054C00011F00C94A32A1A930E94261AE5E0E093A7
:1054D0001A061093FD0BA091B007A23031F40E9480
:1054E00035710E94E621E13009F00EC0A091FF0B5A
:1054F000A13331F4E091C707EA931A930E94721B1B
:10550000E1E3E093FE0B71C1A091B007A83081F4F4
:105510000E94626EFA93EA930E948B1F0E2F1A93D9
:105520000A93EFEFEA93EA93BBDEE03009F05DC146
:10553000A091B007A53021F4A4DFE03009F055C1F7
:10554000E0E3E093FE0B06C0E0E3E093FE0BE4E053
:10555000E0931A064AC1E091D8080E943971089573
:105560001A93E6E0EA930E94E6570E947070A091B9
:10557000D808A83539F4E2E6FAE10E944571E0E086
:105580000E947C70A091D808A33509F510E0A09185
:10559000B007A83021F0A23011F0A53009F411E3D2
:1055A000E3E5EA930E94F25B1A930E94F25BE0E863
:1055B000EA930E94F25BE0E8EA930E94F25BE0E883
:1055C0000E947770E093FE0BE0E00E947C70A09157
:1055D000D808A93459F40E944971E093FD0B0E9448
:1055E0005371EC91E093FF0B60DF11DB5DC10E9412
:1055F000047CA091D708A53411F00C943E2B0E9496
:105600005871E2E3F0E0E093D50BF093D60BA09154
:10561000D808A73741F4ECEDF8E00E945F710E94D2
:1056200064710E943971A091D808A03310F0AA3398
:1056300008F023C02091BF073091C007E8EDF8E0E3
:105640000E945F71E2E0EA930E94795B0E2F0E9454
:105650006471E093FD0B0E9464710E9468710E9466
:105660002E710A931A930E94721B2093BF073093E6
:10567000C007E2E5EA930E94E6571CC0E091D30B15
:10568000F091D40BFA93EA93E091D50BF091D60BFD
:105690000E94E47079F0E0E0E093D208E5E4EA9358
:1056A0000E94E6570E945871E8ECF0E0E093D50BB9
:1056B000F093D60B0E940B7C249608950E94476CB1
:1056C0000E948B6A0E944B6C0E948B6A0E948B6ABC
:1056D0000E945344E2E9F5E00E941F6CE091B1079B
:1056E0000E946D71E0EAF5E00E941F6CE2E0E09339
:1056F000FB030895EDE4F6E00E94AF6EE0E4F0E015
:105700000E94B46EEDECF6E00E94AF6EE0E4F0E0D3
:105710000E94B46EEEE1F6E00E94AF6E0E94836CD0
:105720000E940D67E881E03009F406C0A091B1073E
:10573000AF5FE3E00E94D679E093B1070E941021A9
:105740000E94502121C11A930A9310E0103410F0E6
:105750000C94F52B1A930E94261A00E00E94536CB9
:105760003B97C4F00E947171EA0FFB1F0F010E946A
:10577000536CD001ED93FC930E94A96F0E94C06B03
:105780000F010E94A96F0E94546EEC91EE7FD00130
:10579000EC9301E0ADECB6E00E94756F0E9456708C
:1057A0007597E4F00E947171EA0FFB1F0F01ADECD9
:1057B000B6E00E94756F0E945670D001ED93FC9385
:1057C0000E94A96F0E94C06B0F010E94A96F0E94E6
:1057D000546EEC91E160D001EC9301E0013019F4DA
:1057E0001A930E944B1A1F5FB1CF09911991089526
:1057F0001A9323FE03C00E9476711ED60E94AB400E
:10580000E03011F40C94432CE0E00E947D711038DC
:1058100018F5113219F40E9476710ED61D3439F440
:105820000E9484710E94CB5DE3E0E093AF071B32DE
:1058300061F40E948971EAE2EA93EDE6FAE1FA93F3
:10584000EA93E091B1070E948F711F3221F4E1E0E9
:10585000EA930E94E31132DF1038A8F01F770E940C
:10586000406C89F0A091BA05A23031F4E091310B7F
:10587000EA930E94E31122DFA091BA05A43019F443
:10588000E3E0E093AF070E94A46F109719F00E9425
:1058900093710CF409C0E091B707E03029F00E9441
:1058A0008D13E0E0E093B707199108950E949B7172
:1058B0000E949F710E948B6A0E948B6A0E945344CF
:1058C000A091B207A23021F4E0E7FAE10E941F6C38
:1058D000A091B207A13021F4E7E7FAE10E941F6C22
:1058E000E091B207E03021F4EEE7FAE10E941F6C8C
:1058F0000E94A9710E94896B0E9453440E94AC715E
:105900000E94B1713197FA93EA93E0915005F091BA
:1059100051050E94B6710895E1E003C0E0E001C0C6
:10592000E2E0E093B207C2DF0895A881A03310F04F
:10593000AA3308F01CC00E94BA710E94BF71AAE08D
:10594000B0E00E947C79DF01E881E0530E94C06BE7
:10595000E093BD07F093BE07E2E0E093FB030E94F3
:10596000A9710E94896B0E944B6C0E94AC71A88146
:10597000A33451F40E949F710E94A9710E94896B07
:105980000E944B6C0E94AC7121960895A0E023FC0C
:10599000A1E0A03019F0A881A03009F016C0E89469
:1059A00023F8E7E0E093AF070E949343A091C90773
:1059B000A03019F40E94C47109F407C0E7E0EA932B
:1059C0000E94C97139D5E89424F824FE18C00E94B9
:1059D000CC71EAE5F0E00E94D37119F0A881A13002
:1059E00069F455D5E03051F00E94D971E981EA930C
:1059F000E091C707EA930E9435711ED50BC00E9443
:105A0000CC71ECE2F1E00E94D37121F40E94E071CC
:105A1000E093C807EEC0E0915F0BF091600B0E942D
:105A2000E47111F4E2E00895E0915D0BF0915E0BFA
:105A30000E94E47111F4E1E00895E091630BF091AC
:105A4000640B0E94E47111F4E0E00895EFEF089513
:105A5000A091B007A23021F40E947A440E94A010C5
:105A6000A091B007A83009F441D5A091B007A530A6
:105A700009F429D10AC51A93E2E0EA930E94C83ECC
:105A8000E2E0E093FB03E981EA934FDFA981AF37BE
:105A900021F4E0911D06E37009F403C0E2E0E09315
:105AA000AF07A981A13261F0A33421F40E94BA7139
:105AB000109709F004C0A091B007A23009F011C0FE
:105AC000A091B207A33009F42BDFA091B207A23056
:105AD00019F4E1E0EA93BCDFE091B207E03009F4A9
:105AE0001DDFA981AD3311F00C94D22D0E94934398
:105AF000E091B207E030B9F4E091BD07F091BE0744
:105B0000FA93EA930E94E6211E2F113051F4E0919E
:105B1000BD07F091BE070E946871E0E0EA9398DF4C
:105B200001C0FCDE3FC0E13079F475DFEF3F41F0AA
:105B3000E3E00E94E8710E9484710E94EE7103C04C
:105B4000E1E0EA9385DF2EC0E230F1F40E94BA7101
:105B5000A034E0E0BE07B4F4E091BD07EA930E94F0
:105B6000F571E2E0E093FB030E948B6A0E948B6A6E
:105B70000E9453440E94126C0E940C12E3E0E093D6
:105B8000B20701C0CDDE0EC0E33061F4E091BD0785
:105B9000EA930E94261AE091BD07EA93EFEFEA9399
:105BA0007FD8BEDEA981AD3409F4B6DEA981A43563
:105BB00021F4A091B007A23009F001C0AFDEA981A5
:105BC000AB3231F4E091B507EF5FEA930E94E31145
:105BD000A981AD3231F4E091B507E150EA930E941A
:105BE000E311A981AF3221F4E1E0EA930E94E311CD
:105BF000188122960895E091310BE33631F4A0919B
:105C0000B007A23009F48ADE14C0E23611F488DE4F
:105C100010C0A091BA05A23011F0A63029F4E0918D
:105C2000310BEA930E94E311A091BA05A43009F464
:105C300073DE08950E9484210E947A44E0E0E0939C
:105C4000B207A881A13039F40E94C47121F0A0915B
:105C5000620BA03009F402C061DE02C00E94A010F5
:105C600014C41A930A930E94F97161F10E9406729A
:105C700048F11F770E94406C21F50E940E720E942D
:105C8000C121EF3F09F0D5C30E9435710E94E62182
:105C9000E13021F40E948220E13009F011C00E941D
:105CA0007220E83139F4E091210BEA930E94411906
:105CB000E03009F001C0BDC31A930E941D710E2F80
:105CC00001C099DFB6C30E948421E89421F8E0E086
:105CD000E093B6070E94A01008951A930E94F971EC
:105CE00051F00E94067238F01F770E94406C11F448
:105CF000C8DB01C080DF32C40E94047C0E94F971BD
:105D000011F40C94D92E0E94AE400E2F0A93B3DEEC
:105D1000A0917A0BA03021F4003810F0053808F07B
:105D20000AC00F770E94C3701081EFEFEA930E94C0
:105D30000E720A93B5DAA0917A0BA03011F00038F8
:105D400008F437C00F770A930E94261AE091310BAE
:105D5000E03071F50A93E091BB05EA930E94C121FE
:105D6000EF3F19F00E940B7C85C30E948220E13036
:105D7000F1F40E947720E03061F40A930E941D71D3
:105D8000E03031F0E091C707EA930A930E94721B5A
:105D90000EC0A091B607E02F0E94E56BAE0FBF1FAB
:105DA0001C910A930E940E72EFEFEA9379DA01C018
:105DB00022DF20FE0AC0E0917A0BE03019F4D0D344
:105DC00006D501C05FD5E89420F830E03530F0F416
:105DD000ABE03A9FF001DF01E452FA4FE081E0309E
:105DE00049F0A652BA4F0E941372E8EEF3E00E9407
:105DF000E47009F409C0ABE03A9FF001E452FA4FB5
:105E0000A0E0A083689420F83F5FE0CF0E940B7C65
:105E100031C30E94027CA091B007A33011F40C940E
:105E2000C830E091D207ED3411F00C94ED2FE091E1
:105E3000D307EA3511F00C94A22F24FC83C0E09123
:105E4000D407E0532E2FE091D507E0533E2FE6ED27
:105E5000F7E00E945F710E945371AC91AB3429F45A
:105E60000E9418720E94505B0E2F0E945371AC91D9
:105E7000A43529F40E9418720E94505BAF01E09192
:105E8000650BE31731F5E0E0E093D80B0E94D97180
:105E90004093BF075093C007A091C8070A1759F055
:105EA000E7E0E093AF070093C8072093D70BE0E04B
:105EB000E093C7070DC0A091D70B2A1721F0A0913E
:105EC000C607A03009F004C02093AF072093D70B7A
:105ED00035C0A091C807A03049F4A091660B0E947C
:105EE0002C6BE255FF4FE491EA2309F40CC0E7E084
:105EF000E093AF072093D70BE0E0E093C707E09172
:105F0000D107E093D80BE091D107A091D80BEA1705
:105F1000A9F44093BF075093C0070093C8070E949D
:105F2000D971A091D70B2A1721F0A091C607A030F4
:105F300009F004C02093AF072093D70B273011F44A
:105F40000E94546FE091D307E93439F4E7E00E94EE
:105F5000E8710E94E071E093C707E091D307E03059
:105F600039F4E4E00E94E8710E94E071E093C70711
:105F7000E091D307E03519F4E1E0E093AF07E09159
:105F8000D307EC3449F4E4E0E093AF07E091D407A1
:105F9000E053EA930E94AC17E091D307E334E9F4AD
:105FA000A091D407A13320F0A091D407A93308F021
:105FB00014C00E941B72E091BA07EA930E944C1C25
:105FC000E091D107EA93EFE8FAE1FA93EA930E94AD
:105FD000786E0E94337A0E94BE5DE091D207E03570
:105FE00021F4A091B007A13009F003C00E9489718B
:105FF00065DBE091D207EF3459F4E091D307EE343A
:1060000039F4E091D107EA93E2E9FAE10E942172C2
:10601000E091D207E33569F5E091D307EF3349F515
:10602000A091D407A03360F0A091D407A93340F425
:10603000A091D507A03320F0A091D507AA3308F08E
:1060400018C00E941B72E091D507E0531E2F10303C
:1060500011F40E94C31BE091D107EA93E5E9FAE14C
:10606000FA93EA93E12F0E94606D0E94686D0E948E
:10607000BE5DE091D207E33411F00C948D30E091D5
:10608000D307EF3311F00C948D30E091D507E03356
:1060900019F4EFEFE093BB07A091D407A03320F0F1
:1060A000A091D407A93308F01BC00E941B72E09195
:1060B000BB07EF5FE093BB07E091BA07EA93E0917B
:1060C000BB07EA930E94061BA091B30BB091B40BDF
:1060D000109721F4A091BB07A03408F001C0E7CFCE
:1060E000E091BB07EA930E94261A0E942772E8E912
:1060F000FAE10E9445710E94726D0E945E6C0E94DE
:106100007D5C0E94776D0E94337A0E947D5C0E94C4
:10611000E36D0E94A25C0E948E5DE091D207E434A0
:10612000B9F5E091D307E43499F514E0E1E0E093A8
:10613000D108103538F40E94756FE053F84FE081B4
:10614000E03208F41AC00E94756FE053F84FE08106
:10615000E33259F40E94756FEF52F84FE081E0533B
:10616000EA930E94E6571F5F06C00E94756FE053D6
:10617000F84F0E946C701F5FDCCFE091D007EA936C
:106180000E94745DEBE9FAE10E9445710E948E5D08
:106190000E94097C269608951A930A930E942C72F5
:1061A00011F40C944631E091AF07EF770E2F009376
:1061B000AF070E947A440E941A6CE4E0F0E0FA9380
:1061C000EA930E945344013021F0A091B007A1301E
:1061D00009F00BC0E8EAF5E00E941F6CB4DAE4EFC6
:1061E000F1E00E94A96A0E947A44073049F40E94B3
:1061F0008421E0E0E093B2070E94B3130E94B42828
:10620000043031F4EEE9FAE10E941F6C0E94800F25
:10621000083019F40E94327269D1053019F40E94D5
:10622000327251DD013051F4E89423F8E0E0EA9352
:1062300061DA0093B00742DA0E94A010093071F4CD
:10624000E0E0EA9357DAE0E0E093B607E89423F859
:106250000E94A0100A93E1E0EA9398DB023081F4F7
:10626000E0E0E093B607E0E0F0E00E946871E894B7
:1062700023F80A93E1E0EA9389DBE1E0EA93DADCD0
:10628000033011F40E947F3E0093B007A091B00745
:10629000A73011F00C94F2310E94DD70E4E6F0E0DA
:1062A0000E94E47021F0A091B207A03009F00AC06A
:1062B0000E94EA70E091FC0BA0911906EA1711F018
:1062C0000E94B4280E94AB40E030E9F0E2E00E9476
:1062D0007D711A932ADB1D3409F41EDB1D3399F4FA
:1062E0000E94934398DBEF3F41F0E3E0E093AF0778
:1062F0000E9484710E94EE7106C0E7E8E093AF0748
:10630000E0E0E093B207A091C707A03031F0E09140
:10631000C707A091C607EA1709F455C0E091C7075F
:10632000E150EA930E94871A0E943C72E13021F406
:10633000E0911D06EF7C09F429C0E0E0E093C60778
:10634000E091D70BE03019F0E093AF071EC012E0E8
:10635000E0911D06EC7009F018E0E0915C0BA09153
:10636000C707EA1781F0E0911D06E07439F011E0EB
:10637000EAE2EA93E3EAFAE10E942172E0911D0663
:10638000E07809F019E01093AF071DC00E947A442D
:106390000E94B3130E941A6CE4E0F0E0FA93EA93CF
:1063A0000E945344EBE4EA930E94E843E091C7075C
:1063B000EA930E943E3FE6EAFAE10E941F6CE091F8
:1063C000C707E093C607A091C707A03021F4A091AA
:1063D000C607A03009F406C0E0E0E093C607E7E88E
:1063E000E093AF07A091B007A33011F40E94893C5D
:1063F000A091B007A13009F4FBD9A091B007A23059
:1064000009F42FDCA091B007A83009F475DCA09145
:10641000B007A53009F461DCA091B007A93049F4B8
:10642000E0E0E093B807E091B007EA93E0E0EA9398
:10643000ADDA0991199108950E944172E558F84F1B
:10644000A6E0A0830E944172E658F84FAB81A0837A
:106450000E944172E258F84FAA81A0830E944172C3
:10646000E458F84FA881B981A083B1830E9443709A
:106470000E94DA4A24960895E881EF5FE883A881B4
:10648000A53010F0E0E0E883E88121960895A0911E
:10649000AA07BB27E091A90705C0A091A807BB27C1
:1064A000E091A707F0E031960E94FE6E3596DF017D
:1064B000E5E0F0E00E94D97908951A931091AA07B7
:1064C000E091A907E11781F0A9E01A9FF001E558D2
:1064D000F84FE081E13011F0E23011F4E1E03EC02C
:1064E0001A93CADF1E2FECCFE0E038C01A930E9447
:1064F0008421E2EDF5E00E94AF6EE7E3F0E00E9458
:10650000B46E10E0153050F40E94B870AFEFA08365
:106510000E94B2700E94BE701F5FF4CFEEE3F6E0FF
:106520000E94F46E0E940D67E0911D06E37019F061
:106530000E94C47109F402C0689401C0E89421F873
:10654000EFEFE093C507E0917A0BE03029F408D033
:106550003ED1E89420F802C00E94311119910895AB
:106560000E94027C00E0053058F40E944772A0E0CF
:106570000E944D72EB52FA4FA0E0A0830F5FF3CF61
:1065800000E0053078F50E94C370E081EF3F41F1F3
:106590000E94C370E0810E943E6FB1F00E94C970FA
:1065A000DF010E94207A0E940E6FEA17FB0741F07C
:1065B0000E94C9700E940E6FA083B1830E94527224
:1065C0000E944772A1E00BC0ABE00A9FF001E452C9
:1065D000FA4FE081E03021F40E94C370AFEFA08356
:1065E0000F5FCFCF0E94B11F1E2F1F3F11F40C94DD
:1065F000493350E000E0053048F40E94C370E08168
:106600001E1711F451E002C00F5FF5CF5030D1F5E5
:1066100000E00530B8F50E94C370E081EF3F81F5DE
:106620000E94C37010830E94C9700E940E6FA083E5
:10663000B183ABE00A9FF001EA52FA4FA091BE0B82
:106640000E944D72E952FA4FFF93EF930E94356F0B
:106650000E943A6FAF91BF91EC930E9452720E94D8
:106660004772A1E00E944D72E652FA4FFF93EF93FA
:106670000E94FA61AF91BF91ED93FC9351E002C08B
:106680000F5FC7CF503029F01A930E94B81F1E2FFA
:10669000ACCF30E03530D8F550E000E0053048F5BB
:1066A000503029F5ABE00A9FF001E952FA4F208102
:1066B0002A930E94261A0E944772E081E13059F421
:1066C0002A930E949120E13031F4A32FAF5FE09133
:1066D000350BEA1709F00BC00E942C6BE65DF94FF1
:1066E00020830E942C6BE25CF94F008351E00F5F26
:1066F000D5CF503051F40E942C6BE65DF94F0E94CB
:10670000DA70E25CF94FAFEFA0833F5FC3CF0C9428
:106710004A380E94047CAC81BD81EBE4EC93EC81AF
:10672000FD8131960E945A72EA52FA4FE0810E942E
:10673000657200E00E946F72EC91E03011F00F5F23
:10674000F9CF0E946F72E0E2EC930F5FE02FAC8113
:10675000BD810E94C06B0E945A72E852FA4FDF015D
:106760000E94207A0E945E6C0E947572EE81ABE0FE
:10677000EA9FF001E952FA4F10811A930E94261AFB
:1067800000E00E946F72EC91E03011F00F5FF9CFE2
:106790000E946F72E8E7EC930F5F0E946F72E0E275
:1067A000EC930F5F30E03A3068F4E02FAC81BD81AC
:1067B0000E94C06B0F01A2E2BBE00E947A720F5FE1
:1067C0003F5FF1CF0E946F72EC930C94BE366497DA
:1067D0000E94047C00E010E0153040F40E94B87084
:1067E000E081EF3F09F40F5F1F5FF6CF053021F026
:1067F000A091C507A03009F406C0E0E0E093C5070A
:10680000EA930E946F12053021F4A091C507A130D0
:1068100009F406C0E1E0E093C507EA930E946F1215
:1068200010E0153058F5ABE01A9FF001DF01ED5292
:10683000FA4FE081E03031F0FD01EB52FA4FE08198
:10684000E03009F419C01A930E94CF7062DFABE008
:106850001A9FF001E952FA4F30813A930E94261AAA
:106860001A930E94CF700E94C912ABE01A9FF001E8
:10687000EB52FA4FA0E0A0831F5FD3CF0E940B7CA6
:10688000689608950E94027CA0917A0BA23011F4C0
:106890000C944A3830E0343160F40E9481720E94D6
:1068A0008472DA011296E0E0EC93DA01EC933F5F38
:1068B000F2CF0E94B11F0E2F0F3F11F40C94A134A0
:1068C0000E94356F0E943A6F1E2F1F3F31F0E091FA
:1068D000B6071E1710F0103408F02EC0A091B607AE
:1068E000E12FEA1B3E2F3431F0F40E9481720E94A6
:1068F0008472FA0132960F01E081AE2F0E948A72F3
:106900000E948F72D001EC93FA01A281A43620F08C
:10691000DA011296E3E6EC93DA01AC91AF3F19F499
:10692000E02FDA01EC931A930E94356FFA93EA9301
:106930000E94E5191E2FC9CF0A930E94B81F0E2F7F
:10694000BBCF30E0343110F00C9419350E948172C5
:106950000E948472FA01A381AF3F11F40C941735A1
:106960000E9493720E94261AA091320BA07839F4EB
:10697000FA010280DA011196EC91E01509F457C092
:10698000DA0113962C91ACE02A9FF001E05FFC4FF6
:106990000F01DA011296EC91D001EC930E949372F0
:1069A0000E949D21EF3F41F0ACE02A9FF0010E9440
:1069B0008D6FE058DB01EC93DA011296EC91E03038
:1069C000A1F0ACE02A9FF001E45FFC4FDF010E94E0
:1069D000E06BEC93ACE02A9FF001E35FFC4FDF013A
:1069E000E091300BEF70EC930EC0ACE02A9FF00109
:1069F000E35FFC4FA7E0A083ACE02A9FF001E45FD7
:106A0000FC4FA8E0A0830E9493720E949D21EF3F5B
:106A100019F0ECE0E093FC03DA011296EC91DA0154
:106A20001196EC932A93E1E0EA930E94DD443F5FE4
:106A300089CF0C944A38E7E0E093AF070E946D19C4
:106A4000A8950E94B81DA8950E94FA1FA895EFEF7F
:106A5000E0934A0BE093210BE093C80BE093C30B48
:106A60000E949972EC7F29F0A8E0B0E0E0E00E947B
:106A7000627A089568970E94027CE4EBFAE10E9432
:106A8000AF6E0E944E400E94F63FE091BA07E030A0
:106A900061F0EFEBFAE10E94AF6E0E944E40E09190
:106AA000BA070E949E720E94A2720E94F63F0E9444
:106AB000C31B30E03A3080F43A930E94526DEFE00D
:106AC000EA930E942840E32F0E94606D0E94686D47
:106AD0000E94A6723F5FEECF0E940A40E8ECFAE106
:106AE000FA93EA93EFE0EA930E944E400E94476DCA
:106AF0000E94A6720E940C400E94F63F00E0003106
:106B000010F00C9434360E946D6CE01711F00C9468
:106B1000CB35EEECFAE10E94AF6E0E944E400E942F
:106B2000136BFA93EA930E94A272E0E0E093B60737
:106B3000A091B607A03458F5E091BA07EA93E09126
:106B4000B607EA930E94061B0E94726D3097C9F047
:106B5000E091B607EA930E94261A0E94726DFA939A
:106B6000EA930E94AA720E944E400E94E36DEAE0FE
:106B7000EA930E9428400E94776D0E94337A0E9417
:106B8000A672E091B607EF5FE093B607D1CF0E94FF
:106B9000F63F0E94F63F0E94136B0E948E6E11F02A
:106BA0000C943236EEECFAE10E94AF6E0E944E4039
:106BB0000E94136BFA93EA930E94A2720E94AF7232
:106BC000E0E30E949A6E51F413E0EDB7FEB7FA933A
:106BD000EA931F930E94205D1F91AF01042E052AA6
:106BE000E9F11F5FEDB7FEB7FA93EA931F930E9496
:106BF000E45C1F91EA8FFB8F6C8F7D8F1F5FEDB779
:106C0000FEB7FA93EA931F930E94B7720E94475D02
:106C10001F915A934A930E94AA720E944E400E946A
:106C2000BC72EAE0EA930E942840EA8DFB8D6C8DED
:106C30007D8D0E94337A0E94A6720E94AF72E1E3BA
:106C40000E949A6E51F413E0EDB7FEB7FA93EA93FF
:106C50001F930E94205D1F91AF01C0CF0E94F63F9D
:106C60000E94F63F0F5F4BCF0E94DF3F0E94097CDE
:106C70006E9608950E94047CAC81BD81EC91E17018
:106C80002E2F0E94C1720E94086C0E94136B0E94FA
:106C9000C672E4E0EA930E944344203019F4EBED1D
:106CA000FAE102C0E0EEFAE1FA93EA930E94FE43B1
:106CB0000E94B17134970E942B710E94B6710E949C
:106CC000AE403E2F333409F431E20E9493433D330A
:106CD00011F0313209F402C0E1E02E273D3311F00A
:106CE000313209F401C0CFCF3D3319F4AC81BD81FD
:106CF0002C93E32F0E940B7CCFC10E94047CAD81BA
:106D0000BE812C910E94C1720E94086C0E94136B7C
:106D10000E94C672ECE3EA930E94E843EC81EA9396
:106D20000E9443442A93ED81EA930E94093FEEE3D7
:106D3000EA930E94E8430E94CA720E94B6710E94C0
:106D4000CD72333409F431E2313320F0EC81E05D6F
:106D5000E31708F407C0E32F0E94D272E255FF4FF9
:106D6000E4912E273D3311F0313209F401C0CCCF2C
:106D70003D3319F4AD81BE812C93E32F0E940B7C2F
:106D8000279608950E94027C20E0AF81B8855C912F
:106D90000E94C1720E94086C0E94136B0E94C6720E
:106DA000E2E0EA930E9443445A930E943E3F0E94CD
:106DB000CA720E94B6710E94CD72303310F03A331D
:106DC00008F00EC0203009F450E021E0A52FEAE0E1
:106DD0000E94D679AAE0EA9FF001E30FE0535E2F0C
:106DE0003B3211F4533608F001C05F5F3D3211F4BD
:106DF000513008F401C05150333429F4203009F4E3
:106E000031E250E020E03D3319F4EE81E51708F05F
:106E100005C0AF81B8855C9130E020E03D3311F0D2
:106E2000313209F401C0B6CF3D3319F4AF81B885D2
:106E30005C93C8C00E94027C20E0AF81B8854D9170
:106E40005C910E94C1720E94086C0E94136B0E94A8
:106E5000D572AE81A23031F4FA010E945E6C0E94BC
:106E60001F3F04C05A934A930E94263F0E94CA7251
:106E70000E94B6710E94CD72303310F03A3308F0A0
:106E80001EC0203011F440E050E021E04031E7E244
:106E90005E0734F0DA01E0E1F7E20E94D979AF0150
:106EA000493BEBE05E0724F0DA010E94BF71AF01BD
:106EB000DA010E94D8720E94DD72D097AD013B3298
:106EC00021F44033E5E75E070CF002C04F5F5F4FEF
:106ED0003D3221F40024041605060CF002C0415096
:106EE0005040333431F4203009F431E240E050E0D6
:106EF00020E03D3311F0313209F401C0A4CF3D331D
:106F000021F4AF81B8854D935C935CC00E94027CF4
:106F10000E94C17220E050E04FEF0E94086C0E9476
:106F2000136B0E94D5720E94E272E885EA930E9478
:106F30001544E52FE10FF0E00E942B710E94B6711D
:106F40000E94CD72303310F03A3308F023C0305332
:106F5000431729F04F3F09F05F5F20E005C0A22FE3
:106F6000AF5FEA2FE3702E2FE52FAF81B8850E9427
:106F7000C06B0F01E32FA8E3B7E0F0E00E942E7989
:106F8000AE0FBF1F0E948C6BEA0FFB1FE491D00174
:106F9000EC93432F3B3219F4EE815E1708F002C0E8
:106FA0005F5F4FEF3D3211F4513008F402C0515091
:106FB0004FEFEE815E1720F4313211F03D3309F4CA
:106FC00001C0ABCFE32F0E94097C299608951A9344
:106FD0000A93A091320BECEDEA231E2F00E00C3057
:106FE00040F40E94E7723A96E491E11711F00F5FC6
:106FF000F6CF0E94E7720E941F6CE02FE4C3A2E369
:10700000BBE0E8810E94546EEC91E17019F4E5EE6A
:10701000FAE102C0E9EEFAE1FA93EA930E94FE4334
:10702000219608950E94027C0E94C1720E94086C01
:107030000E94136B0E94D572CADF5E2F0E94CA7233
:107040000E94B6710E94CD723D3211F0363311F4B8
:10705000503009F401C051503B3211F0333311F478
:107060005B3008F001C05F5FA091320BE1E0EA23E2
:107070002E2FACE05A9FF001E450FC4F3A96E49179
:10708000E20FE093320B3D3311F0313209F401C0CD
:10709000CDCFE32F0E94097C269608950E94047CA0
:1070A0000E94C1720E94086C0E94136B0E94D572EC
:1070B000EC81EA93A4DF0E94CA720E94B6710E941A
:1070C000CD72303310F03A3308F010C0A2E3BBE0C9
:1070D000EC810E94C06B0F01A2E3BBE0EC810E9437
:1070E000546EAC91E1E0EA27D001EC933D3311F00E
:1070F000313209F401C0D6CFA091320BE2E0EA238D
:107100002E2FE091330BED7FE22BE093330BE091D8
:10711000340BED7FE22BE093340BE32F0E940B7CCA
:10712000259608950E94FE6A0E9476100E948B6A3E
:107130000E948B6A0E9453440E94E36DEAE0EA9346
:10714000E5DEE13209F4CAC30E948B6A0E948B6AB1
:107150000E944B6CEDEEFAE10E941F6CEDE2FBE049
:107160000E94AF6E67DEE13209F4B8C30E948B6AF9
:107170000E948B6A0E944B6CE3EFFAE10E941F6C45
:10718000EFE2FBE0FA93EA93EAE00E94ED7209F481
:10719000A5C30E948B6A0E948B6A0E944B6CECEF25
:1071A000FAE10E941F6CE4E4FBE00E94F27209F431
:1071B00095C30E948B6A0E948B6A0E944B6CE2E02E
:1071C000FBE10E941F6CE6E4FBE00E94F27209F40E
:1071D00085C30E948B6A0E948B6A0E944B6CE8E018
:1071E000FBE10E941F6CE1E3FBE0FA93EA93E3E624
:1071F0000E94ED7209F472C30E948B6A0E948B6A2E
:107200000E944B6CE1E1FBE10E941F6C0BDFE1325D
:1072100009F464C310E0133010F00C9497390E9405
:107220008B6A0E948B6A0E944B6CE12F0E946D71E9
:10723000E7E1FBE10E941F6C0E94FA720E94534436
:10724000A5E3BBE0E12F0E94C06BFA93EA93E0E173
:107250000E94ED7209F442C3E9E0F0E00E94896BFC
:107260000E945344A8E3BBE0E12F0E94C06BFA9355
:10727000EA93E0E10E94ED7209F430C30E948B6A48
:107280000E948B6A0E944B6CE12F0E946D71E2E2BA
:10729000FBE10E941F6C1A9301DFE13209F41EC367
:1072A0000E94FA720E94FD7249F40E9453700E947B
:1072B00007730E94F27209F411C30AC00E9453704E
:1072C0000E9407730E94AF6EB5DDE13209F406C378
:1072D0000E948B6A0E948B6A0E944B6CE12F0E9475
:1072E0006D71E4E2FBE10E941F6C0E94FA720E9441
:1072F0005344A1E4BBE0EE27A10FBE1F2C9133271E
:10730000EDB7FEB73197FA93EA933F932F93E0E0FE
:10731000EA9390DD2F913F91E13209F4DFC2A1E4BD
:10732000BBE0E12F0E94C06B20831F5F74CFD6C2E9
:107330000E94047C10E01A930E94F5710E940C7365
:107340000E948B6A0E9410730E94626E0E94076DF9
:107350000E948B6A0E941A6C0E9453440E945D6EC8
:107360000E945E6C0E941F3F0E94686C0E941A6C13
:107370000E945344E091460BF091470B0E945E6CD3
:107380000E941F3F0E948B6A0E940D6C0E94534412
:10739000EBE2FBE10E941F6CE0912F0BEA930E944D
:1073A0003E3F0E94686C0E940D6C0E9453440FDEA9
:1073B0000E944F6C00E00330C0F50E948B6AE02F02
:1073C000ED5F0E946D6D0E948170EA930E943E3FC6
:1073D000EBE2EA930E94E8430E948870EA930E94DD
:1073E0001C730E948F7051F40E9497700E94567017
:1073F0000E945E6C0E941F3FE3E707C00E949770E7
:107400000E9456700E94076DE9E4EA930E94E843E7
:107410000E944F6C0E949F70EA930E94433FE3E7F3
:10742000EA930E94E8430F5FC6CF0E94AE403E2F12
:107430003B3211F4103408F001C01F5F3D3211F4EB
:10744000113008F401C011503D3439F41A930E94F0
:10745000261A68DE1A930E944B1A313209F06BCF5C
:107460003DC20E94047C10E00E947A44012F0E94D9
:107470008B6A0E948B6A0E945344EFE2FBE10E94F8
:107480001F6C31E03C3020F5103800F50E948B6A0B
:107490000E942C6B0E94C6721A930E94871AE12FD9
:1074A000EF5FEA930E941C730E943C720E941F735C
:1074B000A091CA0BE7E0EA230E941F73E0911D062A
:1074C000EA93E8E0EA930E94093F13953F5FDACF21
:1074D0000E94800F0E94AE403E2F3D3411F00C946C
:1074E000B03A0E949B71102F1038D0F51A930E9469
:1074F000871A0E948B6A0E948B6A0E944B6CE3E49D
:10750000FBE10E941F6C0E9423730E94026B0E9489
:107510008B6A0E945344E6E4FBE10E941F6CE9EC95
:10752000FBE0FA93EA93E1E00E94ED7209F4D6C120
:107530000E94026B0E948B6A0E944B6CECE4FBE1A0
:107540000E941F6CEAECFBE0FA93EA93E7E00E94EA
:10755000ED7209F4C3C11A930E94BB1A1F5FC4CF16
:10756000313211F0103808F001C07ECFB7C10E944F
:10757000FE6A0E940C730E948B6A0E945344E2E5EB
:10758000FBE10E941F6C10E01530E0F41A930E949A
:10759000C91A0E948B6A0E94596D0E942373E09160
:1075A000C40B0E941F73E091C70B0E941F73E091F0
:1075B000C50B0E941F73E091C60BEA930E94433FE4
:1075C0001F5FE2CF0E94AE400E2F0D34C9F50E941E
:1075D0009B7110E01530A0F51A930E94C91A0E9401
:1075E0008B6A0E948B6A0E944B6CE5E6FBE10E946D
:1075F0001F6C0E94237330E03430E8F40E94026B69
:107600000E948B6A0E944B6CA6E13A9FF001E05207
:10761000F94F0E941F6CA6E13A9FF001E052F94F2A
:107620000E942C73FD017296E4910E94ED7209F4A0
:1076300055C13F5FE1CF1A930E94E91A1F5FCACF7D
:107640004DC10E944F6A0E94761000E0053210F092
:107650000C94E33B0E941E0F0E948B6A0E948B6A6F
:107660000E9453440E942F7331960E941F6C0E9407
:107670004F6C0E942F730E943573A9F40E946D6CA9
:107680001E2FEDB7FEB7FA93EA931F93E0E1EA935A
:1076900079DB1F91E13209F496C0E12FA9E0B0E057
:1076A0000E94627A8CC0E238A0E0FA07A9F40E9436
:1076B000B86E1E2FEDB7FEB7FA93EA931F93E0E181
:1076C000EA9360DB1F91E13209F47DC0E12FAAE06B
:1076D000B0E00E94627A73C0E138A0E0FA07E1F4FA
:1076E0000E9499721E2FEDB7FEB7FA93EA931F938B
:1076F000E3E0EA9347DB1F91E13209F464C00E94A2
:107700001E0F0E949972E11731F0E12FA8E0B0E05E
:107710000E94627AFFCF53C0309751F40E942F73BA
:107720003E960E94236CA6DAE13209F44CC047C0B1
:10773000E130A0E0FA0761F40E942F730E942C73DD
:10774000FD017296E4910E94ED7209F43CC037C0CD
:10775000E230A0E0FA0761F40E942F730E942C73BC
:10776000FD017296E491EA9365DBE13261F127C095
:10777000E330A0E0FA0761F40E942F730E942C739B
:10778000FD017296E491EA93B8DAE132E1F017C0B4
:10779000E430A0E0FA0799F40E942F733E960E940D
:1077A0002F7AE093040CF093050CFA93EA930E946D
:1077B0002F737296E491EA93A9DBE13221F00E94E3
:1077C00070190F5F43CF0991199108951A930E9480
:1077D0007A440E94761010E0133068F50E948B6A9C
:1077E0000E948B6A0E944B6CE12F0E946D71E0EF4A
:1077F000FAE10E941F6C1A9302DC0E94026B0E9445
:107800008B6A0E94FD7251F40E9453700E940773AC
:107810000E94F27211F40C94C8400BC00E94537085
:107820000E9407730E94AF6E05DBE13211F40C94E5
:10783000C8401F5FD1CF0C94C8400E94047C10E068
:107840001A930E94F5710E940C730E948B6A0E9429
:10785000107300E0033038F50E94076BE02FEE5FF5
:107860000E946D6DE02F0E946D71EAE3EA930E9421
:10787000E8430E944F6C0E948F7049F40E949770F9
:107880000E9456700E945E6CDAD2E3E707C00E9445
:1078900097700E9456700E94076DE9E4EA930E9477
:1078A000E8430F5FD7CF0E94AE403E2F3B3211F42A
:1078B000103408F001C01F5F3D3211F4113008F49C
:1078C00001C011503D3439F41A930E94261A7EDF0C
:1078D0001A930E944B1A313209F0B2CF0E940B7CEE
:1078E000249608950E949B710E948B6A0E948B6A65
:1078F0000E945344E8E6FBE10E941F6CE1E0E09344
:10790000BA07EAEBF7E0FA93EA93E5E0EA933ADAAA
:10791000089522970E94027C0E94AE400E2FE091B3
:10792000B207E03011F00C94293E0132D1F4EAEBB9
:10793000F5E0A091CF0BB091D00BEA17FB0761F4F3
:10794000E7E0E093AF07EAE2EA93E1E7FBE10E94B8
:10795000AF6E0E94CB5DABC0E0E0E093B5050E9446
:107960003C730D3331F4E091B505F0E00E94326BC9
:1079700004910D3441F4EAE2EA93E4E7FBE10E946A
:10798000AF6E0E94CB5D063449F4E0E7F6E0E09389
:10799000CF0BF093D00BE0E0E093B505003311F08E
:1079A0000B3229F4E091B505EF5FE093B5050D3298
:1079B00029F4E091B505E150E093B505013329F4D0
:1079C00091DFED3311F40E944373033321F48ADF16
:1079D000ED3309F44FD8063321F4E0E0E093BA0721
:1079E00049D8043329F4E0E0E093BA070E944373D6
:1079F000093411F40E94150FA091BC07A13010F4B6
:107A00000C94C13D023301F56DDFED33E9F40E94C2
:107A10005073D1F4E091BA07EA930E944C1C30E015
:107A2000303190F40E942C6B0E948E6E59F4E32F3B
:107A3000E05DEA93E7E7FBE10E94936EE0E3EA93FF
:107A40000E94EE5D3F5FECCF053331F5E0E0E0935F
:107A5000BA070E94507301F511E01630E8F41A934A
:107A60000E944C1C30E03031A8F40E942C6B0E9424
:107A70008E6E71F4E32FE05DEA93E7E7FBE1FA93A2
:107A8000EA93E12FE05DEA93E0E3EA930E94EE5D82
:107A90003F5FE9CF1F5FE1CF013469F4EAE2EA9387
:107AA000EAE7FBE10E942172E1E0E093AF070E9468
:107AB000097C289608950A3409F4BFDE073311F0D3
:107AC0000C94C13D0E947A44E0E0EA930E94AA0F20
:107AD000E1E0E093B307E0E0F0E0E093AB07F09380
:107AE000AC0730E0353030F40E942C6B0E949F6F61
:107AF0003F5FF8CF0E94FA61EE83FF830E945973C3
:107B0000EEE1F0E00E94E47031F00E9408140E945F
:107B1000FA61EE83FF83E5E0F0E00E94A96A40E0AD
:107B200050E00E94937184F0E0915C05F0915D0556
:107B3000EF57F0403E2F313010F0313108F004C0E3
:107B4000E32F0E94606FAF014093AB075093AC07E7
:107B50000091D105E0E0E093D105013211F00B3244
:107B600009F401C0CBCF0B3221F4E1E0EA930E948B
:107B7000AA0F013209F0B5CFE0E0E093B307E0933C
:107B8000D105A091BC07A23011F00C94223E09331C
:107B900009F457DD053409F4EADC033611F40E94D8
:107BA000C40E083309F4C4DB023409F45ADC03348C
:107BB000A1F51091CE0B0E947A4400E0E091CD0B2C
:107BC000E11711F00C3008F01CC00E948B6A0E9473
:107BD000136B0E94C6721A930E94BE1F1A930E94D2
:107BE0001C73E091BE0B0E941F73E091C10B0E94B9
:107BF0001F730E94356F0E94076D0E94276F0395C7
:107C0000DDCF0E94800FAAD20E2F013221F0E09129
:107C1000CD0BE11709F401C0CECF043499F40E94D2
:107C2000507381F4A0916B0BA03021F4A091690BEB
:107C3000A03031F00E94C9710E948B6A0E94CF4C23
:107C40000E944B1EE091B207E03011F40E94D80F61
:107C50004DC0E130B9F4A091B907AB3010F4013256
:107C600009F405C00E9463170E94800F0AC0E0E07B
:107C7000E093B6070E945E730E946773E2E0E093B0
:107C8000B20734C0E23091F5013269F4E0E0E093EC
:107C9000B2070E947A44EAE2EA93E4E7FBE10E9439
:107CA00021720E94D80F0B3281F4E091B607EA5F8F
:107CB000E093B607A091B607A03418F0EAE3E0938A
:107CC000B6070E945E730E9467730D3279F4A0912B
:107CD000B607AC3020F0E091B607E65001C0E0E016
:107CE000E093B6070E945E730E946773A091AF078E
:107CF000A33009F411CE0E94097C0C9410431A930E
:107D0000E3E0E093B0070E947A440E948B6A0E94ED
:107D10008B6A0E945344E0E8FBE10E941F6C0E94C2
:107D20008B6A0E941A6C0E945344E9E0F6E00E94BC
:107D3000AF6EE0E1F0E00E94B46E10E0E091610B04
:107D40001E17E0F4E12FE05DEA93E8E8FBE1FA9327
:107D5000EA93E0E3EA93E0E00E949A6E49F40E941D
:107D6000756FE75FF94FA1E0A083E12FE05D01C0EF
:107D7000EEE2EA930E94E8431F5FE0CF0E943C736B
:107D8000E0E0E093B505E093B2070E94D80F00C28F
:107D9000E881E03021F4E6E6F7E00E946E73A88106
:107DA000A13021F4E0E6F7E00E946E73A881A230D2
:107DB00021F4ECE6F7E00E946E73A881A33021F471
:107DC000EAE7F7E00E946E73A881A43021F4E0E8AE
:107DD000F7E00E946E7302C51A930A93E0E0E09305
:107DE0007205E093730510E0143190F400E0033065
:107DF00068F4A3E01A9FF001E758FA4FDF01EE277D
:107E0000A00FBE1FE0E2EC930F5FF1CF1F5FECCF3E
:107E10007CC31A9311E0E981E11780F00E94756F2D
:107E2000E255FF4FE491AA81EA2319F0E12FE05DCA
:107E300001C0E0E2EA93CCD41F5FEDCFE8C00E941E
:107E400073730E9478730E949A73F4C00E947373D4
:107E50000E949E730E9475720E94A573F7C00E94D3
:107E60007373E3EAFBE1FA93EA93EE85FF850E94E0
:107E70005E6C0E9475720E94A573E8C00E947373C5
:107E8000E6EAFBE104C00E947373EAEAFBE1FA93BD
:107E9000EA93EE850E9465720E94A5732B96089561
:107EA0000E94047C10E0E1E3E093D008E89431F80C
:107EB000EA930E94745DEEEAFBE10E94457100E0E6
:107EC000E09177050E17E0F40E94136BE758FA4F24
:107ED000E081E03258F4E3E2EA930E94F25B0E9410
:107EE000136BE758FA4FE081E05D05C00E94136B09
:107EF000E758FA4FE081EA930E94F25B0F5FE0CF10
:107F00000E94A7739F010E94F4163A932A93E8EC0B
:107F1000F0E0FA93EA930E9406620E2FA0E031FC93
:107F2000A1E0A03011F4003009F001C0ECCF31FE27
:107F300009C0E0E0E0937705E89431F8E1E00E94C1
:107F40000B7CD6C41F5F123008F4ADCFE0E0E093A5
:107F500077050E940B7CCCC4E0917605E03021F4DB
:107F6000E881EA930E94E657A0917605A13021F4BA
:107F7000E881EA930E94855AA0917605A230F1F437
:107F8000E0917705F0E0E758FA4FA881A083E091EF
:107F90007705EF5FE0937705E0917805EF5FE09379
:107FA0007805A03218F4EF5FE0937805A09178058A
:107FB000A73321F475DFE0E0E09378050FC4A091CA
:107FC0007605A13039F4E8ECF0E00E94EC6CE9E1D0
:107FD000E0939900A0917605A23021F461DFE0E002
:107FE000E0937805E0E0E09376050895EDE0EA930C
:107FF000B3DFEAE0EA93B0DF08951A9310E0E98175
:108000001E1728F4EA81EA93A7DF1F5FF8CF1881D3
:1080100023960895EDE201C0EDE3EA93E8E2EA93E6
:10802000ECDFE4DF08950E9473730E9478730E946E
:10803000AF6E0ED02E9608950E9473730E949E73A9
:108040000E947572FE010E94AF6E02D02C960895B8
:108050001A930A9310E0EA81E03011F408E201C0BB
:108060000A81AB81BC81EE27A10FBE1FAC91A0306D
:1080700011F0101708F007C0AB81BC810E94AB73F0
:108080000E94B073EECFEA81E03039F0EA811E172A
:1080900020F4E0E20E94B073F9CF27C01A930A934C
:1080A00010E0EA81E03011F408E201C00A81E12F1A
:1080B000AB81BC810E94C06BE491E03011F01017DD
:1080C00008F009C0E12FAB81BC810E94C06BE49134
:1080D0000E94B073ECCFEA81E03039F0EA811E17DC
:1080E00020F4E0E20E94B073F9CF1981088125964F
:1080F0000895E091B905A091B805EA17B1F00E9482
:10810000B573AE0FBF1FEC91E093BB050E94B57332
:10811000EA0FFB1FE181E093BA05A091B9050E9427
:10812000BA73E093B905E1E00895E0E008950E9494
:10813000BF73EA0FFB1FA981A0830E94BF73EA0FE0
:10814000FB1F3196A881A083A091B8050E94BA7345
:10815000E093B8053BC3E091D10508951A93E091EF
:10816000D105E03059F40E94F4160E942C7221F4DB
:10817000A091D105A03009F001C0F5CF1091D10533
:10818000E0E0E093D1050E942C7209F011E2E12FAA
:10819000199108950E94047C0E94FA618F010E9447
:1081A000F416EC81FD81E00FF11FFF93EF930E9425
:1081B000FA61AF91BF91AE1BBF0B9D010024021667
:1081C00003061CF40E942C7209F001C0E8CFE0E025
:1081D0000E940B7C269608951A93E9810E94AC7048
:1081E000A0E0A0830E94C473108117FF05C0E12F97
:1081F0000E94CB73A0E0A08316FF05C0E12F0E9470
:10820000D273A0E0A0830E94C473A0E0A083E981A0
:108210000E94A670A0E0A0831881D8C20E94047CAE
:1082200030E0EE81ACE0EA9FF001E15FFC4F1081AD
:1082300016FF17C0E12FEF730E2F0E94D97311F0B4
:108240003A3008F009C00E94E173DF010E942C6BF4
:108250000E94E7733F5FF1CF0E94E1730E94DD72DD
:10826000EC9317FF17C0E12FEF730E2F0E94D97305
:1082700011F0343108F009C00E94ED73DF010E9453
:108280002C6B0E94E7733F5FF1CF0E94ED730E9459
:10829000DD72EC930E940B7C44C2A0970E94027C8A
:1082A000EDA5FEA5A9A9BAA9EA0FFB1FAF01E5E05C
:1082B000F3E0EE83FF8310E01431D0F5AE81BF818F
:1082C000AC91A03059F10E94F36FEFA5F8A9EA171D
:1082D000FB0721F5EE81FF81A181B281E9A9FAA90D
:1082E000AE17BF07DCF0EE81FF81A181B2814A1792
:1082F0005B07A4F00E94F3730E94F873AE0FBF1FD8
:10830000E9A9FAA9AE17BF074CF00E94F3730E94C7
:10831000F873AE0FBF1F4A175B070CF402C01A9325
:108320005BDFEE81FF813C96EE83FF831F5FC4CF4E
:10833000E5E0F3E0EE83FF8310E0143110F00C94DD
:108340004342AE81BF81EC91E03011F00C943C428D
:10835000EAA5EC93E9A9FAA9AE81BF811196ED9344
:10836000FC93EFA5F8A9AE81BF811396ED93FC9322
:10837000EDA5AE81BF811596EC93EBA5AE81BF81D3
:108380001696EC93E091F503A091FC03EA27AE81E9
:10839000BF811796EC93E091FD03AE81BF811896E3
:1083A000EC93E091FE03AE81BF811996EC93AE8110
:1083B000BF811A96E0E0EC93AE81BF811B96EC93EF
:1083C000E887E8A5F9A5309741F00E94B7720E94AE
:1083D000FB73E4E1EA930E946167EEA1FFA130978D
:1083E00051F00E94B772E8A5F9A5FA93EA93E4E187
:1083F000EA930E944D67E0E0EC8F0E94B7720E9402
:1084000038673E2F3B30C8F000E00E94ED73E081FA
:10841000E03011F0053008F002C00F5FF6CF0E9487
:10842000ED73E081E03049F40E94ED730E94007426
:10843000E058AE81BF811A96EC93E0E0EA8B3130D0
:10844000C8F000E00E94E173E081E03011F00431F7
:1084500008F002C00F5FF6CF0E94E173E081E030C8
:1084600049F40E94E1730E940074E05CAE81BF8118
:108470001A96EC93E12F08C0EE81FF813C96EE83C3
:10848000FF831F5F5ACFEFEF0E94097CE3960895A8
:108490001A930A930E940B743097B9F1E0914C053E
:1084A000F0914D05309769F50E940B740E942F7A68
:1084B000E0934C05F0934D05309731F4E0E0F0E0A7
:1084C0000E946E73E0E01AC00E9410740E940B7448
:1084D0000E942F7AF595E7958F01D801E0E0F1E051
:1084E0000E94A779E0938700D801E0E0F1E00E94C4
:1084F000D979E09386000E941074E0E4E0938B0049
:1085000004C0ACE4B5E00E9430700991199108955F
:108510000E94047C00E025E033E010E01431A0F577
:10852000D901EC91E03061F111960E94207A0E940D
:1085300018740CF5D90113960E94207AAC81BD8184
:10854000EA17FB07C4F4F90101801280D9011596DE
:108550000E941D74AE81BF81AE17BF0764F4F9019C
:1085600003801480D90116960E941D74AC81BD81D0
:10857000AE17BF070CF004C0E12FEF5F0E2F04C051
:10858000245F3F4F1F5FCACF003079F0E09156055E
:10859000F0915705A02F0E94D16E31F0A0915605A1
:1085A000B0915705109709F401C030C00E94AE6C1D
:1085B0001597B9F40A93E1E0EA93B9DD0E94136BD1
:1085C000E0935605F09357050E94136B0E942274A6
:1085D000D9010E9427740E942A74E3E0F0E00E940F
:1085E000C36C0E94AE6C5E9721F4E4E0F0E00E9460
:1085F000C36CA0914A05B0914B05139734F0E5E0A8
:10860000F0E0E0935405F093550508C00E942F74E4
:108610000E94C36CE0E0F0E00E9436740E940B7C84
:1086200028960895E0915605F09157053097A1F0EE
:108630000E94AE6C999734F4E0915605EA93E2E01B
:10864000EA9375DD0E94AE6CDD9734F0E09156053B
:10865000EA93E4E0EA936BDDE0E0F0E00E94C36CB3
:108660000E942F740E943674E0E0F0E0E09356051B
:10867000F0935705E0935205F093530508953AD1CE
:10868000ABDBE5E1E093D0050895EA81E093740562
:10869000E881E0937505E091F603E061E093F6036D
:1086A00027C10E94027CA0917405A43120F4A091FE
:1086B0007505A33008F033C0E0917405F0E0ACE03C
:1086C000B0E00E947C798F01E0917505F0E0A4E1B3
:1086D000B0E00E947C799F010E943A74ECE0F0E0E7
:1086E0000E943F74F0E00E942A790E94B26AEE81F3
:1086F000E030A9F0E0917405A3E0EA9FF001E758AB
:10870000FA4FDF01E09175050E94546E4C91552798
:108710000E943A744A93EFE0EA930E9413660E9423
:10872000097C27960895E091F603E07141F0E2E0BC
:10873000EA93B7DFE091F603EF7EE093F603089546
:108740000E944474AF3EE0E0BE0744F4A0910203EF
:10875000B0910303AF33E1E0BE070CF037C00E94D5
:108760004974ED81EA93ED81EA930E941366A0912A
:108770004E05B0914F05549734F4A0915005B09137
:10878000510513970CF010C00E94B171A3E0B0E046
:108790000E945479E758FA4FA0915005B0915105C5
:1087A000EA0FFB1FA981A083E091FA03ACE0EA9FE6
:1087B000F0010E9444740E94C06B0E9456740E9493
:1087C000B1713196E0934E05F0934F0522960895CE
:1087D000E881EA93E091FD03EA93B2DF21960895E0
:1087E0001A9310E00E945B74E03031F00E945B74D9
:1087F000EA93EEDF1F5FF6CF188150C41A930A93F5
:1088000000E010E00E945E74E03021F00832E0E009
:108810001E070CF007C00E945E74EA93D9DF0F5F59
:108820001F4FF0CF1981088163C01A930A9300E0AB
:1088300010E0F801AB81BC810E94657421F0EA81EF
:108840000E946A740CF009C0F801AB81BC810E94DF
:108850006F74BEDF0F5F1F4FECCF1981088103C318
:108860000E94047C0E944474EFEEF0E0EA1BFB0BD4
:1088700031978F010E9474740E943A740E94976A23
:108880000E940B7C35C00E94047CAC810E947C74E9
:108890000E2F11270E9474740E943A740E94976AE6
:1088A0000E940B7CE0C2EA81FB81E0934E05F093CD
:1088B0004F05E881F981E0935005F0935105AA81B5
:1088C000BB81ECE0F0E00E947C790E945674A881A4
:1088D000B981E4E1F0E00E947C7906C0EA81FB8185
:1088E0000E945674E881F981E0930203F093030338
:1088F000249608950E948474143120F41A936CDC39
:108900001F5FFACF0E948B6A0E948B6A0E94AD6A39
:10891000EFE3F1E00E94B26A10E0153048F4A5E1FF
:108920001A9FF001E352FB4FA0E0A0831F5FF5CF39
:1089300010E0143148F4ABE01A9FF001EF5FFB4FF9
:10894000A0E0A0831F5FF5CFE091F603EF7EE093F8
:10895000F603A1C20E948474143100F5ACE01A9FA2
:10896000F001BF01E85FFC4FDF010E94207A0F0198
:10897000DF01EB81FC81AE17BF075CF0E981FA8172
:10898000E015F10534F0FB01E15FFC4FE081E030E0
:1089900009F402C01A9320DC1F5FDECF0E948B6AAD
:1089A000ED81FE81FA93EA930E94AD6AA985BA85AA
:1089B0000E948C740E94B26A55C2A2970E94027CE7
:1089C000E9A50E94AC708F01D8011A96EC91E030B5
:1089D00009F404C2D8011A96EC91E9A3E07849F0B1
:1089E0000E94BC72EBA10E94CB73FA93EA930E949F
:1089F0002D67E9A1E07449F00E94BC72EBA10E94CE
:108A0000D273FA93EA930E942D670E94BC720E946F
:108A10003867E8A3E091FA03EB8FE091FB03EA8F5C
:108A20000E94416DD80111962D913C91D801139669
:108A30004D915C91D80115960E942774EEA3FFA377
:108A4000D80116960E942774ECA3FDA3D8011796AF
:108A5000EC91EC8FE091FB03A0E10E94536AEAA342
:108A6000FBA30E9491740E94FB730E94FB73ECA114
:108A7000EA930E940664D8011896EC91EC8FE030DE
:108A800011F4E8E0EC8F0E9491740E9496745A935E
:108A90004A930E949D740E94A1740E94A8740E942F
:108AA000AB740E9491743A932A930E94AB74EEA126
:108AB000FFA10E94B2745A934A930E9496740E9436
:108AC000AB74A8A5A130B1F43A932A93FA01319678
:108AD0000E94A874FA013196FA93EA930E949D7459
:108AE000F90131960E94B774F9013196FA93EA932D
:108AF0000E94AB74A8A5A230F1F40E94A174319732
:108B00000E94A874EAA5FBA5E40FF51F3197FA931C
:108B1000EA930E949D74EEA1FFA1E20FF31F31972B
:108B20000E94B774EAA5FBA5E20FF31F3197FA93F1
:108B3000EA930E94AB74E8A5E03011F40C94BF46B0
:108B4000D8011896EC91EC8FE091FA03ACE00E940A
:108B5000BC740E94A779ED8FA8A1EA1710F40C94B9
:108B6000F845E1E0E093FB03E03021F0ECA1FDA14A
:108B7000B5970CF402C00E94C274AAA1BBA1ECA1DB
:108B8000FDA1EA1BFB0BDF010E94926FEAA3FBA38E
:108B9000ABA1AA231AF4E0E0EAA3EBA3A8A10E94E8
:108BA0007C74AEA1BFA1F0E00E94CA74EE8FA8A5AC
:108BB000A13021F40E94CD740E94D074A8A5A230E7
:108BC00031F40E94CD740E94B2740E94DC74E0E023
:108BD000E9A30E94E274AE0FBF1FEC91E03039F0C0
:108BE0000E94E2740E946F740E94E774F2CFC7C0C3
:108BF000E1E0E093FB03E03031F0ECA1FDA1E734CC
:108C0000A0E0FA070CF402C00E94C274E8A1EF8F42
:108C1000EAA1FBA1EE0FFF1FACA1BDA1AE1BBF0BD4
:108C2000E3E0F0E00E94A779EAA3FBA3ABA1AA23AB
:108C300022F4E1E0F0E0EAA3FBA3EF8DE150EF8F37
:108C4000EF8DF0E0DE011696AE0FBF1FAC91A032A3
:108C500019F0AF8DA13008F404C0EF8DE150EF8F13
:108C6000EFCFAF8D0E947C74AE2FEEA1FFA10E94CA
:108C7000D16E1CF3EF8DE03011F4ED8DEF8FAF8DE1
:108C8000ECE00E94BC740E94CA74EE8FA8A5A130CB
:108C900021F40E94CD740E94D074A8A5A23031F4B2
:108CA0000E94CD740E94B2740E94DC74E0E0E9A3DB
:108CB0000E94E2740E94657421F0EF8DA9A1AE17A5
:108CC00008F007C00E94E2740E946F740E94E7746B
:108CD000EFCFAF8DE8A1EA1BAE2FED8DEA1768F05C
:108CE000AF8DE8A1EA1BACE0EA9FF001A091FA0386
:108CF0000E94BC740E94CA7401C0E0E0EE8FA8A577
:108D0000A13079F40E94CD74E20FF31F31960E94D6
:108D10003F74AFE00E94536A0E94EF7431960E9444
:108D2000E86CA8A5A23069F40E94CD74E20FF31F8D
:108D30000E943F74AFE00E94536A0E94EF740E9449
:108D4000E86C0E94E274AE0FBF1FAC91A03219F420
:108D5000E9A1EF5FE9A30E94E2740E94657439F013
:108D6000AF8DE9A1EA1BAE2FED8DEA1708F407C01D
:108D70000E94E2740E946F740E94E774ECCFD801E5
:108D80001B96EC91E03021F10E94416D0E9491749C
:108D9000A5DDF801A385A43690F4EFE0E093FD0390
:108DA000F801A385AA3020F0A385AA9367D806C04E
:108DB000D8011B96EC91E05DEA930ADD09C0ECE076
:108DC000E093FD03E2E5EA9303DDEDE4EA9300DDE1
:108DD000EB8DE093FA03EA8DE093FB030E94097C9C
:108DE000AA9608951A9310E0E89427F8143170F4C5
:108DF0000E94286DE03011F00E942F6D1F5FA89532
:108E0000E12FE37011F40E94EB16F0CFEFE0E09356
:108E1000FD030E94EB163FC01A9310E01431F8F4E2
:108E20000E94346DB1F0A85FBC4F0E94207ADF0130
:108E3000EB81FC81EA17FB0764F4F001E85FFC4F6B
:108E4000DF010E94207ADF01E981FA81AE17BF07B6
:108E50000CF002C00E942F6D1F5FA895DFCFEFE0DE
:108E6000E093FD031881259608951A9310E01431BC
:108E700090F40E94346D31F0FD01E25FFC4FE0811F
:108E8000E17009F406C01A93E091F603E170EA93E9
:108E900094DD1F5FECCF199108952C970E94027CFE
:108EA000AD89BE890E94926F0E94F574EB8BFC8B9A
:108EB000ED89FE890E94FA740E94FF74EB89FC8997
:108EC000E017F107D4F00E942E752E2F33270E9451
:108ED0004D750E9454750E945B750E9463750E94D7
:108EE0004D75F8010E94FA74FA93EA930E945B753B
:108EF0000E946D750F5F1F4FE1CF46C02C970E94F7
:108F0000027CAD89BE89E4E0F0E00E94A7790E946E
:108F1000F574EB8BFC8BED89FE89EE0FFF1F0E9431
:108F2000FA740E94FF74EB89FC89E017F10764F181
:108F30000E942E75AE2FED89FE890E948F729F01CF
:108F40000E944D750E945475E98DFA8DEE0FFF1F3A
:108F5000AD8DBE8D0E9478750E946375ED89FE8986
:108F6000EE0FFF1FA98DBA8DAE1BBF0BBA93AA934C
:108F7000F8010E94FA74FA93EA930E945B750E94CA
:108F80006D750F5F1F4FCFCF0E94097C6B960895C0
:108F90000E947D7599F0E0E0E093D10810E000E0D8
:108FA0000E94756F0E94837549F00E94756F0E9440
:108FB00088750E94756F0E948B75F2CF0991199187
:108FC00008951A930A930091670BAA81A53411F4AE
:108FD000E0E062C0AA81A23539F4A091CD07A130AA
:108FE00019F40E94917509F405C00E94A31DE0E0E8
:108FF000E093CD07AA81AB3411F0A33599F4E02FAB
:10900000E470E43011F414E001C013E0E02FE270EA
:10901000E23009F41C5FE02FE170E13009F41F5FDA
:10902000E12F3AC0AA81A13511F0A13799F4E02FC0
:10903000E470E43011F417E001C016E0E02FE270B4
:10904000E23009F41C5FE02FE170E13009F41F5FAA
:10905000E12F22C0AA81A33441F413E0E02FE17094
:10906000E13009F41F5FE12F17C0AA81A73741F44F
:1090700017E0E02FE170E13009F41F5FE12F0CC031
:10908000AA81A03441F415E0E02FE170E13009F449
:109090001F5FE12F01C0EFEF19810881239608952A
:1090A00024970E94027CA091D808A53411F00C945A
:1090B0002549E0E0E093CD070E947070E0E0E09386
:1090C000F50AE0916B0BE030B1F5E091A707A091B4
:1090D000A807EA1739F00E949775E25BF84FE08124
:1090E000E13009F028C0E7E7EA930E94F25B0E94B2
:1090F0009775EF5AF84F0E9426700E94DA6B0E9413
:109100004C5C0E949775E15BF84FDF010E94207A6A
:109110000E94DA6B0E944C5C0E949775EE5AF84FE1
:109120000E949D75E2E0E093CD070E949775E25B97
:10913000F84FA2E0A083E091CD07E03011F00C944D
:1091400018490E94917511F40C9402490E94981DCF
:10915000E1E0E093CD07A091670BA87081F00E9439
:10916000A275E8EEF3E00E94A779DF010E94F87B88
:1091700014F4E1E301C0E0E3EA930E94F25BE091C2
:10918000B90B0E949E720E940D6C0E944C5CA091D3
:10919000670BA47091F00E94A275E0E1F7E20E94D3
:1091A000D979AF01A091670BA07111F041505040E7
:1091B0005A934A93E4E0F0E00FC00E94A2750E9427
:1091C000BF71AF01A091670BA07111F041505040E9
:1091D0005A934A93E3E0F0E0FA93EA930E944C5CDE
:1091E000A091670BA07229F00E94A775E4E0F0E05F
:1091F00004C00E94A775E3E0F0E0FA93EA930E94AE
:109200004C5C16C018E0A091670BA47009F01F5FBA
:10921000A091670BA87009F01F5FA091670BA07267
:1092200009F01F5F0E948B6A0E94086C0E944C5CD0
:10923000A091670BE1E0EA23E13029F4E091F50A1F
:10924000EA930E94F25B0E94AE75A091D808A737FE
:1092500029F4E2E0E093CD07E03009F479C00E9400
:109260007070E2E50E9477700E94B4750E944971A7
:109270001E2F0E946471AF01E1E0EA930E94795BC6
:109280000E2FE091A707A091A807EA1739F00E94D6
:109290009775E25BF84FE081E23009F056C00E941A
:1092A0009775E15BF84FDF010E94207A4E175F0748
:1092B00011F00C949E490E949775ED5AF84F00806A
:1092C00011800E946D6C0E94F873EA17FB0771F120
:1092D0000E949775ED5AF84FDF010E94B9750E9400
:1092E0009775ED5AF84FDF010E94207AE450F54F50
:1092F0000E94C3750E94C7750E94CB750E94086CBE
:109300000E94CE75E5EBFBE10E944571003029F02B
:109310005A934A930E94215C04C0E0E3EA930E94BE
:10932000F25B0E94D4750E948E5D08C0003031F05F
:109330000E94D87518F40A930E941D71E091A80745
:10934000EA930E943C32E093A807E0E0E093CD0767
:10935000A091D808A33421F40E944732E03009F4E8
:109360000EC00E947070E2E50E9477700E94B47592
:109370000E94C9710E948B6A12D30E944B1EA09159
:10938000D808A03421F40E944732E03009F423C009
:109390000E944971E887F987E2E0EA930E94795BCD
:1093A0001E2F0E94DF750E9486190E9441720E9442
:1093B000E575E258F84F10830E944172E558F84F66
:1093C000A7E0A0830E9443700E947070E2E50E94B3
:1093D00077700E94B475A091D808AB3439F0A335EA
:1093E00029F0A13519F0A13709F075C00E94291E96
:1093F000339724F00E944732E03009F466C00E949F
:1094000070700E94EC75E9EDF8E00E945F71A09128
:10941000670BE2E0EA23E23029F4E4E0EA930E94F9
:10942000795B02C0E1E0F0E0E887F987A091D80815
:10943000A13511F0A13721F40E9464711E2F02C0E2
:1094400010917D0BA091670BE4E0EA23E43011F466
:10945000E4E001C0E3E0EA930E94795BAF01A091F0
:10946000D808A33511F0A13731F4E885F9850E94B9
:109470001679E887F9870E94D87520F0A0916B0BC8
:10948000A130C9F41A935A934A93EB85FC85FA9359
:10949000EA930E946A1EEE83FF83AF81AA235AF4E7
:1094A0000E947070E6E6EA930E94F25B0E94F075FB
:1094B000AF81AA23BAF31A935A934A93EB85FC859A
:1094C0000E9422710E94AE7506C00E94C9710E945E
:1094D0008B6A0E946A1E0E94097C2A9608950E9447
:1094E000F675E89422F80E942772E2E7EA930E9458
:1094F000F25BE091D307EA930E94F25BEFE0EA931C
:109500000E94F25BA091D007AA3219F41A9315D3E6
:109510001AC0A091D3070E94756FE450F54FE08107
:10952000EA1721F4E091D307E03349F40E942F6B4E
:10953000A450B54FE091D307EC931A93FED222FCCE
:1095400002C00E948E5D76C20E94F675E091D3073C
:10955000E053AE2F0E94756FE35FF44FE081EA178E
:1095600041F51A93EAD2A091CE07A23019F40E94D5
:10957000FE7509F402C00E940476A091CE07A330C4
:1095800019F40E94FE7509F402C00E940476E0E01E
:10959000E093CE07E093080C0E94756FE35FF44FF1
:1095A000BF01E081EF5FAE2FEAE00E94D679DB01D8
:1095B000EC9340C20E94047C25FCF0C10E94FE7521
:1095C00011F40C94204C0E940C76E658F84F9F0141
:1095D000D9011196EC91E43071F50E9412760E9447
:1095E00015760E941C76F901A481A03021F4A28195
:1095F000B381109709F007C0E8EBFBE10E944571C9
:109600000E94D47515C00E94CB750E9423760E94DB
:10961000CE75EBEBFBE10E9445710E9427760E941C
:109620002D76F901A681B781BA93AA930E94215C95
:109630000E94337638C2E730C9F40E9412760E9445
:1096400015760E941C76EEEBFBE10E9445710E94AC
:1096500027760E94CE75E1ECFBE10E9445710E94E5
:1096600023760E94215C0E9433761DC2E93099F472
:109670000E9412760E9415760E941C76E4ECFBE1B3
:109680000E944571D901EC910E949E720E94CE7594
:109690000E94337608C2E63029F5EAE2EA930E9496
:1096A000745DE7ECFBE10E944571D901EC910E94E9
:1096B0003A76E091650B0E943A76EBE4EA930E94D9
:1096C000F25B0E9423760E94215CE4E5EA930E940B
:1096D000F25B0E9427760E94215C0E948E5D0E94B0
:1096E0000476E1C1E530E1F4D90116960E94B9751E
:1096F000D901EC91EA930E94F25B0E94C7750E9427
:10970000CB750E9423760E94CE75E5EBFBE10E94AB
:1097100045710E9427760E94215C0E943376C3C166
:10972000E83049F50E9412760E9415760E941C7658
:10973000EAECFBE10E944571F901A481AA930E9421
:10974000261A0E94626E309719F00E94626E04C061
:10975000D90114960E942774FA93EA930E94215C1F
:109760000E94D4750E948E5DD9011196E0E0EC93C1
:109770000E94047698C1E13011F00C94004CA09145
:10978000B007A53029F4E091650BE65F1E2F01C0FC
:1097900011E0E12FE05D0E943E760E94756FE35F6D
:1097A000F44F0E949D750E94C7750E94CB750E9460
:1097B00023760E94CE75EDECFBE10E9445710E947C
:1097C00027760E942D76D9011596EC910E949E7203
:1097D0000E94215CA091B007A53069F4EAE3EA9306
:1097E0000E94F25BF901A085AA930E94261A0E94AA
:1097F0005D6E0E9442760E94A7730E94467653C116
:10980000E330F1F4D90116960E94207AF0960E9476
:109810003E76D90116960E94207AE35FF44F0E94AB
:109820009D750E94C775E0EDFBE10E9445710E94A5
:1098300027760E94215C0E94A7730E94467633C15E
:109840000E94917561F0A091CE07A03041F4A091E3
:109850006A0BA13021F40E946D6CE13009F427C03D
:10986000A0911D0BA03059F0E0911F0BF091200B3F
:10987000FA93EA93E8EEF3E00E94D371C1F4E1E3D6
:109880000E943E76E0910E0B0E943A760E94C775C8
:109890000E946D6CEA930BD1E093CE070E94A773F0
:1098A000E093060CF093070CE0E0E0931D0BA09111
:1098B000CE07A03059F0E091060CF091070CFA9316
:1098C000EA93E4E6F0E00E94D37109F025C0A0918C
:1098D000CE07A23019F40E94FE7509F402C00E945E
:1098E0000476A091CE07A33019F40E94FE7509F406
:1098F00010C0A091080CA33030F00E940476E0E084
:10990000E093080C06C00E940C76E558F84FA8E0DA
:10991000A083E0E0E093CE07A0911E0BA130F1F50B
:10992000E091CE0BA091CD0BEA1799F1EAE20E94EB
:109930003E76E0910C0B0E943A760E94C775E0914A
:10994000CE0BEA930E94BE1F0E94CB75E091BE0B26
:109950000E949E720E94CE75E3EDFBE10E9445716C
:109960000E94356FFA93EA930E942D760E948A72C4
:109970000E9451760E948E5DE091CE0BEA930E9488
:10998000401EE091CE0BEA930E94131EE093CE0B93
:1099900005C0E0E0E0931E0B689420F884C00E94AC
:1099A0004732E030F1F00E944172E458F84FAA814A
:1099B000BB81A083B1830E944172E058F84FA88117
:1099C000B981A083B1830E944172E258F84FAC8103
:1099D000A0830E944172E558F84FA4E0A0830E9442
:1099E000437025960895E091DA0AEA930E94F25BAB
:1099F000E091DB0AEA930E94F25B0895F4DF0E9493
:109A000054760E945476E881F9810E945176B2C35F
:109A10001A930E94505B1E2F103021F0E12FE1506D
:109A2000E093D80AE0DFE091D80AEF5F0E949E72CF
:109A30000E94CE75199108950E94047C31E00E9425
:109A40005E7628F00E945371AC91A43308F02AC0CE
:109A500030E00E945371EC91E270E6951E2F0E9457
:109A60005371EC91E1700E2FA091F20A1A1729F4AC
:109A7000E1E0EA27E093F20A31E0A091F30A0A1745
:109A800029F0E1E0EA27E093F30A31E0E091F30AFC
:109A9000EE0FE05DA091F20AEA0FEA930E94F25BFA
:109AA0000E941872E32F0E940B7C249608951A934B
:109AB00010E00E949175E9F10E94981DE6EDFBE12E
:109AC0000E944571E091B90B0E949E720E94CE7572
:109AD000E9EDFBE10E9445710E94A7750E94CE75D9
:109AE0000E94A275A031E7E2BE074CF4ECEDFBE169
:109AF0000E944571E091BA0BF091BB0B13C0EFEDE2
:109B0000FBE10E944571E9810E94676E0E94A27587
:109B1000EA0FFB1F0E94F96EE091BA0BF091BB0BAC
:109B2000E051F742FA93EA930E94215C0E94D475B7
:109B300011E00E946276E12F1CC324970E94027CF0
:109B40000E9462760E94145BE13010F40C947C5009
:109B5000E091DA0AEB3441F4E091DB0AE33219F4E4
:109B60000E94505B1E2FC5C2E435A9F4E091DB0AC8
:109B7000E33221F40E94505BEE83FF83E091DB0A25
:109B8000EF3441F40E94505B1E2F1A930E94E27240
:109B90000E948619AEC2E23411F00C94144FE09189
:109BA000DB0AE13251F4AA85AF3F29F40E94C97162
:109BB0000E948B6AF4DE0E944B1EE091DB0AE134C6
:109BC000E1F40E94505B1E2F113071F4A091CE077A
:109BD000A13019F40E94917509F402C00E94A31DDE
:109BE000E0E0E0931D0B09C0E1E0E0931D0B0E9453
:109BF000FA61E0931F0BF093200BE091DB0AE53450
:109C0000A9F4E2EEFBE10E9445710E94801DF397EA
:109C10003CF00E94505B0E94F96E0E94697601C080
:109C2000E0E3EA930E94F25B0E94D475E091DB0AC4
:109C3000E634D9F40E94757619F40E94505BAF01A6
:109C4000E885F9850E943A6F0E2F003420F0A0912C
:109C50006B0BA13051F40E9481760E946A1EAA8586
:109C6000AF3F19F40E9481769ADEE091DB0AE2357B
:109C700011F00C94D14E0E94757619F40E94505B3D
:109C8000AF0130E0A0916B0BA03021F40E946D6C0D
:109C9000E13009F027C00E944D32E03011F10E94FE
:109CA0000F71E15BF84FA885B985A083B1830E944D
:109CB0000F71ED5AF84FDF01EA850E944B700E9448
:109CC0000F71EF5AF84F10830E940F71EE5AF84F40
:109CD00040830E940F71E25BF84FA1E0A0830E94D5
:109CE00015715DC00E944732E23010F40C94CF4EE3
:109CF0000E94DF750E943F1F3E2F3F3F29F00E94C8
:109D00000E6FA417B5070CF416C00E948A72E41BEC
:109D1000F50B0E941C6F0E94D47039F4E0E0E093D0
:109D2000BE0B3A930E94CC1F03C03A930E94C51FFA
:109D3000689420F803C0E0E0E887E9870E94417258
:109D4000E658F84FDF01EA85F0E0E450F54FE08196
:109D5000EC930E9441720E94E575E058F84FDF01D4
:109D6000EA850E944B700E944172E258F84F1083BE
:109D70000E944172E558F84FA5E0A0830E9443700D
:109D8000E885F985309759F00E94DF75FA010E9445
:109D900016790E9422710E9481760E94F41D6894B7
:109DA00022F8E091DB0AE335F1F50E94505BE88789
:109DB000F9870E940C76DF01E558F84FE081E23028
:109DC00081F4FD01E058F84F008011800E946D6C15
:109DD0000E94F873EA17FB0721F4A091CE07A23086
:109DE00009F01FC00E940C76E458F84FDF010E9472
:109DF000207ADF01E885F985EA17FB0779F40E94EC
:109E00000C76DF01EE57F84FE081EA93FD01E6584A
:109E1000F84FE081EA930E94502603C0E7E0E09308
:109E20001A06689422F865C1E43411F00C947D4F51
:109E3000E091DB0AE33559F4E5EEFBE10E94457160
:109E40000E940B580E943A76E1E0E093D108E0913D
:109E5000DB0AE03511F00C947C4F0E948576E030EF
:109E600011F40C947C4F20E00E94897640F00E940F
:109E70005371AC91A23219F00E948D7609F43CC066
:109E8000E22FE03061F40E945371AC91A33211F4DF
:109E900021E004C00E9491760E94E6572AC0E1307A
:109EA00051F40E945371AC91A43211F422E001C02C
:109EB00020E010E01EC0E23011F0E330D1F40E9447
:109EC00091760E94D261EF3F99F0E12FE295E07F19
:109ED000EF930E9491760E94D261AF91EA0F1E2FFC
:109EE0002F5F243021F41A930E94E65720E001C02E
:109EF00020E00E941872B8CFFCC0E63511F00C9437
:109F0000F34FE091DB0AE33429F50E94505B1E2FEA
:109F1000E0912306E030C9F0E8EEFBE10E944571D4
:109F2000E0912306E0580E949E720E942D76E091F7
:109F30002606F0912706FA93EA930E942D76E09187
:109F40002806F09129060E945176113019F0E0E0C0
:109F5000E0932306E091DB0AE33511F00C94F24F15
:109F6000E0E0EA930E94891CE0E0E093210B0E946C
:109F7000505BE093350B0E949576A1F50E94505BF3
:109F8000E093380B0E94957669F50E94505B1E2F76
:109F9000103019F0E1E0E093320B0E94957611F554
:109FA0000E94505BE0933B0BF0933C0B0E94957634
:109FB000C9F40E94505BE093410B0E94957691F4A6
:109FC0000E949B761E2FE0E0EA931A930E9450268F
:109FD000E03041F4E8EEFBE10E9445710E94086C1C
:109FE0000E94CE7586C0E33411F00C947950E09154
:109FF000DB0AE534B9F4E2EEFBE10E9445710E9410
:10A00000801DF3974CF00E94505BE05FF84D0E947A
:10A01000F96E0E94697601C0E0E3EA930E94F25B68
:10A020000E94D475E091DB0AE634A1F441E050E0EF
:10A030000E94505B0E2F0E94957619F40E94505B8F
:10A04000AF011A930E94136BE05FF84D0E94B77442
:10A050000E946A1EE091DB0AE33571F50E94505BB5
:10A060003197E887F9870E94957619F40E94505B32
:10A07000AF01E8850E94586EE83131F4E091210B80
:10A08000EA930E94371918C0E885EA93FA01E0586C
:10A09000FF4FEA930E945026E03041F4EBEEFBE1E3
:10A0A0000E9445715A934A930E94CE75E885EA93BF
:10A0B000EFEFEA930E945026E091DB0AE134C9F405
:10A0C000EEEEFBE10E9445710E94505B3197E887FC
:10A0D000F987E885EA930E94261A0E948725E030D6
:10A0E00011F0E1E301C0E0E3EA930E94F25B0E9419
:10A0F000D4750E94D15A26CD0E94097C2B960895D2
:10A10000A091F00AA03529F4E091F10AEA930E94A7
:10A110004B1AA091F00AA33529F4E091F10AEA93D1
:10A120000E947D1AA091F00AAB3429F4E091F10A63
:10A13000EA930E94BB1AA091F00AA63529F4E09197
:10A14000F10AEA930E94E91AA091F00AA43511F4E9
:10A150000E9470190E94A07608951A9310E010349E
:10A1600040F40E94756FE35BF94FA981A0831F5FE4
:10A17000F6CF1881229608950E94027C0E94145BFB
:10A18000E13010F40C94F453E091F00AA091DA0A53
:10A19000EA1709F0B5DFE091DA0AE33259F5E09108
:10A1A000DB0AEC3441F4E0E0EA93D7DFE4E0E0934B
:10A1B000AF070E94A676E091DB0AE435D1F4E0E037
:10A1C000EA93CBDFE0910B0CE03029F0EF77A9E0C8
:10A1D000B0E00E94627AE0910C0CE03029F0EF7759
:10A1E000AAE0B0E00E94627A0E94A676E7E0E093DF
:10A1F000AF0704C0EB3411F00C944351E091DB0A3B
:10A20000E13221F4EBE4EA93A8DF3CC0E53211F43B
:10A2100077DF38C0E332D9F40E94AC7631F00E9487
:10A22000B7760E94871A0E94BD760E94C276E081AE
:10A23000EB3461F4E0E0E093C90BE093CA0B0E94B9
:10A24000C276A0E0A083EBE4E093F00A1BC0E13407
:10A25000C9F4EBE4E093F00AA091D80AA03890F496
:10A260000E94505B9F012093C90B0E94C87651F059
:10A270000E94505B9F010E94C87621F00E94505BB3
:10A28000E093CA0BAEC2E33511F00C948A51E09111
:10A29000DB0AE13221F4E3E5EA935FDF3AC0E3321F
:10A2A000D9F40E94AC7631F00E94B7760E945A1A17
:10A2B0000E94BD760E94C276E081E33561F4E091B0
:10A2C000D80AEA930E94711C0E94C276A0E0A08383
:10A2D000E3E5E093F00A1DC0EE34D9F4E3E5E09342
:10A2E000F00AA091D80AAA30A0F4EAE0EA930E940A
:10A2F000D25B10E01A3068F4ABE4BBE0EE27A10FAC
:10A30000BE1F0E94756FE452F54FE081EC931F5F12
:10A31000F1CF67C2E63511F00C94E051E091DB0A11
:10A32000E13221F4E6E5EA9318DF49C0E332D9F4DB
:10A330000E94AC7631F00E94B7760E94C91A0E9442
:10A34000BD760E94C276E081E63561F4E091D80ADC
:10A35000EA930E94FC1A0E94C276A0E0A083E6E580
:10A36000E093F00A2CC0E63531F40E94505B9F0167
:10A370002093C50B24C0E53471F40E94505B9F010B
:10A380002093C40B0E94C87629F00E94505B9F0165
:10A390002093C70B14C0E43591F440E050E00E94D4
:10A3A000505B9F01022E032A11F042E050E00E9410
:10A3B000C87619F00E94505BAF014093C60B11C2E2
:10A3C000E43511F00C94A352E091DB0AE33231F44E
:10A3D0000E94505B3197E093D80AB4C0E03511F089
:10A3E0000C94A25210E00E94897650F00E945371A2
:10A3F000AC91AD3329F00E948D7611F01E3008F03B
:10A4000005C00E94756F0E94CE76EDCF0E94756FD9
:10A410000E94D776EDE30E94DC7611F00C94A252F4
:10A42000E4E5E093F00A10E00E94CB6E70960E9483
:10A430002F7AEF3FA0E0FA0711F40C94A2520E9489
:10A44000E1760E94CB6EFA93EA930E941B67E0309C
:10A4500011F00C94A0520E94CB6E0E94357341F40F
:10A460000E949B76E0930B0CE0E8E0930C0C68C034
:10A47000E238A0E0FA0729F40E949B76E0930C0CE6
:10A480005FC0E138A0E0FA0739F40E94505BA8E011
:10A49000B0E00E94627A54C0309721F0E130A0E031
:10A4A000FA0751F40E94C26EFF93EF930E94505B33
:10A4B000AF91BF91EC9344C0E230A0E0FA0759F4A9
:10A4C0000E94C26EFF93EF930E94505BAF91BF91C9
:10A4D000ED93FC9335C0E330A0E0FA0751F40E94FD
:10A4E000C26EFF93EF930E942F5BAF91BF91EC93ED
:10A4F00027C0E430A0E0FA0719F50E94CB6E7296EF
:10A50000E491EA930E94D25B0E94C26EE093090C30
:10A51000F0930A0C00E00E94CB6E0E94DA6E84F485
:10A520000E94136BE452F54FE081A091090CB091A9
:10A530000A0CEC93A9E0BCE00E94B36C0F5FEBCF78
:10A540001F5F72CF4EC1E03511F00C94F153E091D2
:10A55000DB0AE332D1F40E94AC7631F00E94B77688
:10A560000E94261A0E94BD760E94C276E081E035E4
:10A5700061F4E091D80AEA930E94891C0E94C27695
:10A58000A0E0A083E0E5E093F00AE091DB0AE3328B
:10A5900021F0A091D80AA03408F023C1E0E5E093AF
:10A5A000F00AE091DB0AE13221F4E0E5EA93D5DD3F
:10A5B00018C1E134C1F40E94505B1E2F00E00C3042
:10A5C00088F40E94E7723B96E491E11749F40E94F7
:10A5D000E7723A96E491A091320BEA2BE093320BAA
:10A5E0000F5FEDCFFEC0E63559F5E0E0E093D90A04
:10A5F000A5E3BBE00E94E676FF93EF930E94505BD9
:10A60000AF91BF91EC93EBE2EA930E94E15AE03004
:10A6100059F0A8E3BBE00E94E676FF93EF930E9417
:10A62000505BAF91BF91EC930E94EA76A091D90A5A
:10A63000A33018F40E94C87609F401C0D9CFD1C064
:10A64000ED34D1F4E0E0E093D90AA1E4BBE00E944C
:10A65000E676FF93EF930E94505BAF91BF91EC932E
:10A660000E94EA76A091D90AA33018F40E94C87615
:10A6700009F401C0EACFB5C0E43411F00C947F5363
:10A68000E0E0E093D90A0E94505B9F01E2E0EA9388
:10A690000E94EE5AAF01E3E70E94DC7679F40E9453
:10A6A000F076EA0FFB1FBF01D901E4E6F0E00E945B
:10A6B0007C79E40FF51FDB01ED93FC93E9E40E9444
:10A6C000DC7689F40E94F076EA0FFB1F2083318349
:10A6D000A2E3BBE00E94E6760F010E94F576EC91C2
:10A6E000E160D001EC930E94EA76A091D90AA330F0
:10A6F00018F40E94C87609F401C0C5CF72C0EE34C8
:10A70000A9F4EAE0EA930E94D25B10E01A3068F400
:10A71000A2E2BBE0EE27A10FBE1F0E94756FE452BC
:10A72000F54FE081EC931F5FF1CF5BC0E33449F458
:10A730000E9485760E94505BE0932D0BF0932E0BC8
:10A7400050C0E33589F40E94505B9F01002402163B
:10A75000030624F42B30E0E03E070CF004C0F901BE
:10A760003197E0932F0B3DC0E53529F40E94505BF3
:10A77000E093310B36C0EF3491F40E94505B1E2FF2
:10A78000ECE2EA930E94E15AE12FE295E07FEF9339
:10A790000E94505BAF91EA0FE093300B22C0E0358E
:10A7A00001F5E0E0E093D90AA4E4BBE0E091D90A26
:10A7B0000E94B36FEA0FFB1FFF93EF93E2E0EA936F
:10A7C0000E94955BAF91BF91ED93FC930E94EA7656
:10A7D000A091D90AA23018F40E94C87609F401C0E9
:10A7E000E3CF0E94D15ACACCE0E0E093DB090E949B
:10A7F000097C269608950E94047C0E94145BE13037
:10A8000010F40C948E56E091DA0AE332A9F4E09148
:10A81000DB0AE03519F4E1EFFBE109C0E83419F493
:10A82000E2E1FCE104C0E33531F4EDE2FCE1FA934E
:10A83000EA930E94025C6FC2E43511F00C94C55497
:10A84000E091DB0AE43229F4E5E2F0E00E94FB76D5
:10A850009BC0E33211F4DCD897C0E03511F00C94C2
:10A86000C454C1D8A091D80AA53210F00C94C45495
:10A870000E94FF760E944571EDE3EA930E94F25B2D
:10A880000E94FF760E94357339F40E946D6C0E941D
:10A890009E720E94215C78C0E238A0E0FA0739F489
:10A8A0000E94B86E0E949E720E94215C6DC0E138C9
:10A8B000A0E0FA0739F40E9499720E949E720E94E9
:10A8C000215C62C0309721F0E130A0E0FA0751F43A
:10A8D0000E94FF763E960E942F7A0E9426700E9468
:10A8E000077752C0E230A0E0FA0759F40E94FF76E1
:10A8F0003E960E942F7ADF010E9413720E94215C13
:10A9000043C0E330A0E0FA0751F40E94FF763E9680
:10A910000E942F7AE081EA930E94305C35C0E430D7
:10A92000A0E0FA0789F50E94FF763E960E942F7AF2
:10A93000E093090CF0930A0C10E00E94FF767296E7
:10A940000E942F7A0E942F6BAE17BF0794F40E94CB
:10A95000756FE452F54F0F01A091090CB0910A0CEC
:10A96000EC91D001EC93A9E0BCE00E94B36C1F5FB6
:10A97000E4CF0E94FF7672960E942F7A0E94D776CB
:10A980000E94E1760E94905CC6C1E33571F5E091CA
:10A99000D80AEA930E945A1AE091DB0AE43221F4C1
:10A9A0000E94896D2BD820C0E33211F431D81CC02D
:10A9B000EE34D1F418D810E01A3068F40E94756FA4
:10A9C000E452F54F0F01ABE4BBE00E94AB73D00142
:10A9D000EC931F5FF1CFE0E0E093E60A0E94E1769E
:10A9E0000E94905C0E94D47596C1E63511F00C94DB
:10A9F0003655E091D80AEA930E94C91AE091DB0A21
:10AA0000E43229F40E94836C0E94FE4C2EC0E33293
:10AA100019F40E94084D29C0E53459F40E94F34C02
:10AA2000E091C40B0E949E720E940B77E091C70BCD
:10AA300019C0E63529F40E94F34CE091C50B12C011
:10AA4000E43599F40E94F34CE091C60BE03011F02C
:10AA5000E1E301C0E0E3EA930E94F25B0E94117718
:10AA6000E091C60BF0E00E94517655C1E03511F03F
:10AA70000C945C56E091D80AEA930E94261AE09161
:10AA8000DB0AE43229F4E0E4F0E00E94FB7613C133
:10AA9000E33219F40E94084D0EC1E13411F00C9418
:10AAA00091550E94F34C12E0A091320BECEDEA2399
:10AAB0003E2F00E00C3068F40E94E7723A96E49171
:10AAC000E31729F40E94E7723B96149102C00F5FCE
:10AAD000F1CF0E94086C0E94CE75E091300BE030FF
:10AAE00089F0E8E4FCE10E9445710E94E06B0E945D
:10AAF0009E720E940B77E091300BEF700E949E7265
:10AB00000E94CE75E091310BE03051F0EBE4FCE1B6
:10AB10000E944571E091310B0E949E720E94CE7599
:10AB2000CAC0E43439F50E941577A091D90AA33040
:10AB300000F5E091D90AE03011F00E9411770E94EF
:10AB4000F576EC91E17041F40E94F0760E94067077
:10AB50000E944276E3E707C00E94F0760E940670EA
:10AB60000E940777E9E4EA930E94F25B0E94EA768A
:10AB7000DCCF9DC0ED34C9F40E941577A091D90AAD
:10AB8000A33090F4E091D90AE03011F00E941177DF
:10AB9000A1E4BBE00E941B77EC910E949E720E9490
:10ABA000215C0E94EA76EACF82C0E63531F50E9448
:10ABB0001577A091D90AA330F8F4E091D90AE030D2
:10ABC00011F00E941177A5E3BBE00E941B77EC9186
:10ABD0000E949E720E94215CEBE2EA930E94F25B6B
:10ABE000A8E3BBE00E941B77EC910E949E720E943A
:10ABF000215C0E94EA76DDCF5AC0EE34D1F40E9487
:10AC0000F34C10E01A3068F40E94756FE452F54F6F
:10AC10000F01A2E2BBE00E94AB73D001EC931F5F77
:10AC2000F1CFE0E0E093E60A0E94E1760E94905CBA
:10AC30003EC0E33499F40E94F34C0E94E176E3E5D0
:10AC4000FCE1FA93EA930E94626E0E945E6C0E949D
:10AC500075720E94E1760E94905C29C0E03579F41B
:10AC60000E94F34C0E945D6E0E9442760E94117712
:10AC7000E091460BF091470B0E94427618C0E335F5
:10AC800031F40E94F34CE0912F0BEF5F0DC0EF34D5
:10AC900091F40E94F34C0E94E06B0E949E720E940D
:10ACA0000B77E091300BEF70F0E00E940777EBE359
:10ACB000EA930E94F25B2FC0EB3469F5E091D80A69
:10ACC000EA930E94871AE091DB0AE43229F4E0E873
:10ACD000F0E00E94FB761FC0E33219F40E94084D99
:10ACE0001AC0E134C1F40E94F34C0E943C720E94ED
:10ACF0009E720E940B770E943C720E949E720E947C
:10AD00000B77E091CA0B0E949E720E94215CE6E5DF
:10AD1000FCE10E9445710E94D15A6FCD0E9462767B
:10AD20000C94545A1A930E947070E8EDF8E00E9457
:10AD30005F710E9462760E941F77E181E43471F4B2
:10AD40000E941F7702800E946D6CE05DE01529F083
:10AD50000E941F77E281EA3209F401C057C00E94C5
:10AD600024770E941F77E1810E9428770E941F7735
:10AD7000E2810E9428770E9453711C910E941F77E4
:10AD800033960E945F71E12FE23131F40E942E77F9
:10AD9000E6E0EC93F1D93AC0E13131F40E942E772C
:10ADA000E2E1EC9328DD32C0EF30A9F40E942E7767
:10ADB000EEE0EC930E941C4DE13039F4A091CD07F8
:10ADC000A03019F00E94917509F402C00E94A31DE1
:10ADD0000E9434771BC0EE30C9F40E942E77EFE05A
:10ADE000EC930E941C4DE13089F4A091CD07A03076
:10ADF00019F00E94917509F402C00E94A31DE0E0C1
:10AE0000E093CD07EFEFEA930E949D4D54C21A9351
:10AE10000E942772E4EDF7E00E945F71EAE7EA938F
:10AE20000E94F25B0E94537111971C91E12FE23155
:10AE300031F4E6E0EA930E94F25B9ED937C0E1313B
:10AE400031F4E2E1EA930E94F25BD5DC2FC0EF30EF
:10AE500099F40E94C7750E941C4DE13039F4A0910D
:10AE6000CD07A03019F00E94917509F402C00E942C
:10AE7000A31D0E9434771AC0EE30C1F4EFE0EA93CC
:10AE80000E94F25B0E941C4DE13081F4A091CD073D
:10AE9000A03019F00E94917509F402C00E94A31D10
:10AEA000E0E0E093CD07EA930E949D4DA091D0078A
:10AEB000AA3211F00E948E5DFEC10E94A076089514
:10AEC000AC81A03310F0AA3308F006C00E943B7793
:10AED000E0530E9443770FC0AC81A13410F0A73437
:10AEE00008F006C00E943B77E7530E94437703C0F7
:10AEF000A881B981E0E0EC9325960895AA93EA939E
:10AF0000FA93EFB7EA931A930A931BB10CB1E0914D
:10AF1000430CF0E0EF5EF34F0083A091430CAF5F72
:10AF2000A093430CA23319F4E0E0E093430C0991A1
:10AF30001991E5C21A93E091440CA091430CEA17D1
:10AF4000D1F3F0E0EF5EF34F1081A091440CAF5FBE
:10AF5000A093440CA23319F4E0E0E093440CAAC19E
:10AF6000E091440CA091430CEA1709F074C3ABC103
:10AF70000A921A92FA926A937A938A939A93AA936C
:10AF8000BA93EA93FA93EFB7EA930E944C7749F0A9
:10AF9000A091D108A03021F00E947A0EE13009F48E
:10AFA00001C011C0E091AA0CF0E0EB5BF34FE0812F
:10AFB000ECB9A091AA0CAF5FA093AA0CA43619F427
:10AFC000E0E0E093AA0C0E941A6D18951A930E9473
:10AFD0004C7759F45D9B09C0A091D108A13021F4B0
:10AFE0000E947A0EE03009F013C01091A90C0E9463
:10AFF000756FEB5BF34FA981A0831F5F143609F4D3
:10B0000010E0E091AA0CE117E1F31093A90C02C043
:10B01000E981ECB9A0C20E944C7721F40E947A0E1B
:10B02000E13009F001C017C34EC10E94047C98DFD3
:10B03000E03011F40C9413597DDF1E2FA091100CF9
:10B04000A53618F0E0E0E093D2083091D208E09104
:10B05000D208E03011F00C947A58A0917C0BA1300A
:10B0600021F0A0917C0BA23031F4E12FEF77E09337
:10B07000D808EBE4CEC01A3521F4E1E0E093D20821
:10B08000CAC0123049F4E4E1E093D208E0E0E09372
:10B09000D308E093D508BFC0A0917C0BA33069F41E
:10B0A000173729F01A3310F4103308F402C0E7E020
:10B0B00001C0E0E0E093D40805C01A930E94E14784
:10B0C000E093D408A091D408AF3F99F01093D8082A
:10B0D000E1E0E093D3081093D508E091D408E03084
:10B0E00011F4E5E404C0EAE0E093D208E0E0E09384
:10B0F000D70891C0E13069F4103039F4E2E0E09310
:10B10000D208E0E0E093D70803C0E0E0E093D20883
:10B1100082C0E23059F41093D4081093D508E0E0CF
:10B12000E093D308E3E0E093D20875C0E330F1F494
:10B130000E9452770E945877EA0F0E946277A9F422
:10B14000E091D508E03071F4E4E0E093D208E091BA
:10B15000D3080E94096E0E946B770E945277A0E08C
:10B16000A08303C0E0E0E093D20855C0E43049F486
:10B170001D3019F4EAE5E093D708E0E0E093D20847
:10B180004AC0EA3079F40E9452770E945877EA2741
:10B190000E94627731F4E0E0E093D208E5E4E093C6
:10B1A000D70839C0E431B9F40E9452771083E12FF7
:10B1B000A091D508EA27E093D508E091D308EF5F86
:10B1C000E093D308E0E0E0930F0C133019F4E5E1CD
:10B1D000E093D20820C0E53111F0E63159F41A931A
:10B1E000EFE0FCE0FA93EA93E2EDF8E0FA93EA93F9
:10B1F00067DE11C0E73179F4E0E0E093D20817315F
:10B2000031F4E0910F0CA091D508EA1709F003C0C2
:10B21000E3E4E093D708A091D2083A1719F0E0E0F0
:10B22000E093100C04CF40C1AA93BA93EA93FA9327
:10B23000EFB7EA931A930A9310919B0000919C0038
:10B24000E12FEC71A9F4E091730DF091740DE555C7
:10B25000F34F0083A3E7BDE00E94B36CE83CA0E09D
:10B26000FA0731F4E0E0F0E0E093730DF093740D31
:10B2700009911991E991EFBFF991E991B991A991DA
:10B2800018951A930E9470770E947577D9F30E94DF
:10B290007077E555F34F1081A5E7BDE00E94B36CD0
:10B2A000E83CA0E0FA0731F4E0E0F0E0E093750D4F
:10B2B000F093760DE12F199108950E9470770E9406
:10B2C000757709F0C8C1E0E008950E94047CF5DFBD
:10B2D000E03021F0A0910E0CA03009F0E5C0D1DFE4
:10B2E0001E2FA0917F0DA53618F0E0E0E093790DB8
:10B2F0003091790DE091790DE03059F4113019F465
:10B30000E4E0E093790D1A3519F4EAE0E093790D61
:10B31000C3C0E430C1F4E0E0E093790D1A3229F0C3
:10B320000E946D6CE05DE11769F41093D0071093F3
:10B330007A0DE5E0E093790DE0E0E0930E0CE1E0BA
:10B34000E0937C0DA9C0E530A9F4E0E0E093790D2D
:10B350000E946D6CE05DE11761F00E947C770E94B5
:10B360008577E0917C0DEF5FE0937C0DE6E0E09364
:10B37000790D92C0E63091F4E0917C0D0E948577C2
:10B380000E947C77EF5FE0937C0DE0E0E0937D0D21
:10B39000133019F4E7E0E093790D7EC0E73011F047
:10B3A000E83059F41A93EDE7FDE0FA93EA93E9E700
:10B3B000FDE0FA93EA9384DD6FC0E93081F4E0E0C8
:10B3C000E093790D173131F4E0917D0DA0917A0D64
:10B3D000EA1709F003C0E4E5E0930E0C5DC0EA3023
:10B3E00041F4103011F4EBE001C0E0E0E093790D9E
:10B3F00053C0EB3071F4E0E0E0937C0D10937B0DD3
:10B4000010937A0DECE0E093790DE0E0E0930E0C00
:10B4100043C0EC30A1F5E0917C0DF0E0E852F74F2D
:10B4200010830E947C77EF5FE0937C0DE0917B0DB1
:10B43000E150E0937B0DA0917B0DA03021F4A09111
:10B440007A0DA03009F00EC0EDE0E093790DE091A7
:10B450007C0D0E94096E0E946B77E0917C0DF0E0FC
:10B460000E946B77A0917B0DA03021F4A0917A0D02
:10B47000A03009F403C0E0E0E093790D0DC0ED3099
:10B4800059F4E0E0E093790D1D3031F4EAE5E09302
:10B490000E0CEFEFE0930D0CE091790DE31719F02E
:10B4A000E0E0E0937F0D13CF0E940B7C249608957B
:10B4B000AA93EA93FA93EFB7EA93E091810EA091F1
:10B4C000800EEA1791F0E091CF07E03019F0E89490
:10B4D00026F80AC00E948A77F0E0E030A1E0FA077F
:10B4E00019F4E0E0E093810E03C0E89425F826F813
:10B4F000E0910D0CE03019F0E0E0E093790DE99176
:10B50000EFBFF991E991A99118951A93E091810EF5
:10B51000A091800EEA1721F4E0919B00E072C1F443
:10B52000E091800EF0E0E058F24FA981A0831091E5
:10B53000800E1F5F0E942F6BA030E1E0BE0709F470
:10B5400010E0E091810EE117E1F31093800E03C04B
:10B55000E981E0939C00188122960895E0E0E09351
:10B56000810EA091800EA13020F00E948A7768940D
:10B5700026F80895AA93BA93EA93EFB7EA93E09175
:10B580000D0CE03041F4E0E0E093810E0E946D6C20
:10B59000EF5FE093CF07E991EFBFE991B991A991EE
:10B5A00018950E94897618F00E948D7609F403C0E0
:10B5B0000E941872F6CF0E948D7611F40E941872C4
:10B5C00008950E945371AC91E881EA1729F40E9412
:10B5D00018723197E1E003C4E0E001C40E9498775B
:10B5E000EEE20E94DC76E1F420E030E0EC81D9016B
:10B5F000F0E0AE17BF07A4F4D8010E94D8728F0103
:10B600000E945E7618F00E949D7708F006C00E94A6
:10B61000A1770E0F1F1F0E9418722F5F3F4FE6CFBA
:10B62000F8010E940B7C5EC20E94897628F00E947D
:10B630001F77E181E03208F410C00E945371EC9151
:10B64000E093DA0A0E9418720E945371EC91E09321
:10B65000DB0A0E941872E1E008950C943D601A9391
:10B660000A9310E00E9453710C910B3311F00032D9
:10B6700008F412C0013310F0093308F007C0E02FBE
:10B680000E94D272E255FF4FE4911E2B0E94187265
:10B690000E9453710C91E9CFE12F099119910895FE
:10B6A0000E9498770E945371AC91AD3229F40E94A8
:10B6B00018722FEF3FEF02C021E030E00E945E766B
:10B6C00018F00E949D7708F00CC0D8010E94D87233
:10B6D0000F010E94A177E00DF11D8F010E941872E9
:10B6E000EDCFF901D8010E947C790E940B7C0C946B
:10B6F0007D600E94047C20E030E000E010E0EC81FE
:10B700000E946A7474F4D9010E94D8720F010E94D9
:10B71000A177E00DF11D9F010E9418720F5F1F4F6E
:10B72000EECFF9010E940B7CDDC10E94987720E0EA
:10B7300030E00E945E7618F00E949D7708F016C0F7
:10B74000AC81A13048F0D8010E94D8720F010E944C
:10B75000A177E00DF11D8F0131E0213018F0AC81AF
:10B76000A13008F403C0EC81E150EC830E945371D6
:10B77000AC91AE3211F422E031E0313011F40E948C
:10B7800018723130A9F2AC81A13040F0D8010E948A
:10B79000D8728F01EC81E150EC83F5CFF8010E9463
:10B7A0000B7CA0C11A9310E00E948576E030A1F0D6
:10B7B0000E94897658F00E945371AC91A23231F008
:10B7C0000E948D7619F0E9811E1708F005C00E94CD
:10B7D000756F0E94CE76ECCF0E94756F0E94D7766F
:10B7E0000C949760E8810E942877E881A091F40A80
:10B7F000EA0FE093F40AE881A091F50AEA27E093C2
:10B80000F50AEDC21A9310E00E94A477E491E030AB
:10B8100031F00E94A477E4910E94A977F5CFD1C0BE
:10B820001A9310E00E94756F0E94AE7741F00E945B
:10B83000756FE452F54F0E94C3751F5FF3CF0C94F0
:10B8400038600E94E176ECE5FCE1FA93EA93EC8142
:10B85000FD810E945E6C0E947572E2DF0C9498601C
:10B860001A93ECE3EA93BEDF11E0193080F40E94F2
:10B87000756FE255FF4FE491A981EA2319F0E12F9A
:10B88000E05D01C0E0E2EA93ADDF1F5FEECFEEE3E3
:10B89000EA93A8DF0C9497601A930E94E176E4E69D
:10B8A000FCE1FA93EA93EF81F8850E945E6C0E94B6
:10B8B000757210E00E94756FE452F54FE081E0323E
:10B8C00041F40E94756FE452F54FA0E3A0831F5F1F
:10B8D000F1CFA981BA81EAE0F0E0EA1B1E2F0E94B5
:10B8E000756F0E94AE7741F00E94756FE452F54F7C
:10B8F0000E94C3751F5FF3CFF4C00E947373ECE521
:10B90000FCE1FA93EA93EE85FF85688979890E94C4
:10B91000337A0E94757284DF0E94D4752E96089542
:10B920001A93E2E2EA935EDF10E00E945B74E0307B
:10B9300029F00E945B740E94A977F7CFE2E2EA93B4
:10B9400051DF3FC01A9310E00E945B74E03029F091
:10B950000E945B740E94A977F7CF33C01A930E94AC
:10B96000E176E9E6FCE1FA93EA93AD81BE81E4E693
:10B97000F0E00E94A7790E945E6CA985BA85E4E692
:10B98000F0E00E94D9790E945E6C88E00E945F69B5
:10B990002C9610E00E94756F0E94AE7791F00E9485
:10B9A000756FE452F54FE081E03211F4E0E305C039
:10B9B0000E94756FE452F54FE081EA9313DF1F5F39
:10B9C000E9CF18812396089524971A93E0E0E9833C
:10B9D000EA83EB83EC83AD81BE810E942774E05340
:10B9E000F84F1081103310F01A3308F022C0A981EB
:10B9F000BA818B819C81EAE0F0E060E070E00E9417
:10BA00008179DF01CB01E12FE053FF2766277727FC
:10BA10000E940C79E983FA836B837C83AD81BE81BC
:10BA2000EC91EF5FEC930E942774E053F84F108184
:10BA3000D9CFE981FA816B817C8118810C94C56032
:10BA40000E949877AC81BD810E942774E053F84F23
:10BA50003081303310F03A3308F014C0D8010E941E
:10BA6000D872DF01E32FE0530E94C06B8F01AC81DD
:10BA7000BD81EC91EF5FEC930E942774E053F84F87
:10BA80003081E7CFF8010E940B7C0C941B621A9363
:10BA900010E0AB81BC810E942774E053F84FE08135
:10BAA000E03210F0EB3708F015C00E94A4770F01C8
:10BAB000AB81BC810E942774E053F84FE081D00134
:10BAC000EC93AB81BC81EC91EF5FEC931A3008F4FE
:10BAD0001F5FDFCFA981BA81EE27A10FBE1FEC93B4
:10BAE000E12F18812596089525FE06C00E94836CDB
:10BAF0000E94FC78A895F8CFE0E8FDE0E093F60A14
:10BB0000F093F70AE1E00E947770E093F40A0E9454
:10BB1000B3770E946D6C0E943A7661C11A930A93C2
:10BB2000E0910D0CE03011F00C940362E3E0EA9335
:10BB300059DEE091F40AE295EF70EA930E94E96120
:10BB40001E2FE091F40AEF70EA930E94E9610E2F34
:10BB50001A9348DE0A9346DEE7E1EA9343DEE0E823
:10BB6000FDE0A091F60AB091F70A0E94437AEA1B21
:10BB7000E093800E689425F80C940362EE81EA93BA
:10BB8000B3DFEC81FD810E9445710E94B777B5DE7D
:10BB9000C5DF0C94C560EB81EA93A6DFE981FA81E9
:10BBA0000E9445710E94B377B9DF0C947D60ED81EE
:10BBB000EA939ADFEB81FC810E944571EA81EA9366
:10BBC00011DEE981E03011F0EA930CDEE881E0302B
:10BBD00011F00E94B377A2DF0C941B620E94027CDA
:10BBE00010E0E0E7FCE1A885B985EA17FB0719F446
:10BBF00044E150E002C048EC50E0EA85E093D00810
:10BC0000E89431F8EA93E985FA85FA93EA93EA85AC
:10BC1000EA93EA85EA93E0E0EA93C9DF0E94FA61D9
:10BC20009F010E94F4160E9491740E9406620E2FDA
:10BC300031FC02C0003009F001C0F3CF31FE04C076
:10BC4000E89431F8E1E004C01F5F1230B0F2E0E0A8
:10BC50000E94097C2B9608950E947D7511F40C9426
:10BC60000362E0E0E093D108E2E0EA93AFD910E0AC
:10BC700003E00E94756F0E94837561F00E94756FEA
:10BC80000E9488750E94756FE852F64FE0810E277A
:10BC90001F5FEFCFE3E0EA9399D9E02FE295EF70D1
:10BCA0000E94BE77E02FEF700E94BE77E7E1EA9333
:10BCB0008DD90C9403620E947D7511F40C9403627B
:10BCC0000E94B86EE03021F0E091DA09EA3209F41E
:10BCD00005C00E94B86EE05DE093DA09E0E0E09311
:10BCE000D108EAE5EA9372D9E0E0EA936FD910E06F
:10BCF0000E94756F0E94837511F01F5FF9CF1F5F5F
:10BD0000012F0A9363D910E00E94756F0E9483751A
:10BD100049F00E94756F0E9488750E94756F0E949D
:10BD20008B75F2CFE02FE195EA9350D9EDE0EA93DD
:10BD30004DD90C9403621A930A93F894E0E0E093CF
:10BD4000CF07E091810EE093800E7894E091D809BE
:10BD5000E03011F40C940362EAE5EA93D6DBE0E00C
:10BD6000EA93D3DB10E00E94756F0E94837511F097
:10BD70001F5FF9CF1F5F012F0A93C7DB10E00E94FE
:10BD8000756F0E94837561F00E94756FE852F64FDF
:10BD9000E081EA93BADB0E94756F0E948B75EFCF4A
:10BDA000E02FE195EA93B1DBEDE0EA93AEDB0C9492
:10BDB0000362E881EA9398DEEAE5EA9313DDE09115
:10BDC000D808EA930FDD0E945371EC91E03031F016
:10BDD0000E94917607DD0E941872F5CF9FDE2196B2
:10BDE00008951A930E947070E091D307EA93FADCE9
:10BDF000E4E4EA93F7DCE091D107EA93F3DC14E0A2
:10BE00000E94756FE053F84FE081E43040F00E94EB
:10BE1000756FE053F84F0E94C3751F5FF1CFE0E0EC
:10BE2000EA93E0DC48DF24C11A930E941558E091A0
:10BE3000D708E03011F40C94915FA091D708AA358F
:10BE400041F4A091D308A33020F0E091D908E43464
:10BE500009F04BC00E94B86EE03021F0E091DA08A2
:10BE6000EA32C1F40E946D6CE05DA091DA08EA1735
:10BE700021F0E091DA08EA3221F40E9492561BDFA9
:10BE800008C0EBEDF8E00E945F71E091DA080E94D3
:10BE9000C4772BC00E94B86EE05DA091DA08EA1763
:10BEA00021F50E946D6C1E2FE091DB08ED3421F42A
:10BEB000E091DC08E33209F007C0EDEDF8E00E9404
:10BEC0005F71EEDB1E2F6DDB0E946D6CE11729F0B8
:10BED000E12FE05D0E94C47708C00E946D6CE05DB8
:10BEE000E093DA080E949256E6DEA091D708A534C6
:10BEF00049F4A0917C0BA33019F40E94F72A02C0E8
:10BF00000E945048A091D708A33411F40E94B02A8F
:10BF1000A091D708AB3411F40E94AB2AE0E0E09383
:10BF2000D708A0917C0BA33011F40E94F72AE0E01F
:10BF30009FC0CBD9A0910E0CA43529F4A0E025FC1C
:10BF4000A1E0A03009F03CC0E091D207E03589F4CF
:10BF5000E091D307EA93E6E0EA930E949740A0912C
:10BF6000D307A03828F0E091D307F0E00E942274B4
:10BF700024C0E03729F4E0E0F0E00E9422741DC004
:10BF8000EA3519F40E94075718C0EA3711F429DF7F
:10BF900014C0E23519F40E946F4A0FC0E23719F459
:10BFA0000E94A44A0AC00E94092FE091D107A091E3
:10BFB000D008EA1711F4689431F8E0E0E0930E0C31
:10BFC000A0910E0CAA3531F40E949256B4DEE0E046
:10BFD000E0930E0C52C0A0E025FCA1E0A13049F492
:10BFE000A0E026FCA1E0A03021F4A091CF07A03072
:10BFF00009F001C0B3DAE091CF07E03019F0E15069
:10C00000E093CF070895E0917F0DEF5FE0937F0D00
:10C01000E091100CEF5FE093100CE0910D0CE0301C
:10C0200019F0E150E0930D0C0895A0917C0BA13024
:10C0300021F0A0917C0BA23029F4E3E0E093900082
:10C04000E8E3E9B90895E0E00E94296A0E944A6A9B
:10C0500008951A9314EAE4EA0E94CB7741F40E940F
:10C06000D077183011F0103111F4E0E001C0E2E0B7
:10C0700019910895E4E9E0937400E0E008951A93BB
:10C08000E981E1600E94D57731F40E94D0771034C5
:10C0900011F4E0E04CC04AC01A93E9810E94D577C0
:10C0A00031F40E94D077183111F4E0E040C03EC076
:10C0B0001A93E9810E94D57731F40E94D077183223
:10C0C00011F4E0E034C032C01A93E981E03011F09D
:10C0D000E4EC01C0E4E80E94CB7769F40E94D077D9
:10C0E000E0917300AA81BB81EC93103511F01835F3
:10C0F00011F4E0E001C0E1E01881249608951A935C
:10C10000E981E093740010E0E0917400E07811F4AC
:10C11000163908F005C08BE18A95F1F71F5FF4CF5F
:10C12000E0917400E07811F0E0E001C0E1E01881F6
:10C13000229608950E94047C3D810C8120E089DFD5
:10C14000E030F9F4EE810E94A96DD9F43A93B0DFA2
:10C15000E030B9F40E94D977A1F47BDFE03089F4B4
:10C16000EE810E94416A69F4EDB7FEB7FA93EA9353
:10C170001F930E94466A1F91E03019F47BDFE12F84
:10C1800002C061DFDCCF0E940B7C279608950E94DD
:10C19000047C30E00E811D815CDFE03099F4EF819A
:10C1A0000E94A96D79F40E94D97761F41A9380DF17
:10C1B000E03041F4EC81EA937BDFE03019F45ADFA0
:10C1C000E0E002C040DFE8CF0E940B7C2896089593
:10C1D00022970E94027C50E02B853A85A89539DF92
:10C1E000E03011F00C944661EE850E94A96D11F0CB
:10C1F0000C9446612A935CDFE03011F00C944661A8
:10C200003A9356DFE03011F00C94466122DFE030C3
:10C21000E9F5EE850E94416AC9F5E0E0EE83EF831F
:10C22000EC85FD8531970E94187449F4EDB7FEB78F
:10C23000FA93EA931F930E94466A1F9109C0EDB7D3
:10C24000FEB7FA93EA931F93E1E0EA933DDF1F9173
:10C250000E2FEE81FF81A885B985EA0FFB1F1083A1
:10C260000E94F075003039F4EC85FD85AE81BF8108
:10C27000AE17BF0708F001C0D3CFEC85FD850E9443
:10C28000187421F4F7DEE0E00C940F66DCDEA7CF33
:10C2900068970E94027C20E0E0E0EC8FED8F31E0B7
:10C2A000A895E9A1FAA1662777270E94D97AEA879B
:10C2B000FB876C877D87EE8D0E94DE770E94416E42
:10C2C0000E94466EAA85BB858C859D850E94AF7BAA
:10C2D000EA8BFB8B6C8B7D8B0E94337AFE0172960E
:10C2E000FA93EA930E94F369EE8BFF8B688F798F44
:10C2F0000E94E4770E94A07AAF010E94E477AE8D9D
:10C30000BB27882799270E943A7A0E94F777DE0197
:10C310005A960E94A07AED93FC930AA119A199DE86
:10C32000E030D1F5EDA10E94A96DB1F50E94D97759
:10C3300099F51A93BDDEE03079F5303051F14F5F59
:10C340005F4FEC8DFD8D3196EC8FFD8FAC8DBD8DEB
:10C350001197EBA1FCA1EA17FB0711F430E018C01C
:10C36000EC8DFD8D3197AF8DB8A10E946F74A0DE6A
:10C37000EE8DDA01F0E0EA17FB0751F47BDEEA8D7F
:10C38000FB8DA9A1BAA1EA0FFB1FE9A3FAA389CFEC
:10C39000D4CF70DEE0E002C056DEC1CF0E94097C3F
:10C3A000A6960895A881A03310F0AA3308F004C01F
:10C3B000E881E0530C947967A881A13410F0A73488
:10C3C00008F004C0E881E7530C947967EFEF0C9410
:10C3D0007967A881AA3020F4E881E05D0C94796740
:10C3E000A881AA3020F0E881E95C0C947967E8E53F
:10C3F0000C9479671A930A93F8940091FA0A1091B1
:10C40000FB0A7894F8010991199108951A930A93F7
:10C41000F1DF8F01EA81FB81AC81BD81EA0FFB1F57
:10C42000E01BF10BDF010E94F87B14F4E0E001C097
:10C43000E1E01981088126960895EAE9F7E0FA9388
:10C44000EA93EAEBEA930E94836CE4E0EA93E6E283
:10C45000EA93EEE0EA930E942C66E2E3F8E0FA93B6
:10C46000EA93EAEAEA930E94FC77E8E0EA93E0E2E2
:10C47000EA93E1E0EA930E942C66E2E3F9E0FA93A2
:10C48000EA93E2EDEA930E94026DE2E0EA93E2E1D0
:10C49000EA93E1E0EA930E942C660E948B6A0E9474
:10C4A000026DEFEAF0E0FA93EA930E94FC77E1E094
:10C4B000EA930E9406640E94896DE4E3F0E00E9422
:10C4C000E86CE0E0E093FD03E4E7FCE10E941F6C10
:10C4D000EFE0E093FD0308950895EA81F0E0E5BB05
:10C4E000FBBBF7E1F09365001F98E6E1E093650080
:10C4F000F0936500E881F981E5BBFBBBFFE1F093B8
:10C500006500EEE1E0936500F09365001F9A2396C5
:10C510000895E2E2E5BBE0E0EBBBE7E1E093650014
:10C520001F98E6E1E0936500E7E1E0936500089578
:10C530001F9A0895EBE1E09365000E94A66DEFE17C
:10C54000E0936500E8ECF0E00E94EC6CE6E4EA932E
:10C55000E4EAF0E00E940178E7E4EA93E3E5F0E042
:10C560000E940178E8E4EA930E948B6A0E946D625F
:10C57000E9E4EA93E4E4F0E00E940178EAE4EA9373
:10C580000E94076B0E946D62EBE4EA93E7E6F0E03D
:10C590000E940178ECE4EA93E3E3F0E00E94017882
:10C5A000EDE4EA93E7E7F0E00E940178EEE4EA9335
:10C5B0000E94FC770E946D62EFE4EA93ECE4F0E005
:10C5C0000E940178E0E5EA93E6E4F0E00E94017859
:10C5D000E1E5EA93E4E4F0E00E940178E1E0EA9327
:10C5E0000E94636C0E946D620E949972E13029F48E
:10C5F000E6E1EA93E8E0F0E004C0E6E1EA93E8EC83
:10C60000F0E0FA93EA930E946D62E3E2EA93E5E9CF
:10C61000F0E00E940178E4E2EA93E5E9F0E00E94AC
:10C620000178E5E2EA93EFEFF0E00E940178E7E2BB
:10C63000EA930E940D6C0E946D62E8E2EA930E9408
:10C640000D6C0E946D62E9E2EA930E940D6C0E94FB
:10C650006D62EAE2EA930E940D6C0E946D62ECE268
:10C66000EA930E940D6C0E946D62EDE2EA930E94D3
:10C670000D6C0E946D62EAE3EA930E941A6C0E94BC
:10C680006D62EBE3EA930E941A6C0E946D62ECE328
:10C69000EA93E0EFF0E00E940178EDE3EA930E9474
:10C6A0008B6A0E946D620E94726C0E94FC78E5E3C6
:10C6B000EA93E8E3F0E00E940178E6E3EA93E8E732
:10C6C000F0E00E940178EEE3EA93E8E3F0E00E94F4
:10C6D0000178E0E4EA93EFE0F0E00E940178E1E421
:10C6E000EA93E0EFF0E00E940178E9E1EA93E9E4FF
:10C6F000F0E00E940178E3E9EA93EFE0F0E00E94C5
:10C7000001780E94806DE0E2EA93E0E4F0E00E94AC
:10C710000178EDE1EA930E94686C0E946D62EEE19F
:10C72000EA930E948B6A0E946D62EFE1EA930E9495
:10C73000076B0E946D62E4E4EA93EDE4F0E00E948E
:10C740000178E5E4EA93E1E1F0E00E9401780E94DB
:10C75000806DECE1EA930E94076B0E946D620E947B
:10C76000726C0E94FC78EBE1EA93E8E1F0E00E9451
:10C7700001780E940578EBE1EA93E0E1F0E00E94A5
:10C7800001780E940578E3E4EA93E0E8F0E00E9493
:10C7900001780E94A66DE0E9EA93EFE7F0E00E94DD
:10C7A0000178E6E2EA930E94076B0E946D620E94A4
:10C7B0000578E6E2EA93E4E2F0E00E940178E6E23E
:10C7C000EA93ECE2F0E00E9401780E940578E6E24C
:10C7D000EA930E94606A0E946D62E7E5EA930E9414
:10C7E0000D6C0E946D62E5E5EA930E948B6A0E94DF
:10C7F0006D62EEEFEA93EAE5F0E00E940178E7E58A
:10C80000EA930E948B6A0E946D6208950E940978E3
:10C81000EA0FFB1F0E942F7A8F01AE85AA2362F0D8
:10C82000AD85BE85A03FE0E0BE0734F4AB85BC8596
:10C83000AF33E1E0BE070CF07CC0E985FA85AD8539
:10C84000BE85AE0FBF1FA03FE0E0BE0744F0AD8540
:10C85000BE85EFEEF0E0EA1BFB0BE987FA87EF817C
:10C86000F885AB85BC85AE0FBF1FA034E1E0BE07E5
:10C8700044F0AB85BC85EFE3F1E0EA1BFB0BEF83F3
:10C88000F88749850E941078E3E0EA93EE85FF85FA
:10C890000E940178E4E0EA93EA85FB850E9417781C
:10C8A000E5E0EA93EA85FB85AE85BF850E94787551
:10C8B0000E946D620E941F78E7E0EA93EC85FD8597
:10C8C0000E940178E8E0EA93E885F9850E942678DD
:10C8D000E9E0EA93E885F985AC85BD850E94787525
:10C8E0000E946D6216DE05BB1BBB2EE13FE100E03E
:10C8F00010E0EF81F885E017F10764F050E045178C
:10C9000030F020936500309365005F5FF8CF0F5FD4
:10C910001F4FEFCF0DDEE4E0EA930E948B6A0E9486
:10C920002E780E94AD6A0E9433780E9439780E9466
:10C930003E7875C10E940978EA0FFB1F0E942F7A8A
:10C940008F01E985FA85AD85BE85EA17FB0711F0F1
:10C950000C9419650E94417814F40E9448780E9452
:10C960009972E13029F4E6E1EA93E8E2F0E004C0EC
:10C97000E6E1EA93E8EEF0E0FA93EA930E946D6252
:10C98000E4E0EA930E941A6C0E942E780E943E789E
:10C99000E8E0EA930E948B6A0E9439780E94AD6AAF
:10C9A0000E946D62E2E0EA93EC85FD850E94597871
:10C9B000E3E00E945C78E6E0EA93EE85FF850E9462
:10C9C0005978E7E00E946178A4DD05BB1BBB2EE12E
:10C9D0003FE10B851C85EF81F885E017F1073CF0FE
:10C9E00020936500309365000F5F1F4FF4CF0E94C6
:10C9F00098620E949972E13029F4E6E1EA93E8E056
:10CA0000F0E004C0E6E1EA93E8ECF0E0FA93EA93A0
:10CA10000E946D62E4E0EA930E948B6A0E942E7885
:10CA20000E94AD6A0E9433780E9439780E943E7855
:10CA3000F6C0EF81F885AB85BC85EA17FB0731F5B9
:10CA40000E94667814F40E9448780E941078E3E00F
:10CA50000E9461780E941F78E7E00E945C780E9443
:10CA6000896205BB1BBB2EE13FE10D851E85E98573
:10CA7000FA85E017F1073CF02093650030936500DC
:10CA80000F5F1F4FF4CF0E949862C9C00E946D785B
:10CA90000E947478FF93EF930E9478780E947478D4
:10CAA000AF91BF91EA17FB0710F40C94A1650E94A7
:10CAB000417834F520E030E00E947B78E217F307FC
:10CAC000F4F00E946D780E9482780E947B780E9428
:10CAD00087780E948F78E6E0EA93AC85BD85A21B3B
:10CAE000B30BFD010E945978E7E0EA93AC85BD8560
:10CAF0000E949B780E94A2782F5F3F4FDDCF20C01D
:10CB000020E030E00E947878E217F307CCF00E9432
:10CB10006D780E9482780E9478780E9487780E94BF
:10CB20008F78E6E0EA93F9010E942678E7E0EA933D
:10CB3000F9010E94A8780E94A2782F5F3F4FE2CFB0
:10CB40006EC00E946D780E947478FF93EF930E94EC
:10CB500078780E947478AF91BF91EA17FB0710F0C4
:10CB60000C940F660E94667864F520E030E00E9425
:10CB7000B178E217F30724F10E9478780E94827856
:10CB80000E94B1780E94B878AE85BF85A21BB30B16
:10CB9000FD010E945978E3E0EA93AE85BF850E94CB
:10CBA0009B78E6E0EA93FA010E942678E7E0EA93B0
:10CBB000FA010E94A8780E94A2782F5F3F4FD7CF3A
:10CBC0002EC020E030E00E946D78E217F3073CF1C0
:10CBD0000E9478780E9482780E946D780E94B878CE
:10CBE000F9010E941778E3E0EA93F901AE85BF8569
:10CBF000AE0FBF1FEFEFF0E0EA23FB230E940178A6
:10CC0000E6E0EA93FA010E942678E7E0EA93FA0167
:10CC10000E94A8780E94A2782F5F3F4FD4CF0E9435
:10CC2000097C2F9608951A930A93EB810E945A6FFC
:10CC3000EA5AF64F8F011A930A93E885EA930E9405
:10CC4000E272E2E0EA93E0E1EA93E985EA9304D054
:10CC5000198108812896089525970E94027CEB850A
:10CC6000A6E5B9E10E94B36FEA0FFB1F0E942F7A7D
:10CC7000EE83FF833091FA0310E0EC851E1710F06D
:10CC80000C94D566E989FA89E887F98700E0E09194
:10CC9000FB030E1710F00C94D266E885F985E98B3A
:10CCA000FA8BE6E0EA93EF85F8890E945978E7E08D
:10CCB000EA93EF85F889F0700E940178E0E0EA8756
:10CCC000ED85AA85AE1710F00C94CA66EA85F0E0EF
:10CCD0000E942C79DF010E942C6B0E947C79A8892C
:10CCE0000E948F72AF01E989FA8924913196E98B0C
:10CCF000FA8B203011F40C94C56627FF3DC0E2E0AA
:10CD0000EA93FA010E945978E3E0EA93FA01F0709D
:10CD10000E940178E2E2E5BBE0E0EBBBE7E1E093F3
:10CD200065001F98F6E1F0936500E0936500EE81E1
:10CD3000E5BBEF81EBBBEFE1FEE1E0936500F09333
:10CD40006500E093650031FF04C0F0936500E09357
:10CD5000650026FF10C0F0936500E093650031FF89
:10CD600006C0F0936500E09365004F5F5F4F220FB0
:10CD70004F5F5F4FEECF1F9A220F31FF02C04F5F10
:10CD80005F4F4F5F5F4F0C947966EA85EF5FEA87EC
:10CD90000C946066EE85FF853196EE87FF870F5F06
:10CDA0000C9447661F5F0C943D660E94097C639655
:10CDB0000895E0E0E0930403E8EFFFEFE093820ED4
:10CDC000F093830EE491EF3F39F0E091820EF09101
:10CDD000830E049000920403A0910403A33011F485
:10CDE0000E949A620E94846AE1E0E093FB03E09370
:10CDF000FA03E4E1E09300040895998188810096A4
:10CE000041F0BD81AC81FB81EA8105900D920197D3
:10CE1000E1F7FD81EC810C941F6AB981A88110961D
:10CE200031F0FC81EB816A8161931197E9F7EB8125
:10CE3000FC8125960895E991F991A991B9911D90E8
:10CE40000590011421F40020D1F7EE270895101861
:10CE5000E1F3E1E008F4E2500895E991F991A99134
:10CE6000B991CD0161916D936623E1F7FC010895BD
:10CE7000A991B991EE27FF276D91662311F03196A4
:10CE8000FBCF0895AA27BB27E991F99105900020CF
:10CE900011F01196FBCFFD0108957991E991F99177
:10CEA000A991B991CD01772351F07A9561916D9354
:10CEB0006623C9F7772319F07A956D93FBCFFC01B0
:10CEC00008956991E991F991A991B991CD016623EC
:10CED00051F06A9505900D920020C9F7662319F06C
:10CEE0006A950D92FBCFFC0108955D9BFECFE88112
:10CEF000ECB9219608951A930A93AC81BD810E94E2
:10CF0000207A3097C1F0AA81BB810E94207A8F01DC
:10CF1000309749F00230E0E01E0760F0F8013197E9
:10CF20008F01ED93FC93AC81BD810E94B36C31976E
:10CF3000AE81A08303C0EE81EA93D7DF1981088117
:10CF4000279608952C970E94027C10E0E88DF98DB9
:10CF50003196E88FF98F3197E4912E2FE03011F45C
:10CF60000C945B69E12FE03039F4253211F411E0C3
:10CF700002C00E94BF789EC1E130C1F4253219F48D
:10CF80000E94BF7896C112E0E0E0E98B00E02D320C
:10CF900011F401E08FC12B3219F4EBE2E98B8AC165
:10CFA000203219F4E0E2E98B85C102C0E23039F4A5
:10CFB00050E013E0203311F400687CC102C0E3307C
:10CFC000A1F4203310F02A3308F009C0A52FEAE0BD
:10CFD000EA9FF0015E2FE22FE0535E0F6BC140E04D
:10CFE0002E3211F414E066C110C0E430A1F42033F5
:10CFF00010F02A3308F009C0A42FEAE0EA9FF001FC
:10D000004E2FE22FE0534E0F55C12C3619F402601B
:10D0100015E050C104C0E53011F00C945A69E22FBC
:10D02000E33649F40E94CA78EE89FF89A481AA9365
:10D030000E94D0783EC1E33741F40E94CA780E9432
:10D04000DA780E9438671E2F0AC0E037A1F40E94E8
:10D05000CA780E94DA780E9442671E2F08600F7714
:10D06000403011F0411708F001C0142F40E0E0E01B
:10D07000E88B30E078C0E43611F0E93611F4046052
:10D0800002C0E537A1F4EAE0E88B01FF08C0E0E068
:10D09000FAEC6AE97BE30E94D46C1AE023C0E0E179
:10D0A000F7E260E070E00E94D46C15E01BC0E83548
:10D0B00011F4086004C0E83711F00C945969E0E1FC
:10D0C000E88B01FF08C0E0E0F0E060E070E10E9462
:10D0D000D46C18E007C0E0E0F0E160E070E00E948E
:10D0E000D46C14E0403011F00F7701C041E001FF33
:10D0F00008C00E94CA78AE89BF8914960E94247A1B
:10D1000015C002FF0AC00E94CA78AE89BF89149672
:10D110000E94207A0E943E7909C00E94CA78AE8996
:10D12000BF8914960E94207A66277727EC87FD87AF
:10D130006E877F8702FF16C0AF85AA2362F4EC8555
:10D14000FD856E857F850E941A79EC87FD876E8745
:10D150007F87EDE2E98BE989E03019F01F5F4F5FCF
:10D1600001C00B7F342F00FD14C0151710F43517C4
:10D1700008F00FC007FF08C002FF04C00B7F298919
:10D18000115001C020E301C020E20E94BF7851503D
:10D19000ECCF1417B0F4006102FF0AC00B7FE989DD
:10D1A000EA930E94D078503009F05150115041500C
:10D1B000E0E3EA930E94D078503009F0515041509A
:10D1C000E8CF312FE889E030B9F43030A1F003FF27
:10D1D00005C00E94F0753197E49105C0AE81BF8112
:10D1E000ED91AE83BF83EA930E94D078503009F06E
:10D1F00051503150EACF53C00E94E2780E94AC797E
:10D200002E2F2A3030F003FF02C0295C01C0295ABA
:10D2100001C0205D04FD23C0213350F40E94D96C6D
:10D22000A130E0E0BE07E0E08E07E0E09E0709F4F1
:10D230000BC0431740F4531710F000FF01C014C097
:10D2400020E207FF0CC020E3006102FF08C00B7F53
:10D25000E989EA930E94D078503009F051500E9439
:10D26000BF78503009F0515031500E94E2780E944E
:10D27000E779EC87FD876E877F87E8890E94D96C04
:10D28000FF27662777270E94AC790E94D46CE88537
:10D29000F9856A857B850E94F47B09F0ADCF00FF9C
:10D2A00008C0503031F05150E0E2EA930E94D0784B
:10D2B000F8CF10E04BCE0E94097C6A960895FF9249
:10D2C000F82E22971A930A93DE010E9408798D01A5
:10D2D000DE0116960E9408790E94207AEA83FB8379
:10D2E000DE0114960E9408790E9413721A930A9321
:10D2F000FE0136960E94896B25DEAA81BB81E0E0A3
:10D30000EC93198108812496FF900895A991B99111
:10D31000EE27002460E8E894162E169407941E2A3F
:10D320001EF0A015B10518F0A019B109E62BB7FB46
:10D33000AA0FBB1F669580F708957B816A81F981EA
:10D34000E88177FB770F67FD7160972F9E5781F01B
:10D3500078F0983190F4AA27BB27882708948795FE
:10D36000B795A7959A95D1F7EA23FB23682305C0C3
:10D37000E8947727EE27FF2766276F77769508F4DE
:10D38000606877F9A991B99189919991EA17FB079A
:10D390006807790797FB08950E94B7770E94EB789A
:10D3A00019F40E94F2781DC0E6F7A881B9818A813C
:10D3B0009B81E0E0F0E060E87FE30E94F77711C036
:10D3C0000E94B7770E94EB7819F40E94F27809C0A6
:10D3D000E6F30E94F278A0E0B0E080E89FE30E94CC
:10D3E000137B249608950E94F7780E94F47B39F409
:10D3F000A881B9810E94786E0E942A7A20C0AA81F1
:10D40000BB818C819D810E94FC7B34F40E94F77863
:10D410000E94337AC1DF05C00E94F7780E94337AF8
:10D42000CFDFA881B9810E942A7AA881B9810E94A0
:10D43000247AAA81BB818C819D810E94F7772696F0
:10D440000895E991F99130971AF4E095F0953196A5
:10D450000895E0937100E0E0E0937400E2B3E360CC
:10D46000E2BBE3EFE1BB85E38A95F1F7E0EFE1BBD7
:10D47000E4E4E0937400089588EC90E00197F1F7FC
:10D480000895EA930E943F60E0300895E0E0EA9357
:10D490000C94646080E991E00197F1F708951A9384
:10D4A0000A930C947A44EA9FF001F0E00895FA930D
:10D4B000EA93A02FB0E0ECE3F0E00E947C790895BD
:10D4C000ECE3F0E0FA93EA930895ECE0E093FC03D8
:10D4D000E0E0E093FD030895FA93EA93E4E0F0E0DE
:10D4E000FA93EA93E8E3F0E0FA93EA93FA93EA9383
:10D4F000E1E2EA93E6E7F9E1FA93EA93E0E0F0E0AB
:10D50000FA93EA930C944D41E0E0E093FC03EFE0E2
:10D51000E093FD030895E0E0F0E0FA93EA930895C4
:10D52000FA93EA93E8E2F0E0FA93EA930895E0E0F0
:10D53000EA930C940664E0914605F0914705FA934E
:10D54000EA930895E0914805F0914905FA93EA932A
:10D550000895FA93EA930C94CA40EFEEF0E0FA9340
:10D56000EA930895FA93EA93E2CFEAE4F1E0FA93BA
:10D57000EA93E6E4F0E0FA93EA93E2E3F0E0FA9368
:10D58000EA930895EBE4F0E0FA93EA93EECF0E9479
:10D590004D41E0EFF0E0FA93EA930895E2E3F0E022
:10D5A000FA93EA93E0EAF0E0FA93EA930895A5E0AB
:10D5B0001A9FF001E856FB4F0895319604900092AF
:10D5C000FC03A12FB0E0ECE3F0E00E947C793896F8
:10D5D0000895FA93EA93E2E3F0E008953296FA931D
:10D5E000EA9399CFE091FD03E093FC030C94F2469B
:10D5F000A5E03A9FF001E455FB4F08950E94047C9A
:10D600000C947A44E8E0F0E0FA93EA930895E4E0B9
:10D61000F0E0FA93EA930895FA93EA93E8E3F0E0EE
:10D62000FA93EA930895E02FF0E00895A091CF0BCC
:10D63000B091D00BBD01AEE0B0E00E945479E60F8E
:10D64000F71F0E942F7A30970895E091B505EE0FED
:10D65000EE0FEF5F3E2F0895E32FF0E00895A12F26
:10D66000B0E00895A091CF0BB091D00BBD01AEE01A
:10D67000B0E00E945479E60FF71F0895A9E03A9FA1
:10D68000F001E653FB4F0895319604900092FC039D
:10D69000E0E0E093FD030895A02FB0E0EAE3F0E0BE
:10D6A0000E947C793896FA93EA93D9CFEAE3F0E0C6
:10D6B0000E947C79E85AFF4F8CCFE0915A0BF0E042
:10D6C00008953091B607E1E0E093FA03E2E0E093D9
:10D6D000FB033A930E94261AE091300BE295EF701B
:10D6E000E093FC03E091300BEF70E093FD030895AD
:10D6F000FA93EA93E42FF0E0FA93EA930895E7E3CC
:10D70000F0E0FA93EA93E52FE450F0E0FA93EA931D
:10D710000895FA93EA93FFCEE22FF0E00895FA938A
:10D72000EA93E52FE450F0E0FA93EA93E32FE05810
:10D73000EA93F1CEE2E2FBE0FA93EA930C944D41D6
:10D74000E091590BA0EF0E9486792E2F08953A930D
:10D750000E94261AA091220BAD320895E091300B61
:10D76000E295EF70E093FC03E091300BEF700895C9
:10D770000E947C793396FA93EA93E52FF0E06FCF1D
:10D78000F0E0EA0FFB1F0895FA93EA93E22FE450CA
:10D79000F0E0C5CFACE04A9FF001E05FFC4FBF0175
:10D7A000E081E058DB01EC930895E3E0F0E0FA93C8
:10D7B000EA930895FA93EA93F8CFE550F0E00895DC
:10D7C000E091300BE295EF700895EA1BADEEB6E004
:10D7D000F0E00E942E790895E8ECF0E0FA93EA93E5
:10D7E000E4E6F0E0F6CEF0E0EE0FFF1FE257FB4F6D
:10D7F0000895ACE8B4E0F0E0EE0FFF1FEA0FFB1F66
:10D800000895FA93EA93E12FF0E0FA93EA930895EA
:10D81000E12FF0E0FA93EA930895E2E0F0E0FA9362
:10D82000EA930895E2E2FBE0FA93EA93EAE0EA93EE
:10D830000C941544E1E0F0E0FA93EA930895FA932A
:10D84000EA930C94FE430E942F7AFA93EA93089588
:10D85000E491F0E0FA93EA930895AFE3B1E00E9417
:10D86000A7798F0158CEBD01AAE0B0E00E9454799B
:10D87000E60FF71FFA93EA93EAE0EA930C94154453
:10D880001A930E94261AE091310BE0300895E1E0EE
:10D89000E093FB0340CE0E9453440C943044E0E2FA
:10D8A000EA930C94E843E12FADE4B6E0F0E0EE0F2C
:10D8B000FF1FAE0FBF1F0E94207A08950E943E797D
:10D8C0000E94337A0895E6E0F0E0FA93EA9308952F
:10D8D000E7E0F0E0FA93EA930895A9E0B0E00E944F
:10D8E0004E7A0895E4E1F0E0FA93EA930895F0E0C7
:10D8F000FA93EA930C94263FA1E00E942279A0912A
:10D900001906EA230895E5E0F0E0FA93EA93089512
:10D91000EFE0E0936100A8E0B0E00E944E7AE130D1
:10D920000895E0916205F09163050895E0915E0528
:10D93000F0915F050895AE0FBF1FE3E0F0E00E9495
:10D94000A7790895FA93EA931A930A930C947B1497
:10D95000FA93EA933A932A930C947B14A091580576
:10D96000B09159050895ED91FD913196FE93EE9396
:10D970000895A0916605B09167050895A091680586
:10D98000B09169050895E0934A05F0934B05089519
:10D99000A0E0B0E00E944A7A08950E94437AEA1B10
:10D9A000FB0B0E943E790895E887F9876A877B8799
:10D9B0000895A885B9858A859B850895DF01F001C2
:10D9C000EA1BFB0B0895A4E0B0E00E944A7A089598
:10D9D000FA93EA930C946E44FA93EA930C94FC78CD
:10D9E000A0915205B09153050895A9E01A9FF00146
:10D9F000E65AFA4F089537960E942F7ADF010E9467
:10DA0000207A0895E2E3F0E0FA93EA930895FA9316
:10DA1000EA930C94263F0A921A92FA926A937A93A6
:10DA20008A939A93AA93BA93EA93FA93EFB7EA93F5
:10DA30001A930895E991EFBFF991E991B991A991EC
:10DA40009991899179916991F99019900990089526
:10DA5000ACE01A9FF001EB5FFC4FE08108951A9350
:10DA6000E1E0EA930C94DD44ACE01A9FF001DF01A1
:10DA7000EB5FFC4FE081E0300895E2E0EA930C9424
:10DA8000DD44E1E0E093FA03E093FB030895E091C5
:10DA9000C107F091C2076091C3077091C4070E944B
:10DAA000337A08950E945A1AEBE4FBE0FA93EA9362
:10DAB0000895E12FEF5FF0E0FA93EA930C9453445A
:10DAC000ADE4B6E0F0E00E942E79AE0FBF1F0895DE
:10DAD0000E94247A0E94337A0895F0E0FA93EA9340
:10DAE0000C945344E091B30BF091B40B0895E09182
:10DAF000B50BF091B60B6091B70B7091B80B089510
:10DB0000EAE0F0E069CFE9E0F0E0FA93EA930C9400
:10DB10005344EAE0F0E0FA93EA9308951A93E0EAB6
:10DB2000EA93EA81F0E0E054F14FFA93EA930E941D
:10DB30009A601E2F0895E0EAEA93EA81F0E0E0544B
:10DB4000F14FFA93EA931A930C94C760E4E6F0E07D
:10DB500043CFEA930E944C60E0300895E0EAEA93F4
:10DB6000EBE5F0E0FA93EA93E0E0FFE0FA93EA9362
:10DB7000E6E5FBE00895FA93EA93E0E2EA930C9479
:10DB80004861E0EAEA93E981FA81E050FE4EFA93B7
:10DB9000EA930895EA81F0E0A8E2B0E00E947C797F
:10DBA0000895E0EAEA9339CEFA93EA930C94E86098
:10DBB000E0EAEA93E8E2F0E0FA93EA931A930A9330
:10DBC000E2E2FBE00895E2E2FBE0FA93EA930895D3
:10DBD000EA81F0E0ABE0B0E00E947C79E050F24FE7
:10DBE0008F01AA81AA300895E0EAEA93EBE0F0E021
:10DBF000FA93EA931A930A93EAE4FBE00895EA8120
:10DC0000F0E0EE0FFF1FE050F04F8F01AA81A03827
:10DC10000895E150F0E00895EA81F0E00E942E7945
:10DC2000E058F14F8F01AA81A5300895E4ECFBE0A4
:10DC3000FA93EA93E0E0EA93EACCE1EBFBE0FA93B3
:10DC4000EA93E0E0EA93DECC0E942E790E942A79E2
:10DC5000DF01EA85F0E0AE0FBF1FE8E0F0E00E94D0
:10DC60007C79E050FA4E8F01E0EAEA93CBCC1A932C
:10DC70000A93E1EBFBE098CFAE81BF81888599855F
:10DC80000895EE83FF83688779870895EE81FF8189
:10DC9000688579850895E093B50BF093B60B609392
:10DCA000B70B7093B80B0895F0E0AE0FBF1F089547
:10DCB000EA930E94261A0C947220E091440BF09192
:10DCC000450B0895E0912D0BF0912E0B0895F0E097
:10DCD000A4E6B0E00E947C790895E091BF07F0913E
:10DCE000C0070895E093BC0BF093BD0B0C94861D08
:10DCF000E0E0F0E060E070E00895E093C107F093A9
:10DD0000C2076093C3077093C4070895ADE4B6E0FB
:10DD1000F0E00E942E79EA0FFB1F0895E75FF94FAC
:10DD2000E081E1300895FA93EA93E091BA07E05D6B
:10DD3000EA930895EA930E94EE5DE13008950E940F
:10DD4000FD66A881AF5FEAE00E948679E05D0895F4
:10DD5000A881AF5FEAE00E94D679E05D0895FA936A
:10DD6000EA93E0E0EA930895FA93EA930C940D673E
:10DD7000AAE0B0E00E944E7A0895EA930E94E84338
:10DD800010E00895A6E11A9FF001E854FF4F3E9677
:10DD90000E942F7A0895A6E11A9FF001E854FF4FE0
:10DDA0000895B0E0EA17FB0708957496E491D9014D
:10DDB000EC93089572960E942F7AA02FB0E0AE17D0
:10DDC000BF070895E881F0E0A5E0B0E00E947C790B
:10DDD0000895E0EAEA9397CDEA930E947B1DFA93B7
:10DDE000EA93E9EBFBE00895FA93EA93EFEFEA9305
:10DDF0008ACDE093BA0BF093BB0B08950E94437A4F
:10DE0000EA1BFB0B0895A091BF0BB091C00B0895C6
:10DE1000E0E0E093CD0BE093CE0B0895A091C10B11
:10DE2000B091C20B0895E091C10BF091C20BAC818F
:10DE3000BD81EA0FFB1F0895E093C10BF093C20B65
:10DE40000895E0E0E093BE0B1A930C94CC1F1A9354
:10DE50000E94131E1E2F0895E093BF0BF093C00B7A
:10DE600008951A930E94BE1FD9CFE091BF0BF09185
:10DE7000C00B0895FA93EA930C94D419EA930E9484
:10DE8000BE1F0E94621FE0300895E881EA930E945D
:10DE9000131EE8830895EB81EA930E943A1EFA93D9
:10DEA000EA93EEEBFBE00895E0E0E093D80BE0931B
:10DEB000D70B0895F0E0EE0FFF1F0E942A79089516
:10DEC000ACE8B0E0F0E0EE0FFF1FEA0FFB1F0E948E
:10DED0002F7A0895A091AD07B091AE07EA2BFB2BE6
:10DEE000E093AD07F093AE070895E12FF0E00895B9
:10DEF000A9EDBBE0F0E0EE0FFF1F0895A3E4B6E04C
:10DF0000F0E0EE0FFF1FAE0FBF1F0895EC93EC8102
:10DF1000E150ACE0EA9FF0010895E05FFC4FBF01E3
:10DF2000E0810895E2E0F0E00E94A7790895E09191
:10DF300024066FCEE0932806F0932906F8CFE25E20
:10DF4000F94FA0E0A0830895A0915A05B0915B0518
:10DF50000895A2E3BBE0E091B1070895A5E3BBE01B
:10DF6000E091B107A1CEF0E0EE0FFF1F0895ADECF8
:10DF7000B6E0E52FF8CFAE0FBF1F0E94207ADF0179
:10DF80000895E25EF94FE081FBCBE15DF94FE0815E
:10DF9000EA930C94B220ED93FC93A7CFEE0FFF1FF2
:10DFA0000E942A7908951396ED91FD913197FE9381
:10DFB000EE9308950A930E94A420E0300895A88566
:10DFC000B985EC91C1DFF0E0EA17FB0708951396DD
:10DFD000E0E0F0E0ED93FC930895BD01A9E0B0E02E
:10DFE0000E9454790895EE81FF81A381B481089540
:10DFF000E0E0F0E0ED93FC930895EE81FF81A181D4
:10E00000AA930895E12FA3EEBBE0ADCFAE0FBF1FE3
:10E010000E94207A0895AE0FBF1F0D901C90E12F33
:10E020000895EC55FF4DE491E0300895A885B98539
:10E03000EC91EA93E3E0EA930C949740A885B985C4
:10E04000E0E0EC93E2E0E0931A060895E081F0E06E
:10E050000895AE81BF8117960E94207A3097089567
:10E06000ED91FD913197FE93EE930895E091A9070C
:10E07000A9E0EA9FF001E658F84FEA87FB87AA85F6
:10E08000BB8511960895E091A907EA930E943C325E
:10E09000E093A9070895F0E0ED93FC930895E12F34
:10E0A000A4E3B6E060CFABE3BBE01FCFEE0FFF1FF2
:10E0B000ADCFA5E3BBE0EE27A10FBE1FEC91089505
:10E0C000EA930E94EA20E0300895A8E3BBE0EE273F
:10E0D000A10FBE1FEC910895E081EA930C94E657DE
:10E0E000E8EDF9E0E093F60AF093F70A0895EA9371
:10E0F0000E94F25BE0E00895EA930E94F25B0C94C8
:10E100002C5EA5E3BBE0EE27A00FBE1FEC910895A7
:10E11000A8E3BBE0EE27A00FBE1FEC910895A2E399
:10E12000BBE0EE27A00FBE1FEC91E1700895ABE3BA
:10E13000BBE079CAAE81BF811596EC910895A1E448
:10E14000BBE0EE27A00FBE1FEC910895ACE0EA9F64
:10E15000F001E25FFC4F0895ACE0EA9FF001EB5F55
:10E16000FC4F0895ABE01A9FF001E852FA4F089572
:10E17000ABE01A9FF001EE52FA4F0895AFEFBFEFF8
:10E18000A083B1830895ABE00A9FF001EE52FA4FED
:10E190000895ABE00A9FF001E852FA4F0895FE019E
:10E1A0003596FA93EA930895E091C10BF091C20B72
:10E1B00030970895AFEFA0834FCAE091010CF09122
:10E1C000020CFA93EA930895FA93EA930E94066286
:10E1D000E03008950E94FA61E093010CF093020C84
:10E1E0000895FA93EA93E0E0F0E8FA93EA930C9446
:10E1F0004D13FA93EA93E091FD0BF0E00895FA9342
:10E20000EA930C944D13E091A907A9E0EA9FF0016D
:10E21000E658F84FFA93EA930E94252934CFE0910B
:10E22000A707A9E0EA9FF0010895E091A707EA9304
:10E230000E943C32E093A7070895E091BB05EA9362
:10E240000C945026FA93EA930C94CF4CEE89ABE0F1
:10E25000EA9FF0010895FA93EA93E5C9E091FD0B76
:10E26000EA930E94F6191E2F089537DDFA93EA9378
:10E270000895E093FD0BE0E0E093FE0BE1E3E09313
:10E28000FF0B0E94552A0C940726FA93EA930C94EC
:10E29000025CE9EDF8E0E093F80AF093F90AE3E0B4
:10E2A000EA930C94795BA091F80AB091F90A089569
:10E2B0000E94FA61E093D30BF093D40B0895E0939E
:10E2C000F80AF093F90A0895E3E0EA930C94795B75
:10E2D000E093BF07F093C0070895EF5CEA930C94B6
:10E2E000E843ABE3BBE0E091B1073DCEE7E0E0936C
:10E2F000AF07EA93E0E0EA930EC9EA930E94C83EB2
:10E300000E94AE401E2F0895EAE2EA93EAE6FAE19F
:10E3100026CD0E94A32BE1E0EA930C947A2BE05DDA
:10E32000EA930C94CB5DA0915C05B0915D05A0389B
:10E33000E0E0BE0708950E947A440C943810E0E0B3
:10E34000F0E0E093BD07F093BE07E2E0E093FB034B
:10E350000895E091000431CAE091BD07F091BE0735
:10E3600056CBE0914E05F0914F050895FA93EA934C
:10E370000C944543A091BD07B091BE070895E8EE07
:10E38000F3E00E94D9790895A0E024FCA1E0A03038
:10E390000895E0E0EA93BFC8E091CB07F091CC0785
:10E3A000FA93EA930895FA93EA930E940662E130A1
:10E3B00008950E94FA61E093CB07F093CC0708958B
:10E3C000E0E0E093D70B0895D5DFEA17FB07089547
:10E3D000E093AF07E0E0E093C80708950E94CB5DAB
:10E3E0000E940B2DE093BC0708950E94261A0C94FE
:10E3F0007A44E091B007EA93E0E0EA930E94C62CE9
:10E400000E94DF280E94AB40E03008950E94AE4099
:10E410001E2F1A930E943B2D103808951A93E091F5
:10E42000BB05EA9308950E94207AFA93EA9308952F
:10E43000A8EFBAE098CAE091D407E053E093BA0796
:10E440000895FA93EA93E0E3EA930C94CB5DE091AC
:10E45000D107EA930C94745DE091B007A091AF07E7
:10E46000EA170895E89423F8E0E0F0E031DF0A933A
:10E47000E1E0EA930C94C62CA091C90BE1E0EA23F9
:10E480000895E091A907A9E0EA9FF0010895ABE0A3
:10E490000A9FF001ED52FA4F0895A083ABE00A9F66
:10E4A000F0010895ABE00A9FF001EB52FA4FA1E0B2
:10E4B000A0830895FA93EA93E0EBFAE1FA93EA93E2
:10E4C000EA85ABE0EA9FF0010895FF2766277727EA
:10E4D0000E94337A84E00E945F6928960895AC8197
:10E4E000BD81EE27A00FBE1F089584E00E945F69E2
:10E4F00028960895EE27A30FBE1FEC91D001EC9350
:10E500000895ADEEB6E0A8C80E942E79EA0FFB1F71
:10E51000AF010895E091C10BF091C20B0895B0E0F6
:10E52000EA0FFB1F0895E32FA091B607EA0FEA93C5
:10E530000895A8E0B0E00E944E7A0895F0E0FA93C2
:10E54000EA9308950E941C400C94F63F0E941340E9
:10E550000C94F63F0E941C40E5EDFAE100CC40E04F
:10E5600050E0E02FE05DEA93E8EDFAE1DCCBFE015C
:10E570003896FA93EA930895FE013696FA93EA9351
:10E58000089510914E05009150050895FA93EA936D
:10E590000C945344E6DE31975ECE0E94AE403E2F8F
:10E5A0000C949343E053F0E00895FA93EA9373C90F
:10E5B000EAE0F0E00E947C790895DF01EE27A30FE6
:10E5C000BE1F0895EF81F885FA93EA930895ACE0B1
:10E5D0000A9FF001E450FC4F0895EA930E94C2366E
:10E5E000E1320895FA93EA93E2E0EA930E941A373F
:10E5F000E1320895E6E0F0E08CC80E945344A2E3C3
:10E60000BBE0EE27A10FBE1FEC91E1700895EE0F65
:10E61000FF1FEA0FFB1F08950E94800F0C948B6A66
:10E620000E945344E12FEF5FEA930E943E3FEAE3EA
:10E63000EA930E94E843F6C80E943E3F30C9EA933D
:10E640000E94433F2CC9E12FEF5FEA930E943E3FB7
:10E65000EAE3EA930C94E843DF013E96F4C8A6E1AE
:10E660000A9FF001E854FF4F089570960E942F7A98
:10E67000E038A0E0FA070895EAEBF5E0E093CF0B6D
:10E68000F093D00B08950E94C31BE0E0E093B9071C
:10E690000E9463170E94800FE1E0E093B2070895A3
:10E6A0000E947A440E940C120E94AE400E2F0D333D
:10E6B0000895EE81FF81FA93EA930895EAE2EA93DE
:10E6C000EDE7FBE1FA93EA93E091B60728CEE091FB
:10E6D000B607EA930E94AC170C94800FE093B6053E
:10E6E000F093B70508952A97FE01FA93EA930895E7
:10E6F000E6E9FBE1FA93EA93AE85BF8588899989BB
:10E70000E4E6F0E060E070E00E94D1790E94337AA4
:10E71000AA89BB898C899D89E4E6F0E060E070E01D
:10E720000E94EB790E94337A88E00E945F692C9600
:10E73000FE010895FA93EA930C94F043EFE9FBE1AC
:10E74000FA93EA93EE85FF85B9C8FE01F3CF0E94E4
:10E750008E5D0C94FA61EE27A10FBE1FEC91089517
:10E76000EA930E94AC3F1F5F0895E091B905ACEBBE
:10E77000B5E0F9CBAF5FEAE00E94D6790895E09169
:10E78000B805ACEBB5E0EFCBE981ACE0EA9FF00176
:10E79000E15FFC4F0895EF73A5E1EA9FF001E352BA
:10E7A000FB4F0895EF73ABE0EA9FF001EF5FFB4F83
:10E7B0000895AC81BD81EE27A30FBE1FAC91A030A0
:10E7C0000895ABE00A9FF001EF5FFB4F0895EA0F59
:10E7D000FB1F0F01AC81BD818DCEA5E10A9FF00129
:10E7E000E352FB4F0895EE81FF8101801280A2CC9D
:10E7F000D001F0E00895EAA5FBA5FA93EA93089505
:10E80000FA93EA93FE013A96FA93EA930E942D67EF
:10E8100030E0E02F0895E091B605F091B705089536
:10E82000A6EBB5E0ED91FD913296FE93EE9308953F
:10E83000AE81BF81EA17FB070895EC91F0E0E00D8F
:10E84000F11D0895E0935A05F0935B050895EC914E
:10E85000F0E00895E0935C05F0935D050895E0E035
:10E86000F0E0E0935805F09359050895EBDFE0E000
:10E87000F0E0F0CF1A930A933A932A930895FA930B
:10E88000EA93E091FB030895A0910003B091010386
:10E890000895E0910003F0910103FA93EA93E09167
:10E8A0000203F0910303FA93EA930895E0930003BF
:10E8B000F09301030895A981BA814DCFF801AA818F
:10E8C000BB81EA0FFB1FE4910895AE0FBF1FAC910F
:10E8D000A0300895D801F0E0AE17BF070895AE0F3D
:10E8E000BF1FEC91EA930895A091FB03E4E1EA9F36
:10E8F000F0012E2F3327CDCFECE0EA9FF001A0915D
:10E90000FA03EA9FF00108951A93E1E0E093FB0314
:10E91000E093FA0310E00895EF81F885EA1BFB0B02
:10E9200008953A932A935A934A930895EAA5FBA52A
:10E93000E20FF31FFA93EA930895ECA1EA930C9483
:10E940009A643A932A93EEA1FFA1E40FF51F08956C
:10E95000FA93EA93EBCFEAA5FBA5E40FF51FFA9330
:10E96000EA93EBCFE20FF31FFA93EA930895FA9339
:10E97000EA935A934A930895EA9FF001AEA1BFA18A
:10E98000F0E00895E2E0E093FB03E0E2F0E0EAA3C8
:10E99000FBA30895AE1BBF0BC5CAEE8DF0E0089532
:10E9A000E20FF31F3196FA93EA93ECA1FDA1E40F75
:10E9B000F51F31960C94E86CECA1FDA1E40FF51F56
:10E9C0000C94E86CE9A1F0E0DE0116960895ED8D57
:10E9D000EA930E94A043E9A1EF5FE9A30895E40F41
:10E9E000F51FDF01ECA1FDA112CEED8BFE8BAB89F3
:10E9F000BC8998CAA98DBA8DEA0FFB1F0895E98FCB
:10EA0000FA8FEB89FC89AF89B88DEA0FFB1FEF8B7A
:10EA1000F88FED89FE89AD89BE890E947C790E94BC
:10EA20003E790E94D97AEE87FF87688B798BEB89D4
:10EA3000FC89AB89BC890E947C790E943E790E9446
:10EA4000D97AAE85BF85888999890E94AF7BEA878C
:10EA5000FB876C877D8700E010E00895F8010E9435
:10EA60003E790E94D97A0DD911D906D90E94617BCD
:10EA7000AA85BB858C859D850E94617BAE85BF85FF
:10EA8000888999890E943D7A0E940C7B0E94A27A13
:10EA9000AF015A934A930C948669E98DFA8DE21B73
:10EAA000F30BFA93EA930895E98DFA8DE01BF10BCD
:10EAB000FA93EA930895F901AD8DBE8DEA0FFB1F1D
:10EAC000FA93EA930895ED8DFE8DE01BF10BFA9316
:10EAD000EA93EA8DEA930C949A64F801AD8DBE8DA9
:10EAE000EA0FFB1FFA93EA93EA8DEA930C949A6477
:10EAF000EA0FFB1FFA93EA9308951A930A93E091A1
:10EB0000D809E0300895E852F64FE081E0300895EA
:10EB1000E852F64FE1CAE852F64FE0810E0F1F5F50
:10EB20000895E091CC0BA091CB0BEA170895E091EA
:10EB3000A807A9E0EA9FF0010895E081E05DEA936B
:10EB40000C94F25BA091BA0BB091BB0B0895E091CD
:10EB5000BC0BF091BD0BFA93EA930895E0E0EA93C1
:10EB60000E94F25B0C94C847EA930E94F25B0C94FB
:10EB7000C8470E94207AF096EA930E94745DE2E70B
:10EB8000EA930C94F25BE081EA930C94F25BEEE082
:10EB9000EA930C94F25BE2EBFBE177CB0E94215C01
:10EBA000EBE3EA930C94F25BEBE3EA930C94F25BF5
:10EBB0005A934A930E94D4190E2F003408951A9341
:10EBC000E985FA85FA93EA930895E458F84FA88501
:10EBD000B985A083B18355CCE2E5EA930C94F25B4E
:10EBE000EE81FF813196EE83FF8308951A93E091C1
:10EBF000D107E0531E2FE5EDF7E061CBE091A907C7
:10EC0000A091AA07EA170895E091AA07EA930E9443
:10EC10003C32E093AA070895E091AA07A9E0EA9F91
:10EC2000F0010895A0910C0BA5CDE0930C0BEAE246
:10EC3000EA930E94745DD0CFE0910C0BE05AEA9306
:10EC40000E94F25BA4CFD9011496EC9177CCF90124
:10EC5000A281B381BA93AA9308950E94215CEAE34A
:10EC6000EA930C94F25BD9011196E0E0EC930E94D8
:10EC70008E5DCACFE05DEA930C94F25BEA930E944A
:10EC8000745DAACFFA93EA930C94AE5CE093060C01
:10EC9000F093070CE2E0E093CE07D9011196EC93D4
:10ECA0000895FA93EA937ACFE881F981FA93EA9387
:10ECB0000E94215CECE2EA930C94F25BF4DAAC91F2
:10ECC000A0330895A091F60AB091F70AE0E0EC9322
:10ECD0000895EE81FF81E093BC0BF093BD0B109380
:10ECE000B90B0E94861DE1E3089541E050E00E94C7
:10ECF000505BE887F987EAE3EA930E94E15AE13042
:10ED000008951A93E985FA8532CEE2E2EA930C94EB
:10ED1000E15AC9DAAC91A0320895C5DAAC91AB33AF
:10ED20000895C1DAEC91EA930895EAE3EA930E9428
:10ED3000E15AE13008950E94505BE058FF4F08957A
:10ED4000EFEFE093F00AE093F10A0895E0E0E0933A
:10ED50000B0CE0930C0C08950E94505B3197E093EC
:10ED6000D80AE091F10AA091D80AEA1708950E9402
:10ED70008050E091D80AEA930895E091D80AE09390
:10ED8000F10A0895E091D80AF0E0E35BF94F0895A5
:10ED9000ECE2EA930E94E15AE0300895E452F54F24
:10EDA0000F0181DAEC91D001EC931F5F41CBE4526B
:10EDB000F54FA0E0A0830895EA930E94E15AE13064
:10EDC0000895ECEDFAE0FA93EA930895E091D90AF8
:10EDD0000C94C06BE091D90AEF5FE093D90A0895D3
:10EDE000ABE3BBE0E091D90ABEC8A2E3BBE0E0918F
:10EDF000D90A0C94546EFA93EA930C94FE4CE09169
:10EE0000D80AA6E1EA9FF001E854FF4F0895FA936B
:10EE1000EA930C94215C0E94215CECE2EA930C944E
:10EE2000F25BECE2EA930C94F25B0E94F34CE0E0BC
:10EE3000E093D90A0895E091D90A0C94546EE091B8
:10EE4000F80AF091F90A0895A6EFBAE00C94B36CB1
:10EE5000A091F60AB091F70AEC93F6CFA091F60ACA
:10EE6000B091F70A13970895E0E0EA930E94574D96
:10EE7000E093CD070895AA81BB81EC91E295E07FF4
:10EE8000AE2FEC810895EA0FAA81BB81EC93A88193
:10EE9000B981EC91EF5F0895E091AA0CA091A90CC3
:10EEA000EA170895E091D308F0E0E852F74F08958B
:10EEB0001083E091D308EF5FE093D308E12FA09196
:10EEC000D5080895E093D508E091D408E150E09387
:10EED000D408E0300895E852F74FA0E0A0830895E9
:10EEE000E091750DF091760D0895A091730DB0919C
:10EEF000740DEA17FB070895E12FA0917A0DEA0F30
:10EF0000E0937A0DE0917C0D0895F0E0E053F84F26
:10EF100010830895E091810EF0E0E058F24FE08117
:10EF2000E0939C00E091810EEF5FE093810E0895E5
:10EF30000E94047C00E010E00895B5D9AC91AA339A
:10EF40000895B1D9EC912ECBE12FA981BA810C940F
:10EF5000C06BEA930E94F25B1F5F0895E452F54F85
:10EF6000E081E0300895E881EA930C94F25BE88157
:10EF7000F9816A817B810E94337A0895EA930E9425
:10EF8000E961EA930C94E657EA930E94D95EEAE5B8
:10EF9000E093D6080895EA930E947F60E0300895D8
:10EFA000E0917100E87F1E2F0895E0937300E4E87C
:10EFB000F2CF0A930E945860E0300895FF27662739
:10EFC00077270E94D97A0895EE8DAE85BF8588890E
:10EFD0009989F4DF0E94617BA9A1BAA188279927AA
:10EFE0000E943A7A0E943D7A0E940C7B08950E940A
:10EFF0003D7A0E940C7B0895E2E1F0E0FA93EA93F7
:10F000000895FA93EA930C946D62E8E2F0E00C94B0
:10F01000EC6C0E94027CEE81A6E5B9E10C94B36F22
:10F02000E2E0EA93EE85FF850E943379EACFAE8570
:10F03000BF85AE0FBF1FFD010E943379E2CFE6E02E
:10F04000EA93EC85FD850E943379DBCFAC85BD85E5
:10F05000AE0FBF1FFD010E943379D3CF0E946D62B6
:10F06000E5E0EA9308950E946D62E8E0EA930C946B
:10F070001A6C0E946D62E9E0EA930895EFE3F1E013
:10F08000C0CFEB85FC85AF81B885AE17BF0708956B
:10F090000D851E85ED85FE85E987FA870D871E871C
:10F0A0000B851C85EB85FC85EF83F8870B871C8718
:10F0B00008950E943379A5CFEA93EC85FD85F07021
:10F0C000A0CFEA93EE85FF85F0709BCFED85FE859E
:10F0D000A985BA85AE17BF070895AD85BE85E985B8
:10F0E000FA85EA1BFB0B0895FA93EA930C94216AC4
:10F0F000AB85BC8511CCAF81B885EB85FC85EA1B5F
:10F10000FB0B0895D9010E947C790F010895D0016D
:10F110000E94A779AF01E2E0EA93FA0188CFE3E029
:10F12000EA93FA01AE85BF85AE0FBF1FEFEFF0E0A7
:10F13000EA23FB2366CFA21BB30BEFEFF0E0EA2339
:10F14000FB235FCFE2E2EA931A930A930C946D6279
:10F15000AC85BD85AE0FBF1FEFEFF0E0EA23FB23C8
:10F1600050CFA985BA85ED85FE85EA1BFB0B089576
:10F17000D0010E94A779AF01E2E0EA9308952A93B3
:10F18000ED89FE89FA93EA93FE017596FA93EA9364
:10F190000C947B67EE89FF893497EE8BFF8B089583
:10F1A000ED89FE89FA93EA93FE017596FA93EA9344
:10F1B0000C947B67AE89BF8914960E94207AEE83F7
:10F1C000FF8377CAE885F9856A857B85AC85BD852F
:10F1D0008E859F8508950E949D69E883F9836A83DF
:10F1E0007B830895E881F9816A817B810895EA81B2
:10F1F000FB816C817D810895E991F991309639F018
:10F2000080EA9FE00197F1F7A8953197C9F7089533
:10F210000024AF0DB01D0895EA0FFB1F681F791F72
:10F220000895EA1BFB0B680B790B0895F195E195A6
:10F23000F0400895F09560957095E195FF4F6F4F00
:10F240007F4F0895EE230E2EEA2F19F0EE0F0A9449
:10F25000E9F70895EE0FFF1FEE0FFF1FEE0FFF1FE0
:10F26000EE0FFF1F0895EF2FFF27E7FDFFEF089533
:10F27000FE2FFF0FFF0B6F2F7F2F08956F2F660F4D
:10F28000660B762F0895BA2FBB0FBB0B8B2F9B2FCE
:10F2900008958B2F880F880B982F0895EA17FB0786
:10F2A000E1E00CF0EE270895FA9FF02DEB9FF00DB2
:10F2B000EA9FE02DF10D08957A9F702D6B9F700DE0
:10F2C000F89F700DE99F700D6A9F602D710DFB9F77
:10F2D000600D711DE89F600D711D8827FA9FF02D4C
:10F2E000610D781FEB9FF00D611D781FEA9FE02DE7
:10F2F000F10D681F781F089582D0D6DF0EF496DFD7
:10F3000008958BD0D9DF0EF495DF0895002498E09E
:10F31000AA0F001C0E1A10F40E0E01C0A1609A95DF
:10F32000B9F7EA2FA02D08950024112490E1AA0F27
:10F33000BB1F001C111C0E1A1F0A18F40E0E1F1EF4
:10F3400001C0A1609A9599F7FD01D001089557D0A9
:10F35000EBDF0EF46BDF08953F934F935F93002430
:10F3600011244427552730E2AA0FBB1F881F991F7D
:10F37000001C111C441F551F0E1A1F0A460B570B69
:10F3800028F40E0E1F1E461F571F01C0A1603A959C
:10F3900059F7FD01BC01D001CA015F914F913F9126
:10F3A00008953BD0D9DF0EF445DF0895AFDFEA2F93
:10F3B0000895E894B7FF04C0A095B095119668949D
:10F3C000F7FD34DFB1DFFD010EF430DF0895C4DF57
:10F3D000FD01BC010895E89497FF09C0A095B09580
:10F3E00080959095AF5FBF4F8F4F9F4F689477FD8B
:10F3F00021DFB2DFFD01BC010EF41CDF0895E894AB
:10F40000F7FF02C013DF6894B7FF06C0A095B09560
:10F41000119600F8039400FA0895E89477FF02C06B
:10F4200009DF689497FF0BC00024A095B0958095E4
:10F4300090951196801D901D00F8039400FA089590
:10F44000ED91FC9111970895ED91FD916D917C9155
:10F4500013970895ED93FD936D937C930895059014
:10F46000F491E02D08957A936A93FA93EA930895BC
:10F47000689401C0E89401D09DD0182E862F612D8C
:10F48000192E972F712D1B2EBF2FF12D1A2EAE2F57
:10F49000E12D0895119602D0FE2F1197E199FECF2C
:10F4A000FF93FFB7F894AEBBBFBBE09AEDB3FFBFCD
:10F4B000FF91089507D01196EF93EF2F03D0EF91AE
:10F4C00011970895E19B02C0A895FCCF9FB7F894CF
:10F4D000AEBBBFBBE09A8DB3E81719F0EDBBE29A63
:10F4E000E19A9FBF0895552342F4503811F4E0FF8C
:10F4F00004C03196691F791F6BF050E8572711F44B
:10F500005F93CDC05F3F31F0660F000C5795679554
:10F51000752F08955F9300200AF0CDC0C6C050E853
:10F52000192E1522880F991F9527550F879550E89A
:10F53000072E0522660F771F7527550F67950895CB
:10F54000689401C0E8945F93F2DF703818F07F3F51
:10F5500008F4A5C056E1571BAAF4519558300EF493
:10F56000593030F0EFEFFFEF6FEF7FE777F91AC018
:10F5700077275523B9F0EE0FFF1F661F771F5A95A7
:10F58000D1F710C07727583028F0EF2FF62F672FCC
:10F590005850F9CF552331F076956795F795E79553
:10F5A0005A95D1F700200AF445DE5F9108956894DA
:10F5B00001C0E894309760407040B1F0002426F01C
:10F5C000772312F4009436DE172E7EE1112032F0FC
:10F5D0007A95EE0FFF1F661F111CF9CFEF2FF62F44
:10F5E000612D5F938ADF5F9108954F93AF01FD0115
:10F5F000DA01AB01BC01CA01402D012C142E4F9140
:10F600000895EA0FFB1F681F0895E095F095609537
:10F61000EF5FFF4F6F4F08955F9381DF903871F177
:10F6200050E8152604C05F937ADF903839F17038BE
:10F6300021F1572F591B13F112F4D7DFFACF5831AC
:10F6400018F0AA27BB278827583028F0AB2FB82FEF
:10F6500088275850F9CF552329F08695B795A79557
:10F660005A95D9F7502D512562F0CBDF38F46795C4
:10F67000F795E795739513F41EC0B7DF3EDF5F91F2
:10F680000895EA1BFB0B680B51F010F40094BDDFEA
:10F690006623A2F3EE0FFF1F661F7A95CBF7EE27C6
:10F6A000FF27662777275F910895EFEFFFEF6FE75A
:10F6B0007FEF5F910895EFEFFFEF6FE77FE75F91D7
:10F6C00008955F932CDF703851F3903841F3012493
:10F6D0000894791F23F41CF300203AF3ECCF0F9227
:10F6E0001F932F933F934F93112722279927689FAA
:10F6F000A0018F9F302D410D591F6B9F300D411D73
:10F70000591F8E9F27D0BF9F25D06A9F23D0BE9FB1
:10F710001DD0AF9F1BD0AE9F110D291F391F491F50
:10F72000591FE32FF42F652F522F4F913F912F91A7
:10F730001F910F9066232AF0550FEE1FFF1F661FC3
:10F7400002C073954BF2CFDE5F910895100D211D1D
:10F75000391F02C0200D311D491F591F08955F93A5
:10F76000DEDE703821F411200AF49FCFA4CF903848
:10F7700009F495CF01240894970B1BF4D4F30020CF
:10F78000F3CF792F1F932F933F934F93112411277A
:10F79000222733274427552790E2AE17BF07860755
:10F7A000410730F0AE1BBF0B860B410B089401C024
:10F7B0008894551F221F331F111CAA1FBB1F881FAF
:10F7C000441F9A9551F7F901612D4F913F912F9167
:10F7D0001F91662332F0550FEE1FFF1F661F7A95AB
:10F7E00043F281DE5F910895309760407040089544
:10F7F00000240A160B06089500240A160B060806B4
:10F80000090608955A934A933A932A931A930A93AE
:10F8100008955D814C813B812A8119810881089579
:00000001FF
